:020000040800F2
:1000000000000120E9450008B5270008B7270008CF
:10001000B9270008BB270008BD2700080000000022
:10002000000000000000000000000000BF270008E2
:10003000C127000800000000C3270008C5270008EA
:100040003946000839460008C92700083946000823
:100050003946000839460008D5270008DB27000884
:1000600039460008394600080D28000839460008BE
:10007000E1270008E3270008E5270008F12700082A
:10008000FD270008092800083946000839460008FD
:1000900000000000394600080F2800083946000813
:1000A0003946000839460008394600083946000834
:1000B0003946000839460008394600083946000824
:1000C0003946000839460008394600083946000814
:1000D0003946000815280008394600083946000846
:1000E0003946000811280008212800083946000870
:1000F00039460008000000000000000039460008F2
:1001000039460008394600082D28000839460008FD
:1001100039460008394600083946000839460008C3
:1001200039460008394600083946000839460008B3
:080130003946000839460008B9
:1001380010B5054C237833B9044B13B10448AFF319
:1001480000800123237010BD4C0100200000000036
:100158001814010808B5034B1BB103490348AFF352
:10016800008008BD0000000050010020181401089C
:1001780014214160704714207047406A704700009E
:10018800790100087F01000883010008990100082F
:1001980010B5044604F1100000F05CFCC4F8F80047
:1001A8000148C4F87C0110BD88010008F8B5E6B024
:1001B80004460D4616461F460A4906A800F0CAFE20
:1001C80070996F9A05910492009733466E996D9ACB
:1001D800039102922A466C990191214600F060F839
:1001E80067B0F0BD94010008F8B5E6B004460D46C6
:1001F80016461F46094906A800F0ACFE6F996E9A8C
:100208000491039200976D996C9A0291019233467A
:100218002A46214600F087F867B0F0BD940100082F
:1002280038B500281CBF01680029184A23D1184B8B
:100238001C684FF6F0710C404CF24025AC421FBFD1
:100248001B6819404CF27024A14212D1114D296843
:1002580079B911490B68C3F30B03B3F58A6F1FBF54
:100268000968C1F30B0140F28343994204BF01219D
:10027800117028B905E0094B994204BF012111709A
:100288004068BDE8324001F09FBE00BF6801002011
:1002980000ED00E0002004E00010005C000037489A
:1002A8002DE9F04104460D46216816464A681F4666
:1002B80090478046B8F5403F2ED122680A99936846
:1002C800204698478046B8F5403F25D12368089ACC
:1002D8000799D3F80CC02046E0478046B8F5403F60
:1002E8001AD12368069A39461F692046B8478046BE
:1002F800B8F5403F10D1236829465D69324620464B
:10030800A8478046B8F5403F06D123680B9A09995B
:100318009D692046A847804621680A68204690477C
:100328004046BDE8F0812DE9F04104460D462168BC
:1003380016464A681F4690478046B8F5403F2ED17A
:1003480022680A999368204698478046B8F5403F46
:1003580025D12368089A0799D3F80CC02046E047AE
:100368008046B8F5403F1AD12368069A39461F6976
:100378002046B8478046B8F5403F10D12368294643
:100388005D6932462046A8478046B8F5403F06D109
:1003980023680999DD6900222046A847804621681C
:1003A8000A68204690474046BDE8F0814FF4403047
:1003B80070470000F0B50C4685B0114600281A4673
:1003C8001CBF0568002D0B4B11D082B104B971B95F
:1003D8000D9860B10F9E0E9F0A9B0290049603979A
:1003E8000B980C9E009001962046A8470346184695
:1003F80005B0F0BD020003002DE9F04F0646D0B06D
:100408000868F56DD6F860E0726EB76EF36E00BAE4
:1004180000906C46486800BA60600DF14008886832
:1004280000BAA060C86800BAE060086900BA206134
:10043800486900BA6061886900BAA061C86900BAF1
:10044800E061086A00BA2062486A00BA6062886A95
:1004580000BAA062C86A00BAE062086B00BA2063FA
:10046800486B00BA6063886B00BAA063C86B00BAB7
:10047800E063402058F80C1C58F820CC58F838ACE9
:100488008CEA010158F840CC8AEA01018CEA01099A
:100498004FEAF979401E48F8049BEBD187EA02003D
:1004A80000EA0E00784010EBF5610098DFF824C4EC
:1004B80041186144C81882EABE032B404FEAF06134
:1004C80053405918636859186144CF194FEAB50366
:1004D80083EABE01014081EABE0111EBF765A1681C
:1004E8004D196544A91883EAB0023A404FEAF1650C
:1004F8005A405519E26855194FEAB70282EAB0071F
:1005080065440F4005EBBE0E97EAB00717EBFE6592
:1005180027697D194FEAB10782EA0701654401EAB4
:100528000E01EB18514011EBF36561694D194FEA63
:10053800BE0187EA010E65440EEA030E15EBB00012
:100548008EEA070E0EEBF065D4F818E075446544A2
:10055800AA1881EAB30505404FEAF26E4D40AE4451
:10056800E569AE44E64477444FEAB00080EAB30E4A
:100578000EEA020E8EEAB30E0EEBF765D4F820E011
:1005880075446544691880EAB2053D404FEAF16E4A
:100598004540AE44656AAE44E6440EEBB3034FEA09
:1005A800B70787EAB20E0EEA010E8EEAB20E0EEB1C
:1005B800F365D4F828E075446544281887EAB1053E
:1005C8001D404FEAF06E7D40AE44E56AAE44E64415
:1005D8000EEBB2024FEAB30383EAB10E0EEA000E45
:1005E8008EEAB10E0EEBF265D4F830E0754465443E
:1005F800EF1983EAB00515404FEAF76E5D40AE4447
:10060800656BAE44E6440EEBB1014FEAB20282EAF2
:10061800B00E0EEA070E8EEAB00E0EEBF165D4F8B6
:1006280038E075446544EB1882EAB7050D404FEA97
:10063800F36E5540AE44E56BAE44E6440EEBB000B5
:100648004FEAB10181EAB70E0EEA030E8EEAB70E41
:100658000EEBF065D4F840E07544654481EAB30ECA
:10066800AA180EEA000E4FEAF2658EEA010E7544EA
:10067800DDF844E04FEAB000754480EAB30E654403
:100688000EEA020E15EBB7078EEAB30E0EEBF7650E
:10069800DDF848E04FEAB202754480EA020E65448C
:1006A8000EEA070E69188EEA000E0EEBF165DDF80A
:1006B8004CE07544654405EBB3034FEAB70E1427C5
:1006C8000DF1500CDFF810528EEA010B82EA0B0B89
:1006D8000BEBF36A5CF804BBDA44AA44504483EA9F
:1006E800B10B4FEAF06A8EEA0B0BDA445CF804BBF4
:1006F800DA44AA44524480EAB30B4FEAF26A8BEA1E
:10070800B10BDA445CF804BBDA444FEAB000AA44FF
:1007180080EA020BD6448BEAB30B0BEBFE6A5CF85B
:1007280004BBDA444FEAB202AA4482EA0E0B0AEB8F
:10073800B10180EA0B0B0BEBF16A5CF804BBDA44FD
:100748007F1DAA44282F0AEBB3034FEABE0EBBD382
:100758003C2F61D3502F4DD204EB870CC7F15407BF
:100768005E4CA7FB04A504465D4FA8088EEA010A63
:1007780082EA0A0A5CF804BB0AEBF3655D447D195A
:100788002C1983EAB10A4FEAF4658EEA0A0A55443D
:100798005CF804AB5CF804BB55447D19AA1884EADC
:1007A800B30A4FEAF2658AEAB10A55445D444FEA52
:1007B800B4047D1984EA020AAE448AEAB30A0AEB51
:1007C800FE655CF804AB55444FEAB2027D1982EA33
:1007D8000E0A15EBB10184EA0A0A5CF804BB0AEBBD
:1007E800F1655D447D1915EBB303401E4FEABE0E5B
:1007F800BCD12046F46D1B19F365336EC9183166F8
:10080800716E71447166B36ED218B266F16E40189B
:10081800F06650B0BDE8F08F4EEA010B0EEA010A0F
:100828000BEA020B4BEA0A0A0AEBF36554F827A015
:10083800DFF8B0C0554443EAB10B654403EAB10A96
:100848000BEA0E0B28184BEA0A0A7F1C0AEBF06524
:1008580054F827A0554440EAB30B654400EAB30AAC
:100868000BEAB10BAA184BEA0A0A7F1C0AEBF265DD
:1008780054F827A055444FEAB00040EA020B6544FB
:1008880000EA020A0BEAB30BAE444BEA0A0A7F1CE1
:100898000AEBFE6554F827A055444FEAB20242EA33
:1008A8000E0B654402EA0E0A0BEA000B15EBB101C8
:1008B8004BEA0A0A7F1C0AEBF16554F827A0554455
:1008C8007F1C65443C2F05EBB3034FEABE0EA3D350
:1008D80040E700BF9979825AA1EBD96ECDCCCCCC38
:1008E800D6C162CADCBC1B8F00B581B00168074A5B
:1008F800914200D110B9064801B000BD7C2110F02A
:10090800EFFC4FF4003001B000BD00BFFC09000847
:10091800030002002DE9F0410B4A92E8F85188B033
:10092800694681E8F8510268084B9A4200D118B923
:10093800074808B0BDE8F0811422083000F04FFBEA
:1009480008B0BDE8F08100BFDC090008FC09000818
:1009580003000200152904D20268044B9A4200D110
:1009680008B903487047083000F048BBFC09000884
:100978000300020010B481B013460268074CA2427B
:1009880000D118B901B010BC0548704701B000F19A
:10099800240210BC083000F035BB00BFFC09000879
:1009A8000300020010B481B013460268074CA2424B
:1009B80000D118B901B010BC054870470A4601B00B
:1009C80000F1240110BC083000F070BBFC090008DD
:1009D800030002000123456789ABCDEFFEDCBA981E
:1009E80076543210F0E1D2C300000000000000008D
:1009F80000000000F10800081D0900085D09000852
:100A08007D090008AD09000801040008790F0008F5
:100A1800C50F0008810F0008F0B5A3B004460B48C5
:100A280002900D4616461F46094B0822402104A88D
:100A380000F0D1FA28980190009733462A462146BB
:100A480002A800F01BF823B0F0BD00BFFC090008A5
:100A5800100A000810B5040008BF002408D0054893
:100A6800054B20600822402104F1080000F0B3FA89
:100A7800204610BDFC090008100A00082DE9F041C5
:100A880004460E46216817464A681D469047804628
:100A9800B8F5003F19D1226806999368204698470F
:100AA8008046B8F5003F10D123683146DE683A46E3
:100AB8002046B0478046B8F5003F06D12368079A1C
:100AC80029461D692046A847804621680A682046AD
:100AD80090474046BDE8F08110B500F033FA4FF476
:100AE800403400280EBF034C4FF4C07110F0F8FBDF
:100AF800204610BD0200030010B5044600F022FA9B
:100B080008B9054810BD0021A160D0F87C21116802
:100B180088474FF4403010BD0200030070B504460A
:100B28000D4600F00FFA064E40B1D0F87C0141683E
:100B38008847A84224BF65604FF44036304670BDF0
:100B4800020003002DE9FF4715000C4600D02CB128
:100B5800064600F0F7F95FEA000801D16448C3E0EF
:100B6800D8F8F80001684A689047B0F5003F17D1F7
:100B7800D8F87C118A68404690478146B9F1810FC0
:100B880080F09E80A94508F1FC0A17D2D8F8F80031
:100B98000368D3F80CC02A462146E047B0F5003F69
:100BA80040F08E80D8F8F8000368D3F810C06A4681
:100BB8005146E047B0F5003F76D10AE0002004E056
:100BC800215C0AF800100098401C00900098A84288
:100BD800F6D34FF0000C4749474A484B01AC009800
:100BE800844558D2D3E9007001ADC5E9007010788A
:100BF80000281ABF042086464FF0000E085854F803
:100C08000E5028443E4D05600127D0F800E087606B
:100C1800019D4F681AF80C007D408EEA050585F0A5
:100C2800040E65680F687D4085F0FC05754485F005
:100C3800A30568400AF80C000CF1010CCFE7D3E9D2
:100C4800004501A8C0E9004510782E4D002814BFC2
:100C58004FF0040E4FF0000E01A8744651F80EE054
:100C68000459A6440127CEF80050DEF80040CEF81B
:100C780008704D68019F40687D406C400D68684071
:100C880084F0040480F0FC00041984F057040AF886
:100C98000C400CF1010CCC45D1D3D8F8F800016810
:100CA8004A689047B0F5003F0AD1D8F8F8000368C1
:100CB800D3F80C804A465146C047B0F5003F01D0F2
:100CC800114811E0002006E05AF8201081F06A313E
:100CD8004AF82010401CB0EB990FF5D3B06840F0EB
:100CE8000100B0604FF4403004B0BDE8F08700BFA9
:100CF80002000300B014010868010020240F000856
:100D0800ADBE4ED70DBE75A10100030038B50C4627
:100D1800017A1546CA0702D500F014F908B908483F
:100D280032BDD0F8F80003682146DC682A46A0479F
:100D3800B0F5003F01D0034832BD4FF4403032BD1A
:100D480002000300010003002DE9F84191B00546B7
:100D58000E461746402101A810F0C2FA297AC807A2
:100D680004D5284600F0EEF8040002D1DFF8A4808C
:100D78004BE0D4F8F800DFF8A0800368D3F810C07F
:100D88006A4601A9E047B0F5003F3ED1D4F8F80023
:100D980001684A689047B0F5003F36D1D4F87C1115
:100DA8008A6820469047D4F8F830024618461B68EF
:100DB800D3F80CC004F1FC01E047B0F5003F24D1A2
:100DC800D4F87C0141688847D4F8F83002461846C0
:100DD8001B68D3F80CC001A9E047B0F5003F14D157
:100DE800D4F8F8000268696893689847B0F5003F3E
:100DF8000BD1D4F8F80003681C693A463146A0477D
:100E0800B0F5003F08BF4FF44038404612B0BDE887
:100E1800F08100BF02000300010003002DE9F84142
:100E2800A5B0074688461646402115A810F058FA7E
:100E380000220492402105A810F052FA387AC1071E
:100E48005ED5384600F07EF8050059D0D5F8F80090
:100E58002D4C0368D3F810C06A4605A9E047B0F5E1
:100E6800003F3CD1D5F8F80001684A689047B0F5D2
:100E7800003F34D1D5F87C118A6828469047D5F8C8
:100E8800F830024618461B68D3F80CC005F1FC017F
:100E9800E047B0F5003F22D1D5F87C01416888478A
:100EA800D5F8F830024618461B68D3F80CC005A9D7
:100EB800E047B0F5003F12D1D5F8F800026879682C
:100EC80093689847B0F5003F09D1D5F8F800036852
:100ED8001D6904AA15A9A847B0F5003F01D020460E
:100EE8000FE00A4B0A490B4A0396029101924046C9
:100EF8001C68049B009415AA796800F0E5F900E0E5
:100F0800054826B0BDE8F08101000300B8140108C7
:100F1800936E030026C703000200030004B001011A
:100F280000170145E10A0008010B0008250B00081D
:100F3800B50300084D0B0008150D0008510D0008F9
:100F4800250E00080168024A914218BF0020704728
:100F58002C0F000810B5040008BF002404D0034873
:100F68002060204609688847204610BD2C0F0008DD
:100F780020225C3010F0B2B9F0B58468A3080022D2
:100F880004F0030407E000F15C0555F8226035BA67
:100F980041F82250521C9A42F5D300220BE000F18E
:100FA8005C0502EB830755F82360D500C5F11805E9
:100FB800EE40CE55521CA242F1D3F0BD30B5C46804
:100FC80003690022E31AD5188C5C0544521C082AD0
:100FD8002C77F8D330BD0360C1600261704738B523
:100FE800044615460022626023685A68904700202C
:100FF8006061A061A5604FF4003032BD81604FF49C
:10100800003070472DE9F84304462079D4F80C8065
:10101800450748BF244845D466691D46A8F1010024
:1010280000EAD60306EBC506B6EBC50F666102D229
:10103800A669761CA6611746A66906EB5576A661D1
:101048000E46E918884225D2A8EB03094A463146DC
:10105800F81810F043F92268136839460FE0424641
:10106800384610F03BF923681A68394620469047FD
:1010780007E0311811F00300F1D122681368204607
:101088009847484600EB0809A9F10101A942F0D3A5
:10109800002300E000202A1A3118F81810F01EF971
:1010A8004FF40030BDE8F283040002002DE9FC4F44
:1010B800024685B0D0681369DFF86CC1DFF86C812F
:1010C800A0EB030A506840F004005060002703A812
:1010D80002900DF10C0ED8E9003403A8544DC0E974
:1010E80000342878534D00280CBF00230423994668
:1010F8005CF803305EF80940234401261D601C6833
:101108009E60DCF80430039DDCF80090DEF8046093
:101118005D406540484C654089EA0606474C664094
:101128007519474C6540D8E9006B03AC0028C4E941
:10113800006B0EBF002404200424029E5CF800000B
:10114800345920183F4C04600126046886600398CF
:10115800029E43406340384C7068634089EA00004F
:10116800364C6040034438484340280018BF0120EB
:101178005B1E9B41042F2CBFC0B2D80F02F1140391
:1011880053F8200007F00303C3F10303DB00D84042
:101198000DF807007F1C082F9DD315460C466A6979
:1011A800AB69E868D20842EA4372401E00EA0207C7
:1011B800002302409B420AD8524508D28020E055BD
:1011C8007F1C574516D2AAEB0701E01910E08020D2
:1011D800E05500E0E355E8687F1C8742FAD32A68A7
:1011E800136828469847BAF1000F03D051462046A5
:1011F80010F076F82A68069E059F93686946284687
:1012080098472A68D2F8009021462846C8472B6894
:10121800DA683946284690470EB1A86830604FF41E
:10122800003007B0BDE8F08FB01401085412000870
:10123800680100205FC5109304850012FC68017ADC
:10124800C0F524FF24AF33D426AF698B04B0010165
:1012580000170145F8B501240094002300240DE08F
:10126800009D065D0F5D7E40F643761CF60F86F006
:10127800010635400095641C009DEB189442EFD39D
:101288001846F2BDF8B5002301240094002A11E0A5
:10129800009C85188F1815F8016C17F8015C6E40D2
:1012A800F643761CF60F86F0010634400094009C45
:1012B800E318521EECD11846F2BD00005D1200087A
:1012C8008D120008010000002DE9F84F1D46DDF8D9
:1012D80028900B9F0D9C4FF0FF3300930E469246CB
:1012E800D9F800B0804632465146D847834664B3A1
:1012F800D9F8043032465146404698476FEA0B0207
:10130800521C42EA0B0200996FEAD2735B1C194027
:10131800C2430091521C024300996FEAD2735B1CCE
:101328001940009186F05531484087EA000181F064
:101338005531216080F05531C943491C0843009A52
:101348006FEAD070401C82430092D9F80800012847
:1013580009D17540E943491C0D4300986FEAD572DD
:10136800521C90430AE0F11C85EA9102D243521CB8
:10137800154300986FEAD5735B1C984386F0AA362C
:10138800009086EA0B0686F0AA33F243DB430C98FA
:10139800C2F3C0725B1C42EAD3720099D243521C5A
:1013A80091430091774000998843009987F0AA37C4
:1013B8000F403843BDE8F28F034613F8012B002A8B
:1013C800FBD1181A0138704781F0004102E000BFD4
:1013D80083F0004330B54FEA41044FEA430594EAED
:1013E800050F08BF90EA020F1FBF54EA000C55EA28
:1013F800020C7FEA645C7FEA655C00F0E2804FEAF9
:101408005454D4EB5555B8BF6D420CDD2C4480EADA
:10141800020281EA030382EA000083EA010180EA0A
:10142800020281EA0303362D88BF30BD11F0004F58
:101438004FEA01314FF4801C4CEA113102D040428E
:1014480061EB410113F0004F4FEA03334CEA1333C9
:1014580002D0524263EB430394EA050F00F0A780E1
:10146800A4F10104D5F1200E0DDB02FA0EFC22FADC
:1014780005F2801841F1000103FA0EF2801843FAD0
:1014880005F359410EE0A5F120050EF1200E012AC1
:1014980003FA0EFC28BF4CF0020C43FA05F3C018FF
:1014A80051EBE37101F0004507D54FF0000EDCF178
:1014B800000C7EEB00006EEB0101B1F5801F1BD321
:1014C800B1F5001F0CD349085FEA30004FEA3C0C25
:1014D80004F101044FEA445212F5800F80F09A801B
:1014E800BCF1004F08BF5FEA500C50F1000041EB1F
:1014F800045141EA050130BD5FEA4C0C404141EB23
:101508000101013C28BFB1F5801FE9D291F0000F1D
:1015180004BF01460020B1FA81F308BF2033A3F1CC
:101528000B03B3F120020CDA0C3208DD02F1140CC3
:10153800C2F10C0201FA0CF021FA02F10CE002F1FE
:101548001402D8BFC2F1200C01FA02F120FA0CFCF7
:10155800DCBF41EA0C019040E41AA2BF01EB045140
:10156800294330BD6FEA04041F3C1CDA0C340EDC3E
:1015780004F11404C4F1200220FA04F001FA02F381
:1015880040EA030021FA04F345EA030130BDC4F13F
:101598000C04C4F1200220FA02F001FA04F340EA34
:1015A8000300294630BD21FA04F0294630BD94F0E5
:1015B800000F83F4801306BF81F480110134013DCC
:1015C8004EE77FEA645C18BF7FEA655C29D094EA3D
:1015D800050F08BF90EA020F05D054EA000C04BFBB
:1015E8001946104630BD91EA030F1EBF00210020A6
:1015F80030BD5FEA545C05D14000494128BF41F045
:10160800004130BD14F580043CBF01F5801130BDA8
:1016180001F0004545F0FE4141F470014FF0000033
:1016280030BD7FEA645C1ABF194610467FEA655CE4
:101638001CBF0B46024650EA013406BF52EA033586
:1016480091EA030F41F4002130BD00BF90F0000F74
:1016580004BF0021704730B54FF4806404F13204B0
:101668004FF000054FF0000150E700BF90F0000F69
:1016780004BF0021704730B54FF4806404F1320490
:1016880010F0004548BF40424FF000013EE700BF60
:1016980042004FEAE2014FEA31014FEA02701FBFF0
:1016A80012F07F4393F07F4F81F06051704732F022
:1016B8007F4208BF704793F07F4F04BF41F4002179
:1016C800704730B54FF4607401F0004521F00041D7
:1016D8001CE700BF50EA010208BF704730B54FF061
:1016E80000050AE050EA010208BF704730B511F062
:1016F800004502D5404261EB41014FF4806404F19A
:1017080032045FEA915C3FF4D8AE4FF003025FEA1F
:10171800DC0C18BF03325FEADC0C18BF033202EBA3
:10172800DC02C2F1200300FA03FC20FA02F001FAFD
:1017380003FE40EA0E0021FA02F11444BDE600BFA0
:101748004FF0FF3C06E000BF4FF0010C02E000BF85
:101758004FF0010C4DF804CD4FEA410C7FEA6C5C68
:101768004FEA430C18BF7FEA6C5C1BD001B050EA0B
:10177800410C0CBF52EA430C91EA030F02BF90EAF6
:10178800020F0020704710F1000F91EA030F58BFB5
:10179800994208BF90422CBFD8176FEAE37040F017
:1017A800010070474FEA410C7FEA6C5C02D150EAB5
:1017B800013C07D14FEA430C7FEA6C5CD6D152EA70
:1017C800033CD3D05DF8040B704700BF8446104635
:1017D80062468C461946634600E000BF01B5FFF734
:1017E800B7FF002848BF10F1000F01BD4DF808ED04
:1017F800FFF7F4FF0CBF012000205DF808FB00BFD5
:101808004DF808EDFFF7EAFF34BF012000205DF82E
:1018180008FB00BF4DF808EDFFF7E0FF94BF01207B
:1018280000205DF808FB00BF4DF808EDFFF7CEFF7C
:1018380094BF012000205DF808FB00BF4DF808EDBB
:10184800FFF7C4FF34BF012000205DF808FB00BF8C
:101858004FEA410212F5001215D211D56FF47873D0
:10186800B3EB625212D94FEAC12343F0004343EA73
:10187800505311F0004F23FA02F018BF404270474E
:101888004FF00000704750EA013005D111F00040D8
:1018980008BF6FF0004070474FF00000704700BF6E
:1018A80080F0004002E000BF81F0004142001FBF0D
:1018B8005FEA410392EA030F7FEA226C7FEA236C16
:1018C8006AD04FEA1262D2EB1363C1BFD21841400B
:1018D80048404140B8BF5B42192B88BF704710F0A1
:1018E800004F40F4000020F07F4018BF404211F044
:1018F800004F41F4000121F07F4118BF494292EAAC
:10190800030F3FD0A2F1010241FA03FC10EB0C00D7
:10191800C3F1200301FA03F100F0004302D5494264
:1019280060EB4000B0F5000F13D3B0F1807F06D311
:1019380040084FEA310102F10102FE2A51D2B1F109
:10194800004F40EBC25008BF20F0010040EA0300FE
:101958007047490040EB0000013A28BFB0F5000F7E
:10196800EDD2B0FA80FCACF1080CB2EB0C0200FA34
:101978000CF0AABF00EBC25052421843BCBFD04083
:101988001843704792F0000F81F4000106BF80F4FD
:1019980000000132013BB5E74FEA41037FEA226CC0
:1019A80018BF7FEA236C21D092EA030F04D092F08B
:1019B800000F08BF0846704790EA010F1CBF0020BF
:1019C800704712F07F4F04D1400028BF40F000401C
:1019D800704712F100723CBF00F50000704700F03C
:1019E800004343F0FE4040F4000070477FEA226263
:1019F80016BF08467FEA23630146420206BF5FEA34
:101A0800412390EA010F40F4800070474FF0000333
:101A180004E000BF10F0004348BF40425FEA000CFA
:101A280008BF704743F0964301464FF000001CE0A2
:101A380050EA010208BF70474FF000030AE000BFF8
:101A480050EA010208BF704711F0004302D5404236
:101A580061EB41015FEA010C02BF844601460020A8
:101A680043F0B64308BFA3F18053A3F50003BCFAC3
:101A78008CF2083AA3EBC25310DB01FA02FC634470
:101A880000FA02FCC2F12002BCF1004F20FA02F277
:101A980043EB020008BF20F00100704702F120026A
:101AA80001FA02FCC2F1200250EA4C0021FA02F2CB
:101AB80043EB020008BF20EADC7070474FEA40029F
:101AC800B2F1FE4F0FD34FF09E03B3EB12620DD964
:101AD8004FEA002343F0004310F0004F23FA02F0CE
:101AE80018BF404270474FF00000704712F1610F75
:101AF80001D1420205D110F0004008BF6FF000404C
:101B080070474FF00000704753B94AB9002908BF21
:101B180000281CBF4FF0FF314FF0FF3000F070B9C4
:101B2800ADF1080C6DE904CE00F006F8DDF804E02C
:101B3800DDE9022304B070472DE9F047089E0D4601
:101B480004460F46002B4AD18A42944665D9B2FA18
:101B580082F343B102FA03FCC3F120029F4020FA4A
:101B680002F217439C404FEA1C4E1FFA8CF5B7FB54
:101B7800FEF1220C0EFB117742EA074201FB05F049
:101B880090420AD91CEB020201F1FF3780F01B8159
:101B9800904240F2188102396244121AA4B2B2FB90
:101BA800FEF00EFB102244EA024400FB05F5A542B4
:101BB8000AD91CEB040400F1FF3280F00681A5422B
:101BC80040F203816444023840EA0140641B00216A
:101BD8001EB1DC400023C6E90043BDE8F0878B4214
:101BE80008D9002E00F0EC800021C6E9000508465F
:101BF800BDE8F087B3FA83F1002949D1AB4202D39B
:101C0800824200F2F780841A65EB0302012017462E
:101C1800002EE2D0C6E90047DFE702B9FFDEB2FADC
:101C280082F3002B40F08F808A1A4FEA1C471FFA74
:101C38008CFE0121B2FBF7F507FB1520220C42EAC6
:101C480000420EFB05F0904208D91CEB020205F198
:101C5800FF3802D2904200F2CA804546121AA4B256
:101C6800B2FBF7F007FB102244EA02440EFB00FE29
:101C7800A64508D91CEB040400F1FF3202D2A645A0
:101C880000F2BA801046A4EB0E0440EA05409FE734
:101C9800C1F120078B4022FA07FC4CEA030C05FA35
:101CA80001F420FA07F3FD40234300FA01F94FEA53
:101CB8001C401FFA8CFEB5FBF0F81C0C00FB1855F5
:101CC80044EA054408FB0EF5A54202FA01F20BD9D5
:101CD8001CEB040408F1FF3A80F08780A54240F22B
:101CE8008480A8F102086444641B9DB2B4FBF0F33D
:101CF80000FB134445EA044403FB0EFEA64508D93D
:101D08001CEB040403F1FF306BD2A64569D9023BF2
:101D1800644443EA0840A0FB0283A4EB0E049C42FF
:101D2800C6461D4655D352D056B1B9EB0E0364EBE7
:101D3800050404FA07F7CB40CC401F43C6E90074FA
:101D48000021BDE8F087C3F1200102FA03FC20FA64
:101D580001F225FA01F19D402A434FEA1C471FFA78
:101D68008CFEB1FBF7F007FB1015110C41EA054199
:101D780000FB0EF58D4204FA03F408D91CEB0101AF
:101D880000F1FF382FD28D422DD902386144491B0A
:101D980092B2B1FBF7F507FB151142EA014205FBC8
:101DA8000EF1914208D91CEB020205F1FF3816D258
:101DB800914214D9023D6244521A45EA004139E77A
:101DC8003146304609E73946E7E61046FCE6C145A4
:101DD800AAD2B8EB020E63EB0C050138A4E745461E
:101DE800EAE7034695E74046D1E7D0467CE7023D5F
:101DF800624433E708460BE76444023843E700BF10
:101E0800704700BF1348144A08B54FF00043C0E9B3
:101E180000230422002342610122C2614FF4805151
:101E280007220383C0E90233C0E90933C0E90C1271
:101E38000361837680F8203080F82C30826380F844
:101E48003C30C36402F04AFC18B1BDE8084000F019
:101E580009BC08BD6C010020002401400268084B41
:101E68009A4282B00AD14FF0B0431A6E42F400721F
:101E78001A661B6E03F400730193019B02B070474E
:101E8800002401400268054B9A4201BF4FF0B0425E
:101E9800136E23F400731366704700BF00240140DB
:101EA80030B585B000240546CDE901440394FFF719
:101EB800A9FF144802F0AAFF08B100F0D3FB1148AB
:101EC800039401A9CDE9015402F066FD08B100F0C0
:101ED800C9FB0C4802F0C4FE08B100F0C3FB4FF088
:101EE800FF31084802F0FAFC064802F071FF054885
:101EF80002F04EFD0446034802F014FF204605B0E8
:101F080030BD00BF6C010020014B024A1A607047C7
:101F18006C0100200024014008B50948FFF7C0FF04
:101F280068B1084BB3F8AA304FF6FF72934216BF58
:101F380040F6E442044B5343B3FBF0F398B208BDB8
:101F4800002000B40075FF1FD8084C0013B500230B
:101F5800ADF80630FFF7E0FF04461948FFF7A0FF89
:101F6800184BB3F8C820B3F8A8108A4204FB00F055
:101F780018D040F6E443B0FBF3F364205B1A434304
:101F8800521A93FBF2F31E331BB2ADF80630BDF8BC
:101F980006305BB21B02ADF80630BDF8060000B291
:101FA80002B010BD4FF47A7240F6FF73B0FBF3F342
:101FB8005343A3F53923A3F50C6340F6C412E0E7B5
:101FC800001000B00075FF1F4FF0B04382B09A6A4E
:101FD80022F480529A629A6C42F480529A649B6C02
:101FE80003F480530193019B002002B070474FF027
:101FF800B04382B09A6C02439A649B6C034001938D
:10200800019B02B0704708B50420FFF7F0FF0120DC
:10201800FFF7EDFF0220FFF7EAFF002211460B2031
:1020280002F092FF0B2002F0C1FF002211460C20A3
:1020380002F08AFF0C2002F0B9FF002211460D20A1
:1020480002F082FF0D2002F0B1FF002211460E209F
:1020580002F07AFF0E2002F0A9FF002211460F209D
:1020680002F072FF0F2002F0A1FF0022114610209B
:1020780002F06AFF102002F099FF00221146112099
:1020880002F062FF112002F091FF00223620114673
:1020980002F05AFFBDE80840362002F087BF000072
:1020A80008B503F0CBF910B16FF0040008BD064B7A
:1020B8009A6942F040429A614CF2FA321A6103F08E
:1020C800CFF90028F2D0EFE700400058F0B585B00E
:1020D80000230C4600930646A8B3FFF7E1FF054628
:1020E80070BB03F0ABF988BB1A481B4A0223019363
:1020F800D0F8E01506F1784302EA8121B3FBF1F745
:1021080001FB1733DB0A0293D0F8E00504F17841AC
:102118000139314402EA8022B1FBF2F002FB1011CE
:10212800C3EBD1230133694601A8039303F018FADE
:1021380020B102280CBF01256FF0010503F090F9CA
:10214800284605B0F0BD6FF00505F9E76FF0040506
:10215800F6E700BF0070FF1F00FCFF03014B18608B
:1021680000207047D00100202DE9F04F89B0B0F170
:10217800006F06460F460092C0F0C580DFF89881D0
:10218800664DD8F8E03505EA832303F10063013B87
:10219800984200F2B880002800F0B880002900F0CA
:1021A800B58040EA02035B0740F0B080FFF778FF94
:1021B8000446A0BB03F042F9002840F0AA80D8F8F2
:1021C800E01506F1784205EA8121B2FBF1F301FB43
:1021D8001322009B03F17843013B3344B3FBF1F036
:1021E80001FB1033DB0A01334FEAD22AA3EBD222D8
:1021F800012A039388BFC6F30A050AF58038C6F199
:10220800080398BF009D069388BFC5F500654FEA8F
:10221800C828B346039B9A4505D303F021F9204605
:1022280009B0BDE8F08FA6F10803069A1A44954252
:1022380019D804950197CDF814B04FF00009059B03
:1022480009EB0301049B99453ED3009BAB442F4403
:102258005D1BB5F5006F28BF4FF400650AF1010A50
:1022680008F50068D6E753F8081F5A68B2F1FF3F2F
:1022780008BFB1F1FF3FD8D0294B186810B96FF0EB
:102288000504CAE7B8F1000F04D04FF400624146D4
:102298000EF0C0FBDFF88890D9F80030CBF30A00C5
:1022A80039461844AAB20EF0B5FB4FF40061404617
:1022B800FFF70CFF08BBD9F8003001934FF4006317
:1022C800CDF814800493B8E7019B07914B4402931F
:1022D8000120D3E9002303F0FDF888B90799019B91
:1022E800D1E9000259F80310029B5B689A4208BFC3
:1022F800884205D109F10809A1E76FF001048CE7CC
:102308006FF0030489E74FF0FF3488E76FF00504A6
:1023180085E76FF0040482E70070FF1F00FCFF03ED
:10232800D0010020B1F1006F70B511D30B4BD3F879
:10233800E0650B4B03EA862303F10063013B9942F6
:1023480006D840B139B192B20EF064FB002070BDDE
:102358004FF0FF30FBE76FF00500F8E70070FF1F54
:1023680000FCFF03B0F1006F10B40DD3084BD3F895
:10237800E045084B03EA842303F10063013B9842DC
:1023880002D810BCFFF7A2BE4FF0FF3010BC704758
:102398000070FF1F00FCFF034FF0B04382B0DA6CFF
:1023A8000243DA64DB6C03400193019B02B070477F
:1023B80070B5012086B00024CDE90444FFF7ECFF96
:1023C8000220FFF7E9FF0420FFF7E6FF01250222BC
:1023D8000DEB00014FF404134FF09040CDE90123B9
:1023E800204E039503F00AF94FF4441301A94FF066
:1023F8009040CDE90235019503F000F904230DEB77
:1024080003013046CDE90135CDE9034403F0F6F880
:1024180022463046082103F017FA4FF4806301A9D9
:102428004FF09040CDE90134039403F0E7F8082316
:1024380001A93046CDE90135CDE9034403F0DEF8C2
:1024480022462146062002F07FFD062002F0AEFD5E
:1024580022462146072002F077FD072002F0A6FD5C
:1024680006B070BD0004004808B51248124A134B64
:10247800C0E9002300230122C0E90232C0E9043385
:10248800C0E90633036203F0F1F908B100F0EAF895
:102498000848002103F03BFA08B100F0E3F80548CA
:1024A800002103F05AFA18B1BDE8084000F0DAB884
:1024B80008BD00BF94020020005800405D3E302057
:1024C80070B596B005461422002103A80EF0DAFE76
:1024D8003822002108A80EF0D5FE2A68304B9A420F
:1024E8005BD18023089308A84FF440230E9303F090
:1024F8008FFF08B100F0B6F84FF0B0444FF4C05069
:10250800E36C43F00103E364E36C03F0010302931B
:10251800029B12230026CDE903030323CDE90563BB
:102528004FF09040042303A9079303F067F8A36DC5
:10253800DFF870C043F48003A365A36D1A4C03F45D
:1025480080030193019B26620D23C4E900C3204642
:102558008023C4E90266C4E90436C4E9066602F0C9
:1025680085FD08B100F07EF8104AEC63A562104CB6
:102578000E23C4E900231021002380222046C4E949
:102588000213C4E90423C4E90633236202F06EFD92
:1025980008B100F067F8AC63A56216B070BD00BF63
:1025A8000058004044000240D40100205800024076
:1025B8003402002000B59BB04822002108A80EF084
:1025C80061FE1822002102A80EF05CFE03F0EAF971
:1025D8004FF0B0420120D2F8903023F01803C2F82F
:1025E8009030D2F8003423F4C06343F40073C2F887
:1025F8000034D2F8003403F4C0630193019B242310
:10260800089381230B930023CDE91003B02208A877
:10261800CDE9122303F03EFB08B172B6FEE74F2363
:10262800CDE90230CDE90400CDE90600022102A877
:1026380003F0CAFD08B172B6FEE71BB05DF804FBF3
:1026480008B501F0F9FFFFF7B5FFFFF7B1FEFFF797
:10265800DAFC00F018FE40F6B83000F049FA00F055
:1026680019FEFCE772B6FEE700B58DB02C220021FA
:1026780001A80EF007FE1748174B03601F2383605D
:102688004FF080420023C0E90433C0E90723836187
:102698004FF48073436204F041F808B1FFF7E2FF9A
:1026A8000C4804F067F908B1FFF7DCFF4FF000535E
:1026B80000220793074808924FF4807301A90292F9
:1026C80006920B9304F08AF808B1FFF7CBFF0DB020
:1026D8005DF804FBE80200200028004010B504461D
:1026E80090B03822002102A80EF0CCFD2268194BC8
:1026F8009A422CD14FF48033029302A84FF480738E
:102708000F9303F085FE08B1FFF7ACFF4FF0B0431D
:102718000220D3F8902042F40042C3F890209A6D2A
:1027280042F480629A659B6D002203F4806311462F
:102738000193019B02F008FC022002F037FC002202
:102748002A20114602F000FC2A2002F02FFC10B0CB
:1027580010BD00BF002800407047000008B501F018
:1027680081FF044B0120C3F88800BDE8084003F04E
:1027780071B900BF0004005801F07BBF08B501F033
:1027880078FF00F063FCFFF713FEFFF73CFCBDE8A1
:102798000840FFF769BE08B501F064FFBDE80840CE
:1027A8000121002003F006B970477047FEE7FEE7F5
:1027B800FEE7FEE7FEE77047704770477047000086
:1027C800014804F0FDB800BFE8020020012003F032
:1027D80041B8022003F03EB870477047014802F044
:1027E800BFBD00BFD4010020014802F0B9BD00BF41
:1027F800C0030020014802F0B3BD00BF6003002001
:10280800FFF7F2BF7047704770470000014804F0B7
:102818009BBC00BF20040020014803F003BF00BF99
:10282800E8020020014804F0F6BA00BF4C0300207B
:102838002DE9F04389B080460020109E0790894614
:1028480015461F46FDF7ECFCF0B9104CCDE9009099
:10285800CDE9020407AB0E480593142304933A46C6
:10286800434629460068FDF7A5FD2346324604F194
:10287800140153F8044B42F8044B8B42F9D1079BDF
:10288800337509B0BDE8F0830120FAE72003002082
:10289800AC1401087FB5124C00253C2302A86375CF
:1028A800CDE90255257500F0C5F8042303AA009464
:1028B80012210C48FFF7BCFF0B49142220460EF0EA
:1028C800D1FC0646B0FA80F0400960750090074BCD
:1028D8002A46294602200DF095FF304604B070BD07
:1028E80034030020F2140108DE060020D414010885
:1028F800054808B50823036004F0A8F818B1BDE836
:102908000840FFF7AFBE08BD4C0300204FF0B043AE
:1029180007B55A6E42F001025A665B6E002203F058
:102928000103019311463220019B02F00DFB322076
:1029380003B05DF804EB02F039BB00000CB407B536
:10294800054A05AB102101930EF06EFB03B05DF84C
:1029580004EB02B0704700BF0415010830B585B01C
:10296800044602A80D460EF08BF9BDF90C30064A54
:1029780000931021029B2046FFF7E0FF2046FEF758
:102988001BFD288005B030BD041501084FF0B0428A
:1029980010B5936823F4004393600EF0F9F90F4BD8
:1029A80001241C7000F0B8F80DF0C2FE0C480DF0C0
:1029B800D9FE0C4B4FF400421A6103200DF0D8FEEB
:1029C800FFF7A2FA00F014F900F050FC0DF0CCFF6C
:1029D80021462046BDE810400DF0E6BF5803002010
:1029E80065290008004000580DF0F4BF08B5FFF74E
:1029F80093FA40F6B83398420CD8B0F5E16F0BD390
:102A0800FE23A0F5E16058434FF49663B0FBF3F062
:102A1800C0B208BDFE20FCE70020FAE77FB5684693
:102A280000F0CAF80198FFF749F800B207B05DF85E
:102A380004FB0000194A38B5D2F88035591C044601
:102A480019D101F01DFE054601F026FE054401F0EE
:102A58001DFE2B0EE3712B0CA3712B0A6371030E61
:102A6800E370C0F30742C0F307232571C0B2A27018
:102A78006370207038BD190AC3718171190C1B0E5F
:102A880041710371D2F88435C370D2F88405C0F35C
:102A98000722C0F30743000EE9E700BF0070FF1FDD
:102AA80038B5094BD3F8803503600133054609D1A1
:102AB80001F0E6FD044601F0E9FD444001F0ECFDBB
:102AC80044402C6038BD00BF0070FF1F0121022068
:102AD8000DF054BF002102200DF050BF00207047B8
:102AE800024B187808B100F0BBB8704758030020B3
:102AF80082B00190019802B000F04EB94FF0B04397
:102B080082B0DA6C42F00202DA64DB6C03F0020392
:102B18000193019B02B070472DE9F043254C87B023
:102B280001F0C0FD01F0C6FD01F0CCFD0123002538
:102B380002934FF48059032301A9204604934FF4CC
:102B4800005803950595FFF7D9FFFFF7D7FFFFF763
:102B5800D5FFFFF7D3FFCDF8049002F04FFD01A990
:102B680020464FF40067CDF8048002F047FD01A924
:102B780020464FF40046019702F040FD01A9204687
:102B8800019602F03BFD2A464946204602F05CFECB
:102B98002A464146204602F057FE2A463946204634
:102BA80002F052FE2A463146204602F04DFE07B09A
:102BB800BDE8F0830004004810B50446FFF7C6F9E5
:102BC800074BA36040F30F20FEF724FF054B064A8E
:102BD8002360064B6060C4E90323002010BD00BFDA
:102BE8000000484200007A440D093E00AB0305008E
:102BF80000207047014B1868704700BF5C03002035
:102C08000320704708B501464FF47A72002380020A
:102C1800890DFEF779FF08BD4FF47A73A0FB030313
:102C2800800A40EA83507047034B98689A6890423C
:102C3800FBD1C043704700BF0028004008B5FFF72C
:102C4800F3FF014B186008BD5C03002008B5FFF7CF
:102C5800EBFF024B1B68C01A08BD00BF5C030020D5
:102C6800024B187808B1FFF7DFBF704759030020FF
:102C780010B5074B074C0122DA654FF480712046E6
:102C880003F096FC4FF0FF332363002010BD00BF14
:102C980000280040E802002002460021014803F015
:102CA800A0BE00BFE802002002460121014803F04F
:102CB80098BE00BFE802002010B58CB02C2200217D
:102CC800044601A80EF0DEFAFFF7D2FF0C4B0D48C0
:102CD8001B681C440023089306934FF00053E443F9
:102CE800079301224FF4807301A902940B9303F018
:102CF80075FD08B1FFF7B6FC00200CB010BD00BF91
:102D08005C030020E802002038B50546FFF78CFF79
:102D180002210446074803F06BFEC4F309024FF48E
:102D28007A71A2FB0121920AA30A2A8043EA805001
:102D380038BD00BFE80200200148002103F058BE5A
:102D4800E80200200148012103F052BEE8020020F9
:102D5800F8B50F4D2E78CEB90E4C4FF0FF372763DC
:102D6800FFF782FCFFF784FF4FF48071204603F0E1
:102D78001FFC2046276303F0DFFD32462046022170
:102D880003F02FFEFFF75AFF01232B700020F8BD38
:102D980059030020E8020020014610B54FF47A726A
:102DA80000238002890DFEF7AFFE0146FFF73CFFC6
:102DB8000446FFF739FF031B8B4200D310BD00BF49
:102DC800F7E70EF0EDB8000010B5064C02212046DA
:102DD80003F00EFE0221421C2046BDE8104003F01D
:102DE80000BE00BFE80200201648174A08B54FF495
:102DF800E133C0E9002300230C22C0E90233C0E913
:102E08000523C0E90733C0E90933036104F07DFFF6
:102E180008B1FFF727FC0B48002105F0F2F808B1CC
:102E2800FFF720FC0748002105F00BF908B1FFF770
:102E380019FC044805F0C5F818B1BDE80840FFF7CB
:102E480011BC08BD200400200044004070B596B0B5
:102E580005461422002103A80EF014FA3822002196
:102E680008A80EF00FFA2A68334B9A4261D1022360
:102E7800089308A8314B0A9303F0CAFA08B1FFF780
:102E8800F1FB4FF0B0430C219A6D2D4C42F4003207
:102E98009A659A6D02F400320292029ADA6C42F054
:102EA8000102DA64DB6C03F001030193019B022346
:102EB8000026CDE903130323CDE905634FF09040C5
:102EC800072303A9079302F099FB1E4826621423DF
:102ED800C4E900031023C4E9023620468023C4E96C
:102EE8000436C4E9066602F0C1F808B1FFF7BAFB78
:102EF800154AEC67A562154C1323C4E90023204644
:102F080000238022C4E90233C4E90423C4E9063358
:102F1800236202F0ABF808B1FFF7A4FB2520C5F83F
:102F2800804000220221A56202F00EF8252002F05E
:102F38003DF816B070BD00BF0044004004000C000E
:102F4800C0030020800002406C00024060030020A3
:102F580002680E4B9A4210B5044616D14FF0B042A3
:102F68000C21936D23F4003393654FF0904002F0E9
:102F7800F1FBE06F02F0EEF8D4F8800002F0EAF816
:102F8800BDE81040252002F01FB810BD00440040E5
:102F980008B50A460146024804F03AF8002008BD80
:102FA8002004002013B5114B114C18604FF4001386
:102FB800009302AB13E90600204604F0A6FF23683D
:102FC800DA69D103FCD4DA695202FCD59A68084858
:102FD80042F480029A6004F0DEFF064904480122A8
:102FE80004F04CFF002002B010BD00BFB404002064
:102FF80020040020BC04002008B5074B1860FFF728
:1030080002F8FFF7F1FE054AD2F8803043F000637A
:10301800C2F88030002008BDB8040020000800581D
:1030280008B54FF0B04308489A6B42F400329A63EF
:103038009A6B22F400329A63FFF78AFF0F2001F09F
:10304800C3FF002008BD00BF2004002008B50748C2
:1030580004F05BFE08B1FFF705FB054802F006F82F
:1030680018B1BDE80840FFF7FDBA08BD20040020EC
:10307800C00300200268044B9A4203D1034B00208E
:103088001B681847704700BF00440040B804002080
:1030980002680B4B9A4210B504460FD1094B1B68C6
:1030A8002BB1D0F8902012B9074801219847204643
:1030B8000549BDE81040012204F0E0BE10BD00BF84
:1030C80000440040B4040020BC04002013B5134C95
:1030D80023785BB9E37C03F0FF023BB9104B114640
:1030E800022002B0BDE810400DF08CBBFFF7D2FB08
:1030F80000380C4B18BF0120400018701A78022ABB
:1031080002BF00222270E2741B7800930022064B53
:10311800114603200DF076FB02B010BDDE0600203C
:1031280060150108D00400207C15010838B5184C3A
:1031380023785BBBE37C03F0FF023BBB154D2B6898
:10314800012B0CD92B68042B09D81146124B0220ED
:103158000DF058FB114A0421012000F0ADFB2B684B
:10316800042B13D900220E4B114602200DF04AFB06
:10317800FFF790FB00380B4B18BF01204000187078
:103188001B78022B02BF00232370E37438BD00BFF5
:10319800DE060020CC04002093150108B8150108AC
:1031A800BD150108D0040020002213B5154B164C9C
:1031B800114603200DF026FB01220821134802F0D6
:1031C80043FB4FF47A70FFF793FC4FF480614FF0A4
:1031D800904002F033FB207021780D4A0D4B0029F6
:1031E80018BF13460022009311460B4B01200DF027
:1031F80009FB06480022082102F026FB237802B0CA
:1032080010BD00BF18160108D104002000040048B2
:1032180007160108F01501083016010870477047B5
:10322800022808B50ED801221021074802F00CFB2D
:103238003220FFF75DFCBDE808400348002210215A
:1032480002F002BB08BD00BF00040048054B1B7814
:10325800B3FA83F35B09037100234371024B012224
:103268001A707047D1040020DD060020034A0023AD
:1032780013715371024A1370704700BFBE040020D7
:10328800DD060020704708B5FFF780FBBDE8084061
:1032980000F0D4BC4FF0FF300DF000BC70470000C8
:1032A800014BD870704700BF5C000020014B1874B8
:1032B800704700BF5C00002007B5064B00221B5C6E
:1032C80000931146044B02200DF09CFA03B05DF800
:1032D80004FB00BF601601084616010808B5022065
:1032E80000210DF0A3FBBDE8084001480DF006BE23
:1032F8002C060020002101200DF098BB13B50D4CC1
:10330800A0B120600C480DF0ABFD21680A480DF013
:103318002FFE09480DF0F2FD236800930022074BA9
:10332800114601200DF06EFA02B010BD42F2107382
:103338002360E7E7740000202C06002064160108CB
:1033480013B50D4C206023680BB90C4B23600C4857
:103358000DF086FD21680A480DF00AFE08480DF0B8
:10336800CDFD236800930022064B114601200DF085
:1033780049FA02B010BD00BF0C000020A086010071
:10338800440600208D16010837B5044600283AD0B7
:1033980090F90650002D38D11F480DF061FD2A46DE
:1033A80029461E4B02200DF02DFAE379012B0CBFA4
:1033B8001B4B1C4B2A46294602201B4D0DF022FAB6
:1033C800E3792B70194B1868FFF7BAFF184B186888
:1033D800FFF794FF2978174A174B012918BF13469E
:1033E800002200931146154B01200DF00BFA94F9B9
:1033F8000530019394F9043000930022104B1146D4
:1034080002200DF0FFF903B030BD00220D4B11462C
:1034180002200DF0F7F9EAE7C8050020D2160108E6
:10342800E716010804170108F80500200C00002021
:1034380074000020CD160108C916010821170108DB
:10344800591701084017010838B504460D460748C2
:103458004FF40061FEF786FF30B92A46214603483B
:10346800BDE83840FEF780BE38BD00BF00F0030855
:103478000A460149FEF756BF00F0030870B5164822
:103488000DF0EEFC05F042FA044650B10022134B51
:10349800114602200DF0B6F9BDE8704010480DF055
:1034A8002DBD104D104B0246014602200DF0AAF921
:1034B80001260E4B2E702246214602200DF0A2F95D
:1034C8000B4805F0B5F82878314604F007FE0248A5
:1034D8000DF014FDE0E700BF2C060020821701085C
:1034E800FC05002000000020A0170108B4170108FF
:1034F8005C00002030B587B0FFF778FA0446FFF784
:1035080053FE02A8FFF7A2FE474B07221A70474A4C
:103518001178002943D00021117008221A70444AFA
:103528005968127862F07F020A705A6824B204EB74
:10353800440404EB4414FE21B4FBF1F45470022259
:103548003C493D4C0978012988BF00225A70637AAA
:1035580033B104F0A5FE012802D120460DF080FC0D
:10356800364B3148D978002204F0C4FE04460028BE
:1035780044D10146324B012203200DF043F9314872
:103588000DF06EFC304B2F481968A14238BF214618
:103598000DF0EEFC2B480DF0B1FC07B030BD2B4907
:1035A8002B480A7822B9057805F0FF02002DC7D00C
:1035B800002202701E480A7059680078087059681D
:1035C8004A705A68562191705A680121D1705A6818
:1035D80024B204EB4404FE2104EB4414B4FBF1F4DC
:1035E80014715A68022151715A689DF80D10917131
:1035F8005A689DF80C10D1710822A1E7063410D141
:1036080004F048FE04460028B9D04FF47A7301222A
:10361800B0FBF3F30021009303200E4B0DF0F2F8FA
:10362800ADE70024ABE700BF040000205C060020E3
:10363800C4050020D0040020C80500205C0000203C
:10364800D31701082C06002074000020F306002080
:10365800DD060020E217010800B503468DB00028FA
:103668002CD0407802280AD003282AD0164B0022F2
:10367800114602200DB05DF804EB0DF0C3B81A7FB7
:103688000B92DA7E0A929A7E09925A7E08921A7EE4
:103698000792DA7D06929A7D05925A680492DA6852
:1036A800039293F914200292B3F9122001921B7C21
:1036B80000930022054B11460DF0A4F80DB05DF8FB
:1036C80004FB034BD3E700BF0018010817180108D3
:1036D8008918010801284FF000020CBF024B034B68
:1036E800114602200DF08EB8A8180108BA18010872
:1036F8001FB50446002831D00378002B2ED01D4872
:103708000DF0FCFB002211461B4B02200DF07AF84D
:1037180094F91830039394F90A300293237C0193A7
:10372800E368009300221146144B02200DF06AF85A
:103738000022134B114603200DF064F8237A012B65
:103748000ED1617A0F4A104B002908BF1346002298
:10375800009311460D4B02200DF054F804B010BD33
:1037680000220B4B1146022004B0BDE810400DF0BA
:1037780049B800BF14060020D3180108041901082D
:1037880035190108CE180108CF1801084219010897
:103798005319010808B5104B0122002102201A70A4
:1037A8000DF044F90D480DF0A9FB0D4B1B788BB1BA
:1037B8000C4B1A7872B9DB7C63B90B4B1A68042A74
:1037C8009EBF1A6801321A600021BDE80840102027
:1037D8000DF02CB908BD00BF5C060020440600208F
:1037E800F8050020DE060020CC040020044B1B78DE
:1037F800022B03D1002108200DF018B9704700BF33
:103808000000002008B505F08AF880B904F048FDEA
:1038180001280CD1BFF34F8F0549064BCA6802F443
:10382800E0621343CB60BFF34F8F00BFFDE708BDD5
:1038380000ED00E00400FA0510B505F003F910F1F9
:10384800080F07D1064B0022BDE8104011460220A0
:103858000CF0D8BF013001D1024BF4E710BD00BF16
:10386800611901087719010870477047704700000F
:10387800012837B5044603D0022817D003B030BD5D
:1038880001464FF0904001F0D9FF00220546009014
:10389800084B114620460CF0B5FF012DEED1002152
:1038A800022003B0BDE830400DF0C0B80021082068
:1038B800F7E700BF8F19010873B505460C46164691
:1038C80004F002FD0346002838D0002426480DF0F5
:1038D800C7FA264B24481968A14238BF21460DF083
:1038E80047FB214802B0BDE870400DF007BB4A68AD
:1038F800F05CD0540133DAB2A242F8D31C4B0D70FD
:103908001B78012B88BF00244C701A4C637A33B1A2
:1039180004F0C6FC012802D120460DF0A1FA164B8E
:103928001648D978002204F0E5FC044640B901465F
:10393800134B012202200CF065FFC7E70F49DAE7B5
:103948000634C2D104F0A6FC04460028BED04FF4C9
:103958007A730122B0FBF3F3002100930220094B94
:103968000CF050FFB2E700BF2C06002074000020C6
:10397800D0040020C80500205C00002004000020BE
:10398800D3170108E2170108044B1B7823B9044A2E
:1039980005210120FFF790BF704700BFD004002029
:1039A800AD19010810B5002490B03C22214601A8A9
:1039B80000940DF067FC2F4B2022DA7219788DF8ED
:1039C800001059788DF8011099788DF80210D9787F
:1039D8008DF8031019798DF8041059798DF80510B0
:1039E80099798DF80610D9798DF80710197A8DF81C
:1039F8000810597A8DF80910997A8DF80A108DF8FF
:103A08000B2021460DF10B0258180131007B02F8FA
:103A1800010F1C29F8D193F828208DF8282093F855
:103A280029208DF8292093F82A208DF82A2093F848
:103A38002B208DF82B2093F82C206AB193F83F2087
:103A480052B10DF12B0100229818013290F82C0088
:103A580001F8010F142AF7D107484FF40061FEF767
:103A680081FC20B9044840226946FEF77DFB10B06E
:103A780010BD00BF7800002000F80308014940226B
:103A88000CF0C8BF00F8030870B52A4D28796B7987
:103A98004D2BC0B233D1C0EB001080000A2838BFCC
:103AA8000A204FF47A735843234BAC791860EB79AA
:103AB8004D2BE4B22BD1C4EB0414A40095F82C30A0
:103AC8001E4E63BB95F83F304BBB42F21070FFF7B8
:103AD80015FC3068FFF734FC2B7A194A1949DBB218
:103AE80013706B7A184ADBB213700023EA1892F845
:103AF8002C20D2B2CA540133142BF7D170BD6B7984
:103B0800482B0ABF4FF461636B795843C6E7EB79DA
:103B1800482B0ABF4FF46163EB795C43CEE7FFF7AC
:103B2800EDFB012C38BF01244FF47A735C433460F9
:103B3800CFE700BF78000020740000200C000020B0
:103B4800F2060020DE060020D004002010B590B058
:103B580000213C2201A800910DF094FB4022344939
:103B680068460CF057FF9DF800203AB99DF801000F
:103B7800562803D19DF8021001290FD000222D4BA1
:103B8800114601200CF03EFEFFF70CFF4FF47A704F
:103B9800FEF7AEFFFFF778FF10B010BD264B1A7086
:103BA800587099709DF80310D9709DF80410197118
:103BB8009DF8051059719DF8061099719DF8071028
:103BC800D9719DF8081019729DF8091059729DF85D
:103BD8000A1099729DF80B1001F03F01D972D87A3A
:103BE800D1B288421BD89DF8282083F828209DF858
:103BF800292083F829209DF82A2083F82A209DF877
:103C08002B2083F82B200DF12B010022981801326C
:103C180011F8014F80F82C40142AF7D1BAE701F1C6
:103C280040006844194410F8340C08730132D6E790
:103C380000F80308B319010878000020F0B50B2339
:103C48008BB0122200240125CDE906320327562322
:103C58001721CDE9043122465F4B03942146CDE973
:103C680001550097284609940CF0CCFD5B4B009554
:103C780022462146CDE9017402200CF0C3FD02263C
:103C88000523CDE900632246554B02942146304670
:103C98000CF0B8FD534B009522462146CDE901743E
:103CA80030460CF0AFFD09A9204604F01BFE099B25
:103CB800C3F307220292C3F307421B0E019200933B
:103CC8002246494B214630460CF09CFD09A928465E
:103CD80004F008FE099BDAB20392C3F307220292AA
:103CE800C3F307421B0E0192009322463F4B214625
:103CF80030460CF087FD3E4B3E48009422464FF478
:103D0800FA710DF04FF83C4B3C48009422464FF4B2
:103D1800FA710DF047F83A4B3A4800942A464FF4A6
:103D2800FA710DF03FF82046FEF718FA08B1FEF7D1
:103D380099FC354B009400224FF4FA6133480DF09A
:103D480031F8334A002101200CF02CFF314A0021C0
:103D580002200CF027FF304A002104200CF022FF3B
:103D68002E4A002108200CF01DFF00F0BDFB2C4955
:103D78002C4804F06DFD2C4804F05AFC21480DF045
:103D8800BDF82A4B0021187804F0A8F928490094B6
:103D9800284B0968284800220DF004F826480DF041
:103DA800ADF8FFF7D3FE254A002110200CF0FAFEEB
:103DB800234A00214FF480600CF0F4FE214B224886
:103DC8001968224B009400220CF0ECFF1E480DF0FD
:103DD80095F80BB0F0BD00BFF51901083C1A0108B1
:103DE8005D1A01087E1A01089F1A0108C01A010805
:103DF800A53200081406002073380008E0050020EA
:103E080071380008C8050020F5370008FC050020B7
:103E180031840008FD340008413800088534000862
:103E280000000301100000205C00002000000020BA
:103E380074000020E53200082C0600203531000807
:103E4800B13100080C000020440600209D3700080E
:103E580030B50024A3B07C22214603A802940DF0BB
:103E680011FA53238DF808304FF4AB73ADF80A30CC
:103E780001238DF80C30ADF80440FEF7B7FD00B211
:103E880000EB400000EB4010FE23B0FBF3F08DF890
:103E98000D0001A800F0CDFBC0B143000133DBB237
:103EA8000B4C8DF80E302C228021201D1D460DF064
:103EB800E9F90298BDF80C302060A380A57122466C
:103EC80007210120FFF7F8FC23B030BD5823E7E7AE
:103ED8005D060020F0B50378592B95B0044640F0F4
:103EE800EF8105295FD84378443B162B5BD8DFE880
:103EF80013F01E015A000E015A0016015A005A000A
:103F08005A005A0079005A00F9005A005A005A001B
:103F180093015A005A009D005A005A005A0017008F
:103F28008578482D17D1B14A14210120FFF7C4FC28
:103F380041F28830FEF7DCFD0022AD4B114601202E
:103F48000CF060FC40F6B830FEF7D2FD15B0BDE8C5
:103F5800F040FFF757BC532D0ED130228021A548E1
:103F68000DF090F9FFF774FF41F28830FEF7C0FDBD
:103F7800A04A152101206DE0432D16D1002404A884
:103F88008DF8104004F0CCFA9A4A4C23137056234B
:103F980093709DF81030547001204133D070137124
:103FA8000521FFF789FC15B0F0BD442DFBD1914CDC
:103FB8002C228021201D0DF065F9002325706370E7
:103FC80001255623A370E5702571FEF70FFDFE232A
:103FD800B0FBF3F000EB400000EB401060712246AC
:103FE8000621C7E78378303BDBB2092BDBD8824C4C
:103FF800824A23702378DBB253727E4A59231370A6
:104008004D23537023783033937003210120FFF739
:1040180053FC237800930022794B114601200CF0C1
:10402800F1FB15B0BDE8F040FFF7BCBC8578482D22
:1040380015D1704A562313709370032313711723F5
:1040480053710B2300210120937112235170D070FA
:10405800D371082115B0BDE8F040FFF72DBC432D02
:10406800A1D1644C00213C2205A804910DF00AF965
:1040780004A8FFF703FD2422802104F10C000DF0B1
:1040880001F99DF8103063709DF81130A3709DF808
:104098001230E3709DF8133023719DF8143063716A
:1040A8009DF81530A3719DF81630E3719DF817300F
:1040B80023729DF81830257063729DF81B509DF887
:1040C8001930A3729DF81A30E3722A4607A925739E
:1040D80004F10D000DF007F905F10D012246C9B2F2
:1040E80001205EE7807839280CD83038C0B2FFF755
:1040F80095F8404A2378137063785370A3789370C7
:10410800032137E715B0BDE8F040FFF73DBC8078E4
:104118003928F7D83038C0B2FFF781F8E9E7807856
:104128003928EFD83038C0B2FFF77AF8E1E783785A
:10413800303BDAB2092AE5D8C578303DEAB2092A17
:10414800E0D80179A1F14802D2B20B2ADAD82D4879
:1041580040FA02F2D007D5D40A224D2902FB0355B2
:104168003FD13C235D43284B4FF47A706843186075
:10417800264B1860FFF7C2F81E4A2378137063783D
:104188005370A3789370E378D37023791371052162
:104198000120FFF791FB194B5622012600271F70BB
:1041A8005A709E70DE70A178303901EB8100E17899
:1041B800303901EB4001C9B2197122795A71144A98
:1041C8001278D2B21A720C4A1278D2B25A72FFF727
:1041D800E9FB104B00953A46394630460CF012FB85
:1041E800E1E64829BFD14FF46163BBE7E41A01084F
:1041F800F91A01085D060020D0040020780000208C
:104208001B1B0108DEF7FFFF740000200C000020D4
:10421800F2060020441B01088678A6F13007FBB29D
:10422800092B3FF66FAFC078A0F13005EBB2092B30
:104238003FF668AF2379A3F14802D2B20B2A3FF6C2
:1042480061AF6D4941FA02F2D2073FF55BAF0A222E
:104258004D2B02FB07552ED13C225543674A592165
:104268001170532151709670D0701371052101207F
:10427800FFF722FB624B5622012600271F705A7057
:104288009E70DE70A178303901EB8100E178303919
:1042980001EB4001C9B299712279DA71594A127851
:1042A800D2B21A72584A1278D2B25A72FFF77AFB0F
:1042B800564B00958FE7482BD0D14FF46162CCE77D
:1042C800502B5DD102297FF66EAE4378303B012B2F
:1042D8003FF669AE8378312B7FF465AE0B2904D89D
:1042E800FFF752FB0021454A44E6454D484F02344A
:1042F800002614F8012FA919303AD2B20A730B7BA1
:10430800CDE9026323780022CDE9006311463B46DC
:10431800012001360CF076FA0C2EEAD1FEF7B2FF36
:10432800364B50221A7056229A70002401225C7073
:10433800DA7003F8042F2A190134127B0C2C02F1CD
:10434800300203F8012FF6D10022502311460093C2
:104358000120304B0CF056FA00232B7056236B705B
:104368000123AB70EB70274B1B78DBB22B72264B0B
:104378001B78DBB26B72EC72FFF714FB1121B2E70A
:10438800412B7FF410AE4378432B7FF40CAE1629F3
:104398007FF409AE204D421C002312F8011FE95496
:1043A8000133142BF9D1FEF791FE1C4B5B7D012BD9
:1043B80019D113490023EA5CC8180133D2B2142B6F
:1043C80080F82C20F7D1104B00221A701B78DBB232
:1043D8004B72FFF7E7FA094A631E15349C4206D16F
:1043E800064A1621C6E5084B02221A70F3E713F8AD
:1043F800011F02F8011BF1E7DEF7FFFF5D06002051
:1044080078000020F2060020D00400207B1B010861
:10441800C61B0108EE1B0108DE060020340300203D
:1044280070B5054686B00C4600293BD028480CF0EC
:1044380065FD2678EEB1002D48D068682E78C0B1A9
:10444800032E0BD0072E2FD0022E12D16978012906
:104458000FD00B060DD4FFF73DFD0AE06B78012B5A
:1044680007D10078012802D0022800D008B904F04A
:104478000DF8237C052B15D894F90A20059294F998
:1044880009200492134A52F82330039394F9083010
:10449800CDE901630022E368009311460E4B032027
:1044A8000CF0B0F906B070BD6B78012BE1D1027841
:1044B8000A4B02F001021A702AB9094B114603206F
:1044C8000CF0A0F9D5E7074B0022F7E72E46D0E716
:1044D800E0050020741C01081C1C0108C40500200C
:1044E800091C0108131C0108034B0022C3E902221E
:1044F8000122C3E900227047F406002000487047F3
:10450800F40600204FF0B04382B0DA6C0243DA645C
:10451800DB6C03400193019B02B070472DE9F04129
:1045280086B000240220154D0594FFF7EBFF042008
:10453800FFF7E8FF124F03944FF4807601230DEB49
:104548000001CDE901632846032304934FF4005882
:1045580001F054F801A93846CDF8048001F04EF86E
:1045680022464146384601F06FF928462246314630
:1045780001F06AF9204606B0BDE8F0810004004861
:1045880000080048032810B50ED8012810D868B9CB
:1045980002460B484FF4807101F056F90022094891
:1045A8004FF4005101F050F9002010BD0122F0E74E
:1045B800002203484FF4807101F046F90122EEE72A
:1045C8000004004800080048022070470020704797
:1045D8000120704700280CBF0F20162070470000EC
:1045E8000D48854600F027F80C480D490D4A002370
:1045F80002E0D458C4500433C4188C42F9D30A4A90
:104608000A4C002301E013600432A242FBD30CF0F1
:1046180041FEFEF715F8FEE700000120000000202B
:104628004C0100206C2701084C0100209024002038
:10463800FEE700207047704710B5032000F072FCB9
:1046480001F018FB064B18600F20FEF747FA0446E6
:1046580018B9FEF7AAF8204610BD0124FBE700BFF1
:10466800B80000204FF0E022136923F00203136121
:1046780070474FF0E022136943F00203136170475B
:10468800014BD3F8900570470070FF1F014BD3F81A
:10469800940570470070FF1F014BD3F898057047C9
:1046A8000070FF1F024A536823F0010353607047EC
:1046B800002004E0024A536823F002035360704765
:1046C800002004E0024A536823F004035360704753
:1046D800002004E08068C0F380007047F7B500232D
:1046E80001930446002800F0E980856D25B9FDF79F
:1046F800B5FBE56584F8545023689A68D00040F10A
:10470800A1809A68D10000F1B480A26D42F0100235
:10471800A265E26D42F00102E26501251846FFF745
:10472800D9FFA26D02F01002024340F0C980A26DC9
:10473800206922F4817242F00202A2659A68D207C7
:104748005DD4226BA67E94F82CC0003A18BF0122D3
:104758001703D4E902120A43217E42EA8132617EBC
:1047680042EAC13242EA4632002842EA4C02B4BF69
:1047780020F000414FF400113A430A4394F8201006
:10478800012903D1002E76D142F48032616A21B129
:10479800A66A01F4E07131430A43D968E66C21F452
:1047A800FE3121F4FF711143D96094F83C2061680F
:1047B800012A01F0404C4CEA060609D1D4E9102739
:1047C8003A433243A66C324342EA0C0242F00106F5
:1047D8001F693E4A3A4032431A6121F00042B2F161
:1047E800804F0CD0B1F1004F09D0394ED6F80827C8
:1047F80001F4701122F470120A43C6F808275A69A6
:10480800666BA16B22F0070232435A615A6922F0A3
:10481800700242EA01125A61002835D19A6A62F0A0
:104828000F029A625B6903F007039E423CD10023A2
:10483800E365A36D23F0030343F00103A365284652
:1048480003B0F0BD9A68234922F0104222F0170203
:1048580042F080529A60204A1268B2FBF1F20132AB
:1048680052000192019A002A3FF44BAF019A013A93
:10487800F7E7002552E7A16D41F02001A165E16D40
:1048880041F00101E16581E7B0F5001FCAD19A6ADC
:10489800E269013A92006FF00F0102F01C0201FA7E
:1048A80002F2216E0A43BCE7A36D23F0120343F022
:1048B8001003A365E36D43F00103E3650125BEE73B
:1048C800A36D43F01003A365F8E700BF02FCFF1FC8
:1048D80000200140400D0300B8000020F8B54569EC
:1048E800082D04460E460AD00368DB68D80705D5AC
:1048F800A36D43F02003A3650120F8BD0425FEF74E
:10490800EFF8074623681A682A4221D0A26D42F4BC
:104918000072A265DA6812F4406F14D1A27E92B9CF
:104928001A6812070FD51846FFF7D4FE28BB5A6835
:1049380022F00C025A60A26D22F4807222F0010269
:1049480042F00102A265207E00BB0C221A60D4E767
:10495800711CD8D0FEF7C4F8C01BB04201D8002E95
:10496800D0D123681B682B40CCD1A26D84F8543079
:1049780042F00402A2650320BFE7A26D42F02002C4
:10498800A265E26D42F00102E265DCE70020B4E7CF
:104998000368186C70470000F7B50023019390F87E
:1049A8005430012B044600F0C580056806690123D0
:1049B80080F854302846FFF78DFE002840F0B48078
:1049C800D1E90020022826F0040300F08280B3F128
:1049D800004FC2F3110E13D1AB6A43EA0E03AB6268
:1049E8008B68686903EA022323F07C4323F0FF0302
:1049F80020EA02210B43002A6B6126DB002055E0E8
:104A0800236E00F01F074FF00F0C0CFA07FC6FEA3B
:104A18000C0623EA0C0CBEF1000F11D1C2F384631B
:104A2800BB4043EA0C0323668008E36901309842DF
:104A3800D6D8A86AC2F38363BB4006403343CEE7A7
:104A480092FAA2F3B3FA83F3EAE73B493B48D1F879
:104A58000837824203F0E07519D11B02CED4D1F891
:104A6800083723F0E0732B4343F40003C1F80837F9
:104A7800334B1A68334BB2FBF3F20C2302FB0333BC
:104A88000193019B002BB9D0019B013BF8E72E480D
:104A9800824210D113F08070B0D1D1F8083723F0DA
:104AA800E0732B4343F08073C1F80837002384F880
:104AB800543003B0F0BD254882429FD113F48000E2
:104AC8009CD1D1F8083723F0E0732B4343F48003DB
:104AD800EAE7B3F1004F01BFAB6AC2F311018B43A0
:104AE800AB62002A8ADA154813498242D1F808379E
:104AF80009D1D1F8082703F0A07322F0E07213431C
:104B0800C1F808377AE71048824204D1D1F808275B
:104B180003F44003F1E70D4882427FF46FAFD1F808
:104B2800082703F0C073E8E7A26D42F02002A265EF
:104B38001846BBE70220BCE700200140001000B087
:104B4800B8000020400D0300004000B8002000B469
:104B5800026838B504461046FFF7BCFD08B90020C6
:104B680038BD9368990707D4936823F0004323F06E
:104B7800170343F010039360FDF7B2FF054623685F
:104B88009B685B07EBD5FDF7ABFF401B0228F6D906
:104B980023689B685A07F2D5A36D43F01003A365F9
:104BA800E36D43F00103E3650120D9E773B5002302
:104BB800026801939368DD07044602D5002002B01D
:104BC80070BD9168214B194209D0A36D43F01003C1
:104BD800A365E36D43F00103E3650120EFE7936804
:104BE80023F0004323F0170343F001039360184BAD
:104BF800D3F8083718021CD4637E012BDED0FDF7EA
:104C08006FFF144E054622681368DB07D6D49368F5
:104C1800D9075FBF9368334043F001039360FDF702
:104C28005FFF401B0228EED923681B68DA07EAD425
:104C3800CBE7094B094A1B68B3FBF2F30133019335
:104C4800019B002BD8D0019B013BF8E7170000809F
:104C580000200140E8FFFF7FB8000020400D03005E
:104C680038B504460068FFF735FD054620BB94F8C3
:104C78005430012B20D0012384F854302046FFF70C
:104C880095FFB0B9A36D226823F4706323F0010384
:104C980043F48073A3651C23E065136084F8540013
:104CA800936823F0004323F0170343F00403936051
:104CB80038BD84F85450FBE70220F9E7026838B59C
:104CC800936891680446C80701D4002038BD990745
:104CD800FBD4936803F00503012B19D1936823F0E3
:104CE800004323F0170343F0020393600323136088
:104CF800FDF7F6FE054623689B68DB07E5D5FDF75B
:104D0800EFFE401B0228F6D923689B68DA07F2D524
:104D1800A36D43F01003A365E36D43F00103E3655E
:104D28000120D3E770B5044600284BD0836D43F0CB
:104D380002038365FFF70CFF054668B92046FFF7B5
:104D4800BDFF054608B90123A3652268936823F0CF
:104D5800104323F01703936023685A6822F467729C
:104D680022F003025A6040F29F321A60D968164A4C
:104D78000A40DA601A6922F040421A615A6922F040
:104D880007025A611A6A02F0F0221A625A6A02F09D
:104D9800F0225A62DA6A02F0F022DA629A6A0B4A60
:104DA80000269E62D2F8083723F0FE73C2F808374F
:104DB8002046FDF767F8E6652666A66584F8546020
:104DC800284670BD0125FBE700023E830020014014
:104DD80010B590F85430012B044615D0012380F803
:104DE8005430FFF7B5FE58B92046FFF767FF38B9CA
:104DF800A36D23F4807323F0010343F00103A3653B
:104E0800002384F8543010BD0220FCE7F7B50023D6
:104E1800019390F85430012B04467FD0012380F889
:104E28005430FFF74BFF23689A6812F001020546D9
:104E380007D0A36D43F01003A365002384F8543012
:104E48002DE0A16D364F21F4817141F00201A16579
:104E5800DE68D96826F4FF4626F07C0621F4004176
:104E6800360421F00301360CD960082099683940CE
:104E780041F0004199609968002913DA01990131DC
:104E880001910199B1F52E3FF5D3A36D23F01203DB
:104E980043F01003A365002384F854300125284605
:104EA80003B0F0BDD3F8B410013801F07F010A4413
:104EB800DCD199681A48014041F001019960D3F8A2
:104EC800B41021F07F0141EAD202C3F8B4209A68F5
:104ED800024042F002029A60FDF702FE074623688C
:104EE8009A68D20708D4DA683243DA60A36D23F0EF
:104EF800030343F001039FE7FDF7F2FDC01B0228FF
:104F0800EDD923689B68D907E9D5A36D43F0100351
:104F1800A365E36D43F00103E365BFE70225BEE740
:104F2800E8FFFF7F0749CA6822F4E062030212041F
:104F380003F4E063120C134343F0BF6343F40033FC
:104F4800CB60704700ED00E0164B30B5DC68C4F369
:104F58000224C4F10703251D042B28BF0423062DB2
:104F68004FF0FF358CBF033C002405FA03F321EA18
:104F78000303A54022EA0502A340002843EA0203EE
:104F8800ACBF00F16040084A4FEA0313B8BF00F015
:104F98000F00DBB2AABF00F56140135480F800335C
:104FA80030BD00BF00ED00E014ED00E0002807DB95
:104FB800044A4109012300F01F00834042F82130D0
:104FC800704700BF00E100E000280CDB43090649F8
:104FD80000F01F0020330122824041F82320BFF354
:104FE8004F8FBFF36F8F704700E100E070B5D0E9D5
:104FF80013456560446D14B1D0E916456560D0E984
:10500800105404F01C060124B4406C60046863600A
:105018008368102B0BBFA260A160E160E26070BDE5
:105028000268416CD3B210B5083B1424B3FBF4F307
:105038000B4CA24288BF0B4A21F0030199BF01F132
:10504800804202F50232521807338264064AC2646B
:1050580003F01F03012202FA03F3036510BD00BF2A
:10506800070402401C0802408008024038B50028A6
:105078005ED002682F4B9A424FF014014CD82E4B49
:105088001344B3FBF1F32D499B00C0E9101302232D
:1050980080F825301368056923F4FF4323F0700373
:1050A8001360D0E9024323432B43456911682B431E
:1050B80085692B43C5692B43056A2B430B43136052
:1050C800FFF7AEFFB4F5804F04BF0023436042688A
:1050D800816C02F07F030B60D0E91314013A032AB4
:1050E8004C6020D8164A174981651A44013B920042
:1050F800012103F0030301FA03F300214265C365AC
:105108001160114A536400230122C36380F82430DC
:1051180080F82520184638BD0C4B1344B3FBF1F337
:105128000B499B00B1E70023C0E91533C365EAE7E3
:105138000120F0E707040240F8FFFDBF000002402D
:105148003F8200104009024000090240F8FBFDBF01
:105158000004024038B5002841D00268136823F0E3
:10516800010313601F4B9A424FF0140130D81E4BB5
:105178001344B3FBF1F31D499B00C0E9101301244C
:1051880003F01C0304FA03F3002515604B60FFF7D6
:1051980047FF836C41681D60D0E913325A604A1E8C
:1051A800032A06D8124B0B449B0094401D60114BF8
:1051B8005C640023C363C0E91533C0E90B33C0E95D
:1051C8000D33C36580F8253080F82430184638BD83
:1051D800094B1344B3FBF1F308499B00CDE70120C9
:1051E800F5E700BF07040240F8FFFDBF00000240DA
:1051F8003F82001000090240F8FBFDBF0004024096
:1052080070B590F82450012D04463BD090F82560E5
:105218000125AE4280F824504FF000062CD102251B
:1052280080F825500568C6632E6826F001062E60B2
:10523800FFF7DCFE036BBBB12B6843F00E032B605A
:10524800A36C1A68D20342BF1A6842F480721A60CB
:10525800636D1BB11A6842F480721A602B6843F0C0
:1052680001032B60002070BD2B6823F004032B6022
:105278002B6843F00A03E2E78023C36380F82460C5
:105288002846F0E70220EEE7034640B190F82520D3
:10529800022A06D00422C263002280F824200120BA
:1052A80070470268806C116821F00E011160016876
:1052B80021F480710160116821F001011160D3E9C6
:1052C800100202F01C0101228A404260D3E9132136
:1052D80051605A6D32B1116821F480711160D3E9BF
:1052E800162151600122002083F8252083F824002C
:1052F800704710B590F82530022B03D00423C36300
:10530800012010BD03681A6822F00E021A601A689C
:1053180022F001021A60826C136823F48073136010
:10532800D0E9101303F01C02012393404B60D0E92D
:1053380013325A60436D33B11A6822F480721A60CE
:10534800D0E916325A60012380F82530836B002497
:1053580080F8244013B198472046D2E71846D0E792
:1053680070B4426C046C036826681D6802F01C0265
:105378000421914031420FD015F0040F0CD01A6867
:1053880092065EBF1A6822F004021A60036B61601D
:10539800002B33D070BC184702219140314217D0FE
:1053A80015F0020F14D01A68940606D41A6822F071
:1053B8000A021A60012280F82520114A93428CBF04
:1053C800104B114B5960002380F82430C36ADFE783
:1053D80008219140314211D029070FD5196821F0D1
:1053E8000E011960012303FA02F26260C36380F8B8
:1053F8002530002380F82430436BC9E770BC704720
:105408008000024000040240000002400A4A53693A
:1054180043F4802330B55361EFF3108472B6002350
:10542800CD58C5500433B3F5807FF9D11369DB0338
:10543800FCD484F3108830BD00400058064B5A69EC
:10544800002ABFBF054A9A6002F188329A60BABF43
:105458005869C00F00207047004000582301674575
:10546800044B5A6942F000425A615869C043C00F60
:10547800704700BF0040005870B50546FDF730FB87
:10548800124E04463369D90313D43369DA0744BF8B
:10549800012232614CF2FA32134011D10B4E3069BD
:1054A80010F480200BD0FDF71BFB001BA842F6D39D
:1054B80004E0FDF715FB001BA842E3D3032070BDF1
:1054C800024A1361024A01205360F8E7004000587D
:1054D800040700202DE9F041184D98462B78012B40
:1054E80006460C46174626D001232B704FF47A70D7
:1054F80000236B60FFF7C0FFA0B9012E16D1104A38
:10550800536943F0010353612760BFF36F8FC4F8F9
:1055180004804FF47A70FFF7AFFF094A536923EA12
:105528000603536100232B70BDE8F08139462046FD
:10553800FFF76CFFEDE70220F6E700BF0407002045
:1055480000400058054A536923F47E7343EAC000BB
:1055580040F4803040F0020050617047004000582D
:105568002DE9F041234F3B78012B054688463FD073
:1055780001233B704FF47A7000237B60FFF77CFFB8
:10558800044688B92B68042B13D11B4A536943F48A
:10559800803343F0040353614FF47A70FFF76CFFD4
:1055A8000446154B1A681B6800233B702046BDE86B
:1055B800F0814FF0FF33C8F800306E68D5E901324A
:1055C8001344B3420AD93046FFF7BCFF4FF47A7050
:1055D800FFF752FF50B1C8F800600446064A536905
:1055E80023F47E7323F002035361DAE70136E5E71B
:1055F8000224DBE704070020004000582DE9F04FA3
:10560800524C00234FF00F090A6832FA03F501D112
:10561800BDE8F08F012505FA03F818EA020200F048
:105628008E804E68032706F003054FEA430E07FAFB
:105638000EFC6F1E012F6FEA0C0C32D8876807EA40
:105648000C0ACF6807FA0EF747EA0A078760476827
:1056580027EA0808C6F300179F4047EA080747608B
:10566800C76807EA0C088F6807FA0EF747EA0807C1
:10567800022DC76017D14FEAD30800EB880803F062
:10568800070AD8F820704FEA8A0A09FA0AFB27EABB
:105698000B0B0F6907FA0AF747EA0B07C8F82070DF
:1056A80001E0032DDCD1076805FA0EF507EA0C07BF
:1056B8003D4316F4403F056041D023F0030707F14E
:1056C800804707F5803703F0030CBD684FEA8C0C60
:1056D8004FF0070E0EFA0CFEB0F1904F25EA0E0EB1
:1056E8002FD01B4DA8422ED005F58065A8420CBFCF
:1056F8000225072505FA0CF545EA0E05BD60256863
:10570800D74316F4801F0CBF3D40154325606568DC
:1057180016F4001F0CBF3D4015436560D4F8805057
:1057280016F4803F0CBF3D401543C4F88050D4F8B0
:105738008450B60354BF3D401543C4F88450013328
:1057480062E70025D6E70125D4E700BF0008005826
:1057580000040048374A2DE9F04F00234FF0010AB2
:105768004FF0070B4FF00F0931FA03F401D1BDE8F0
:10577800F08F0AFA03FC1CEA010654D023F0030454
:1057880004F1804404F5803403F00307A568BF00E2
:105798000BFA07F8B0F1904F08EA050E45D0264DF0
:1057A800A84244D005F58065A8420CBF022507250C
:1057B800BD40754517D1D2F8805025EA0605C2F8D4
:1057C8008050D2F8845025EA0605C2F8845015683E
:1057D80025EA06051560556825EA06055560A56899
:1057E80025EA0805A560056803265C0006FA04F4A6
:1057F80023FA06F6254300EB8606056003F0070545
:10580800376AAD0009FA05F527EA050737628568A2
:1058180025EA04058560456825EA0C054560C568E4
:1058280025EA0404C46001339EE70025C0E701258A
:10583800BEE700BF00080058000400480369194289
:1058480014BF0120002070470AB18161704781624E
:1058580070470000044AD168014208B502D0D06000
:10586800FEF706F808BD00BF0008005810B504464A
:1058780000284AD090F8413003F0FF021BB980F8A5
:105888004020FCF71DFE242384F8413023681A6861
:1058980022F001021A60626822F070621A619A6846
:1058A80022F400429A60D4E90221012924D142F469
:1058B80000429A605A6842F0007242F400425A600C
:1058C800DA6822F40042DA60D4E904210A43A169C3
:1058D80042EA0122DA60D4E907210A431A601A6809
:1058E80042F001021A6000202023606484F84130ED
:1058F800206384F8420010BD42F4044202299A60F1
:1059080004BF4FF400625A60D4E70120F3E710B5F2
:1059180090F84120202A0346D4B21CD190F84020A8
:10592800012A18D0242280F841200268106820F04B
:1059380001001060106820F4805010601068014366
:1059480011601168002041F00101116083F84140A5
:1059580083F8400010BD0220FCE710B590F8412004
:10596800202A0346D4B21BD190F84020012A17D030
:10597800242280F841200268106820F0010010609D
:10598800106820F4706040EA01211160116800205D
:1059980041F00101116083F8414083F8400010BDD7
:1059A8000220FCE7024A136843F4807313607047CF
:1059B800000400580D4B10B55B690C4628B99A05D0
:1059C80007D500F027F820B110BD9B0501D400F0E1
:1059D80019F8074A1369012C23F00403136101D154
:1059E80030BFF1E740BF20BF20BFEDE700040058FB
:1059F80000ED00E0024B186800F4C060704700BF7B
:105A080000040058024A136843F480431360704747
:105A1800000400580C4A136823F4804313600B4BAE
:105A28001B6832214B430A49B3FBF1F351698905DD
:105A380000D533B9536913F4007F14BF0320002045
:105A48007047013BF2E700BF00040058B80000208F
:105A580040420F000B4A136823F0070343F0020388
:105A68001360094B1A69012842F004021A6105D132
:105A780030BF1A6922F004021A61704740BF20BF84
:105A880020BFF6E70004005800ED00E04FF0B043F7
:105A98001868C0F3404070474FF0B0431868C0F32F
:105AA800400070474FF0B042536823F47F4343EA05
:105AB8000023536070474FF0B0431868C0F340604C
:105AC800704700007FB54FF0B0432C4AD3F8083137
:105AD800C0F3031003F00F0352F82040284A52F88D
:105AE8002330B4FBF3F4FFF785FF264B054693E814
:105AF8000700B5F5007F04AB03E9070010D0224B7F
:105B08009C4218D303F5B70303F67F539C4229D967
:105B180003F5741303F510639C4225D802230BE0A8
:105B28001A4B9C4207D91A4B9C421BD903F53703E1
:105B380003F5D853F0E7002304AA02EB830353F8D4
:105B48000C4C144D2B6823F0070323432B60FCF700
:105B5800C7FF06462B6803F007039C4206D10020C6
:105B680004B070BD0123E7E70024EAE7FCF7B8FFBB
:105B7800801B0228EED90320F2E700BFEC1C0108C5
:105B88008C1C010830140108C0CF6A00BFEA21014B
:105B98003F933402004000584FF0B04310B59A6864
:105BA800D96812F00C0205D00C2A4AD101F003037F
:105BB800012B50D14FF0B0412B480B6813F008036C
:105BC80006D00B6813F0080337D1D1F8941007E01A
:105BD8000C68240756BFD1F894300968C3F303232F
:105BE80050F82330002A0CBF184600204FF0B0416F
:105BF8008A6802F00C020C2A1ED1CA6802F003025D
:105C0800022A2ED0032A06D10B68184A13F4801FE3
:105C1800174B18BF13464FF0B042D068D168D2680E
:105C2800C0F306205843C1F302130133B0FBF3F06D
:105C3800530F0133B0FBF3F010BD0B68C3F303132C
:105C4800CEE7042A0AD0082A05D11B6813F480136A
:105C580004D10748CAE700231846C7E703480023CA
:105C6800C4E7024BD7E700BFEC1C01080024F4008E
:105C78000048E80108B5FFF78FFF4FF0B043044A2A
:105C88009B68C3F3031352F82330B0FBF3F008BD4D
:105C98008C1C01082DE9F0410446002853D04FF030
:105CA800B0439D68DE6803689B0605F00C0506F0A6
:105CB800030668D5026A1DB10C2D46D1012E44D1C8
:105CC800002A40D04FF0B043A16A1A68170756BFA0
:105CD800D3F894301B681B0903F0F00399421FD9CD
:105CE8000846FFF7EFFE00282DD14FF0B0421368A9
:105CF80043F0080313601368A16A23F0F0030B4311
:105D08001360606AFFF7CEFEFFF7B4FFAB4B186075
:105D1800AB4B1868FCF7E2FE002834D0BDE8F081F0
:105D28004FF0B042136843F008031360136823F080
:105D3800F0030B431360606AFFF7B4FE0846FFF7F1
:105D4800C1FE0028E0D00120E8E74FF0B043002A68
:105D580054D01A6842F001021A60FCF7C1FE0746E7
:105D6800FFF79AFE002842D04FF0B042136843F084
:105D7800080313601368A16A23F0F0030B43136050
:105D8800606AFFF78FFE2368D80748D4236899070D
:105D980000F18C8023681E0740F1FA80A3694FF058
:105DA800B046002B00F0E180D6F89430E16903F0AA
:105DB8001002914200F0C48003F00302022AC2D00C
:105DC800D80740F1B380D6F8943023F00103C6F821
:105DD8009430FCF785FE0746D6F89430990740F1D1
:105DE800A580FCF77DFEC31B112BF5D904E0FCF759
:105DF80077FEC01B0228B3D903208FE71A6822F068
:105E080001021A60FCF76CFE0746FFF745FE002802
:105E1800B9D0FCF765FEC01B0228F6D9ECE7082DBF
:105E280003D00C2D05D1032E03D16368002BADD10F
:105E380089E74FF0B043A1681A6822F480120A4338
:105E48001A606268B2F5803F10D11A6842F4803255
:105E58001A60FCF745FE0746FFF718FE002895D1A3
:105E6800FCF73EFEC01B6428F6D9C5E7B2F5041F4F
:105E780004D11A6842F400121A60E6E7196821F49E
:105E880080311960196821F400111960002AE0D1E5
:105E9800FCF726FE0746FFF7F9FD00283FF476AF2A
:105EA800FCF71EFEC01B6428F5D9A5E7042D23695D
:105EB80003D00C2D0ED1022E0CD1002B3FF443AF92
:105EC8004FF0B0426169536823F0FE4343EA01632F
:105ED80053605FE74FF0B046BBB1336843F480735B
:105EE8003360FCF7FDFD074633685A0507D573682C
:105EF800626923F0FE4343EA026373604AE7FCF7F2
:105F0800EFFDC31B022BEFD976E7336823F48073C8
:105F18003360FCF7E5FD074633685B057FF53AAF6C
:105F2800FCF7DEFDC31B022BF6D965E74FF0B04244
:105F3800E169D2F8943023F010030B43C2F894308F
:105F48004FF0B047D7F8943043F00103C7F89430C6
:105F5800FCF7C6FD0646D7F894309A0718D4FCF724
:105F6800BFFD831B112BF6D946E7D6F8943023F0F2
:105F78000103C6F89430FCF7B3FD0746D6F8943011
:105F88009B0705D5FCF7ACFDC31B112BF6D933E7EE
:105F98002368580754D50B4F3B68D90514D4FFF72D
:105FA80001FDFCF79DFD06463B68DA050CD4FCF7BD
:105FB80097FD831B022BF7D91EE700BFB80000200E
:105FC800BC00002000040058E3684FF0B046002BE6
:105FD80058D023F08003052B02BFD6F8903043F049
:105FE8000403C6F890304FF0B046FCF779FDD6F8B8
:105FF800903043F001030746C6F8903041F28838E4
:10600800D6F890309B0705D4FCF76AFDC31B4345BF
:10601800F6D9F1E6E36823F00403812B1BD1FCF7E2
:106028005FFDD6F8903043F08003C6F890300746FD
:106038004FF0B04641F28838D6F89030180504D5AC
:10604800E06A00284AD1002068E6FCF749FDC01B39
:106058004045F1D9D0E6FCF743FDD6F8903023F05F
:106068008003C6F8903007464FF0B04641F28838B2
:10607800D6F890301905E3D5FCF732FDC01B404532
:10608800F6D9B9E6FCF72CFDD6F8903023F080035A
:106098000746C6F8903041F28838D6F890301A058D
:1060A80016D4FCF71DFDD6F8903023F00103C6F88E
:1060B800903007464FF0B04841F28836D8F8903013
:1060C8009B07BDD5FCF70CFDC31BB342F6D993E67D
:1060D800FCF706FDC01B4045DFD98DE60C2D4ED0E0
:1060E8004FF0B04302281A6822F080721A6033D148
:1060F800FCF7F6FC0546FFF7DEFC38BBD4E90C31AB
:106108004FF0B0420B43D0682D4901400B43E16B7F
:106118000B43216C0B43616C0B43A16B43EA0123D6
:10612800D360136843F080731360D36843F08053DF
:10613800D360FCF7D5FC0446FFF7BDFC002882D1EC
:10614800FCF7CEFC001B0A28F6D955E6FCF7C8FC7C
:10615800401B0A28CFD94FE6FCF7C2FC0446FFF7DC
:10616800AAFC30B94FF0B042164BD1680B40D3604F
:10617800D4E5FCF7B5FC001B0A28F0D93CE6012859
:106188003FF4CCAD4FF0B043226BDB6803F0030162
:1061980091427FF4D8AD616B03F070028A427FF4BC
:1061A800D2ADA16B03F4FE42B2EB012F7FF4CBAD6D
:1061B800626C03F0604393423FF445AFC3E500BF10
:1061C8008C80C111FCFFFEEE2DE9F0410D4604461E
:1061D80010B90120BDE8F081684E336803F0070369
:1061E8008B4216D323689A0727D54FF0B047A26889
:1061F800BB6823F0F0031343BB60FCF771FC064651
:10620800BB68DB0319D4FCF76BFC831B022BF7D9A3
:1062180011E0336823F007030B433360FCF760FC9D
:106228000746336803F00703AB42DBD0FCF758FCA2
:10623800C01B0228F5D90320CCE72368580617D5D8
:106248004FF0B0476269D7F8083123F00F0343EAEB
:106258001213C7F80831FCF743FC0646D7F8083193
:10626800D90305D4FCF73CFC831B022BF6D9E2E7E3
:1062780023685A0713D54FF0B047E268BB6823F488
:10628800E0631343BB60FCF72BFC0646BB689B032B
:1062980005D4FCF725FC831B022BF7D9CBE7236831
:1062A800180714D54FF0B0472269BB6823F4605330
:1062B80043EAC203BB60FCF713FC0646BB685903FC
:1062C80005D4FCF70DFC831B022BF7D9B3E7236831
:1062D800DA070FD4294C236803F00703AB4239D8F7
:1062E800FFF7C8FC264B1860264BBDE8F04118683C
:1062F800FCF7F4BB6268022A1DD1FFF7C7FB002830
:106308003FF467AF4FF0B04641F28838B36823F0E6
:1063180003031343B360FCF7E3FB0746B368626803
:1063280003F00C03B3EB820FD4D0FCF7D9FBC01BEE
:106338004045F3D97FE7032A02D1FFF7BCFBDEE72C
:1063480012B9FFF7A9FBDAE74FF0B0431B685B050A
:10635800D8D43EE7236823F007032B432360FCF7D8
:10636800BFFB0646236803F00703AB42B8D0FCF72F
:10637800B7FB801B0228F5D95DE700BF0040005835
:10638800B8000020BC00002008B5FFF773FC4FF0F0
:10639800B043044A9B68C3F3022352F82330D84021
:1063A80008BD00BFCC1C010808B5FFF763FC4FF01F
:1063B800B043044A9B68C3F3C22352F82330D84041
:1063C80008BD00BFCC1C01084FF0B043D3F89000C3
:1063D800C0F3400070474FF0B0410209D1F888304F
:1063E80002F47F22000123EA020300F47F20034322
:1063F800C1F8883070474FF0B041020CD1F88830AE
:10640800120423EA020343EA0040C1F888007047F7
:1064180070B5066816F48036044638D0FFF7C2FA1D
:10642800FCF75EFB614E05463368DB0529D54FF066
:10643800B043616BD3F8902002F44072914214D0BB
:10644800D3F89010D3F8902042F48032C3F890200B
:10645800D3F8902021F4407022F480328D07C3F8DD
:106468009020C3F8900000F190804FF0B042616B2B
:10647800D2F8903023F440730B43C2F890300026D2
:1064880005E0FCF72DFB401B0228CDD90326256823
:10649800E8070AD54FF0B0416268D1F8883023EA9E
:1064A800124392B21343C1F88830A9070AD54FF0B6
:1064B800B041A268D1F8883023EA124392B213435C
:1064C800C1F88830AA0609D54FF0B0422169D2F840
:1064D800883023F440630B43C2F88830AB0502D5FB
:1064E800206AFFF788FF680502D5606AFFF783FF17
:1064F800290502D5A06AFFF77EFF6A0602D5606902
:10650800FFF769FF2B0602D5A069FFF764FFE805CE
:1065180002D5E069FFF75FFFE90610D54FF0B042FA
:10652800E168D2F8883023F440730B43C2F888300E
:10653800B1F5807F02BFD36843F08073D3602A042B
:106548000ED54FF0B042216BD2F8883023F040438B
:106558000B43C2F8883019B9D36843F08073D3600D
:106568006B0410D54FF0B042E16AD2F8883023F0BE
:1065780040530B43B1F1005FC2F8883003D1D368B0
:1065880043F48033D360304670BDFCF7A9FA41F27A
:1065980088360546FFF718FF01283FF466AFFCF779
:1065A8009FFA401BB042F5D970E700BF00040058BD
:1065B80030B590F82C30012B02464FF0020022D063
:1065C800174B82F82D00CA24012582F82C505C62F2
:1065D80053245C62B1F5807F146B996914D121F45E
:1065E80088519961596C24F0010421F000415964E3
:1065F8001463DD650A4BFF2159620020012382F8EC
:106608002D3082F82C0030BD21F408519961D96CE5
:1066180024F0020421F00041D9641463D865E9E745
:106628000028004070B50B4E036B756D1D40EA07DE
:10663800044603D50123F365FCF7C3FBAB0704D578
:106648000223F365204600F0CBF9012384F82D30AE
:1066580070BD00BF0028004038B50A4CE36823F03D
:106668002003E360FCF73CFA0546E3689B0601D586
:10667800002038BDFCF734FA401BB0F57A7FF4D916
:106688000320F6E7002800402DE9F041114DEC68A1
:1066980014F0400407461AD1EB6843F08003EB601E
:1066A800FCF71EFA4FF003080646EB685B0601D4B8
:1066B800032C02D12046BDE8F081FCF711FA801BBB
:1066C800B0F57A7F84BF87F82D800324EDE7002496
:1066D800F0E700BF0028004038B50F4CE36823F00E
:1066E8008003E360A3699B06054606D4FFF7B4FF61
:1066F80010B1032085F82D0038BDA36923F02003CD
:10670800A361FFF7A9FF10B1032085F82D00A36945
:1067180043F02003A361EFE70028004038B50446A2
:1067280000284BD090F82D3003F0FF021BB980F8F9
:106738002C20FBF7D3FF0223214D84F82D30EB6882
:10674800DB0632D4CA236B6253236B622046FFF701
:106758009BFF78BBAB6923F08E6323F04003AB61EA
:1067680021696368AA690B431343A2691343AB61A8
:10677800D4E9022343EA02432B61D4E90931EA68E8
:106788000B4322F4F8521343EB602046FFF7A4FFB3
:1067980080B9D4E90713AA690B4322F06042134376
:1067A80062691343AB61FF236B62012384F82D30C8
:1067B800002002E0024BFF225A6238BD0120FCE7AC
:1067C800002800400023092803D840EA0310C0B27B
:1067D80070470A380133C0B2F5E700002DE9F047E9
:1067E80090F82C30012B05464FF0020069D00123A8
:1067F80085F82C304E4B85F82D00DE6806F440767F
:10680800B6F5807F78D04C69087891F8019091F8B6
:1068180002A091F82470002A55D19B6913F0400317
:1068280008BFCB70FFF7CEFF80464846FFF7CAFF88
:1068380002465046FFF7C6FF81463846FFF7C2FFBB
:106848000B6ACF78234343EA875343EA090343EAB1
:10685800084343EA022343EA0063354ACA205062E8
:10686800532050628C6A8869B4F5807F946945D159
:1068780024F4885494610124D465B6F5807F09BF57
:10688800CB6913640343536418BF5064284B4A68A8
:106898001A672A6B42F001022A639A6942F4885205
:1068A8009A61244AD2F8803043F40033C2F8803029
:1068B8001F4BFF225A620020012385F82D3085F8EE
:1068C8002C00BDE8F087B4F1803F07D0B4F5000F85
:1068D80004D09B6913F0400308BFCB700B6ACA78D9
:1068E8001C4344EA0A0444EA004343EA092343EA0E
:1068F800825343EA0763B0E70023AEE724F4085461
:1069080094610224D465B6F5807F09BFCB6993648E
:106918000343D36418BFD064054B4A685A672A6B8F
:1069280042F002022A639A6942F40852B8E700BFAB
:10693800002800400008005890F82C20012A03463F
:106948004FF0020012D00A4A83F82D00CA21516282
:1069580053215162916941F020019161FF215162F7
:106968000020012283F82D2083F82C00704700BFF7
:106978000028004090F82C20012A03464FF002001E
:1069880019D00D4A83F82D00CA2151625321516252
:1069980091690A4841F080019161D0F8801041F472
:1069A8008021C0F88010FF2151620020012283F865
:1069B8002D2083F82C00704700280040000800585C
:1069C800064B5A6D520610B5044603D54022DA65C7
:1069D800FCF7FAF9012384F82D3010BD0028004097
:1069E8007047890001F1804101F531410A60704723
:1069F800890001F1804101F53141086870470000C4
:106A0800034AD2F8903043F40043C2F890307047FC
:106A180000040058034AD2F8903023F40043C2F827
:106A28009030704700040058074B1A6822F0400263
:106A38001A6040F441704FF4B85218605A601A68EE
:106A480042F040021A6070470000015837B5054609
:106A580000284ED0837903F0FF046BB1032C0BD0D0
:106A6800254B4FF400629A612868FFF7DDFF002488
:106A780001232B71AC602FE000236B712846FBF7D4
:106A880045FF1E4AD2F8903043F48053C2F8903044
:106A9800002CE5D102234FF0B042AB71D2F894300C
:106AA80023F40043C2F89430154B1B681C214B4358
:106AB800DB0C64214B430193019B93B90124AC6027
:106AC800FFF79EFF0C4B9A6842F400629A604FF4FD
:106AD80000629A61002CC7D00123AB71204603B035
:106AE80030BD019B013B0193D2F894305B04E3D4A1
:106AF800E6E70124F2E700BF000400580008005848
:106B0800B800002037B5174D2B6802461C204343B8
:106B1800DB0C6420434314480193019B93B9012083
:106B28009060114C21732B681C214B43DB0C6421B2
:106B38004B430193019B6BB9012090600A4BDB68C2
:106B480003B030BD019B013B019383689C07E4D5EA
:106B58000020E6E7019B013B0193A368DB07E9D529
:106B6800ECE700BFB80000200000015837B5184D09
:106B78002B6802461C204343DB0C64204343154822
:106B88000193019BA3B901209060124CFF2323734A
:106B98002B681C256B43DB0C64256B430193019B1D
:106BA80073B9012090600B4BDB680B7003B030BDEC
:106BB800019B013B019383689C07E2D50020E4E731
:106BC800019B013B0193A368DB07E8D5EBE700BF16
:106BD800B8000020000001580F4B13B51B680F4C7C
:106BE800182253431B0D64225343014601936269E3
:106BF800019B02F0040223B902238B60012002B03A
:106C080010BD019B013B0193606910F00200F6D0B2
:106C1800002AECD11046F2E7B80000200004005822
:106C280007B50379012B0FD10A4B1B681822534370
:106C38001B0C0193FFF7EEFE019B013B0193019BA7
:106C4800002BF9D1FFF7DCFE03B05DF804EBFFF78A
:106C5800C3BF00BFB8000020F8B51E468379012BDA
:106C6800154604460F46DAB22DD14379012B2AD0B6
:106C7800022342718371FFF7D3FF0D212046FFF7EE
:106C8800C9FEFFF73FFF390A2046FFF73BFFF9B27D
:106C98002046FFF737FF2E44B5420ED12046FFF7B6
:106CA800AFFEFFF799FFA06801230038A3714FF0EA
:106CB800000318BF01206371F8BD15F8011B2046B9
:106CC800FFF720FFE8E70220F6E7F8B51E468379CC
:106CD800012B154604460F46DAB22FD14379012B12
:106CE8002CD04271FFF79CFF1D212046FFF792FE32
:106CF800FFF708FF390A2046FFF704FFF9B22046DC
:106D0800FFF700FF00212046FFF7FCFE2E44B542A6
:106D18000ED12046FFF774FEFFF75EFFA06801233F
:106D28000038A3714FF0000318BF01206371F8BD4C
:106D380029462046FFF71AFF0135E8E70220F6E763
:106D4800F8B51F468379012B154604460E46DAB27C
:106D58002CD14379012B29D04271FFF761FF06F04E
:106D6800EF03A3F184025342534123713146204675
:106D7800FFF750FEFFF7C6FE2F44AF4210D1FFF7D2
:106D88003FFE842E02D02046FFF726FFA06801238D
:106D98000038A3714FF0000318BF01206371F8BDDC
:106DA80015F8011B2046FFF7ADFEE6E70220F6E7DF
:106DB800F8B51E468379012B154604460F46DAB20C
:106DC80027D14379012B24D04271FFF729FF394697
:106DD8002046FFF71FFEFFF795FE00212046FFF72C
:106DE80091FE2E44B5420ED12046FFF709FEFFF76B
:106DF800F3FEA06801230038A3714FF0000318BF09
:106E080001206371F8BD29462046FFF7AFFE013522
:106E1800E8E70220F6E737B50023ADF8043001AA09
:106E2800022312210546FFF7C3FFBDF804400223E1
:106E380064BA01AAA4B219462846FFF781FFE207FF
:106E480002D5284609F076FBA30702D5284609F0A3
:106E580077FB600702D5284609F09CFB210702D57D
:106E6800284609F09DFBE20602D5284609F09EFB5C
:106E7800A30602D5284609F087FB600602D52846F6
:106E880009F064FB210606D514F4807118BF0121AE
:106E9800284609F061FBA20502D5284609F06CFBDB
:106EA800630402D5284609F087FB03B030BDF8B566
:106EB8001E468379012B154604460F46DAB227D1C0
:106EC8004379012B24D04271FFF7AAFE0E212046F8
:106ED800FFF7A0FDFFF716FE39462046FFF712FE22
:106EE8002E44B5420ED12046FFF78AFDFFF774FE07
:106EF800A06801230038A3714FF0000318BF0120D8
:106F08006371F8BD15F8011B2046FFF7FBFDE8E7A4
:106F18000220F6E7F8B51E468379012B154604468C
:106F28000F46DAB22BD14379012B28D04271FFF7F3
:106F380077FE1E212046FFF76DFDFFF7E3FD39467A
:106F48002046FFF7DFFD00212046FFF7DBFD2E443A
:106F5800B5420ED12046FFF753FDFFF73DFEA0686E
:106F680001230038A3714FF0000318BF012063719B
:106F7800F8BD29462046FFF7F9FD0135E8E702206C
:106F8800F6E7026852E8003F23F0C00342E8003108
:106F980002680029F5D102F1080353E8003F23F401
:106FA800000302F1080C4CE800310029F3D120233A
:106FB800C0F888307047000010B5026852E8003FFA
:106FC80023F4907342E8003102680029F5D10F4C90
:106FD80002F1080353E8003F234002F1080C4CE893
:106FE80000310029F4D1C36E012B07D152E8003FCC
:106FF80023F0100342E800310029F7D12023C0F81C
:107008008C300023C366436710BD00BFFEFFFFEF4F
:10701800F8B504461346D4F88850202D32D1F1B182
:10702800EAB1E06FA4F85620A4F8542000262122E3
:10703800C4F890602165C4F88820226888B1124F8E
:10704800C762124F0763124F2832C0E90D76FEF768
:10705800D7F830B11023C4F89030C4F88850012014
:107068000FE0236840221A62226802F1080353E8FD
:10707800003F43F0800302F1080141E80030002896
:10708800F3D1F8BD0220FCE79D700008E570000808
:10709800F170000808B50346806A1B681B6813F086
:1070A800200317D1A0F85630026802F1080353E80C
:1070B800003F23F08003083242E8003102680029CB
:1070C800F2D152E8003F43F0400342E80031002982
:1070D800F7D108BDFBF7CEFFFBE7704708B5806A1C
:1070E800FFF7FBFF08BD7047806A38B50468D0F821
:1070F8008830D0F88C50A268120606D5212B04D10E
:107108000023A0F85630FFF73CFFA3685B0606D5BE
:10711800222D04D10023A0F85E30FFF74DFFD0F8F0
:10712800903043F01003C0F89030FFF7DCFF38BD13
:1071380008B5806A0023A0F85E30A0F85630FFF743
:10714800D2FF08BD704700000368D9691A682DE9A5
:10715800F04140F60F0631429D68044610D18E0674
:1071680040F1978002F0200605F080573E4300F07A
:107178009080436F002B00F08580BDE8F0411847F0
:10718800AB4EAC482E401040304300F08280CF0711
:1071980009D5D00507D501201862D4F8900040F031
:1071A8000100C4F890008F0709D5E80707D5022029
:1071B8001862D4F8900040F00400C4F890004F071B
:1071C80009D5E80707D504201862D4F8900040F0E4
:1071D8000200C4F890000F070BD502F020003043DE
:1071E80007D008201862D4F8900040F00800C4F8CE
:1071F80090000E050AD5500108D54FF400601862BA
:10720800D4F8903043F02003C4F89030D4F890308C
:10721800002B37D08B0609D502F0200205F08055E7
:107228002A4303D0636F0BB1204698472668D4F8E9
:107238009020B36802F0280203F0400353EA0205E5
:10724800204621D0FFF7B8FEB3685F0617D522683D
:1072580002F1080353E8003F23F04003083242E8F4
:1072680000310029F3D1D4F8800040B1724B836318
:10727800FEF73FF830B1D4F88000836B7DE72046F5
:10728800FFF731FFBDE8F081FFF72DFFC4F89050FC
:10729800F8E7E06E012840F08980CE0640F186804C
:1072A800D00640F1838010221A629A6851064BD5A5
:1072B800D4F8802011684A6892B2002AE2D0B4F863
:1072C8005C009042DED9A4F85E200A6892062FD4AA
:1072D80053E8002F22F4807243E800210029F7D1F7
:1072E80003F1080252E8002F22F0010203F108001E
:1072F80040E800210029F3D103F1080252E8002FE9
:1073080022F0400203F1080040E800210029F3D1EF
:107318002022C4F88C20E16653E8002F22F01002E6
:1073280043E800210029F7D1D4F88000FDF7ACFF2D
:1073380002232367B4F85E30B4F85C10C91A89B226
:107348002046FFF7FFFE9DE7B4F85E20B4F85E0024
:10735800B4F85C1080B292B2002893D0891A89B22E
:1073680000298FD053E8002F22F4907243E80020C0
:107378000028F7D1314D03F1080252E8002F2A40C6
:1073880003F1080646E800200028F4D12022C4F8BA
:107398008C206067E06653E8002F22F0100243E873
:1073A80000200028F7D102232367C9E7CF0209D5B7
:1073B8006E0207D54FF4801220461A62BDE8F041EC
:1073C80000F0A0BD08060BD502F0800005F400050A
:1073D800284305D0A36F002B3FF454AF2046CCE6DA
:1073E8004F0611D556060FD553E8002F22F040025C
:1073F80043E800210029F7D12023C4F88830A16789
:107408002046FBF737FE3DE70D0206D5500004D5B0
:107418002046BDE8F04100F077BDCB017FF532AFE3
:10742800002ABFF62FAF2046BDE8F04100F06BBD43
:10743800010000102001000439710008FEFFFFEF71
:10744800D0F88C20B0F86010222A08B5036855D10E
:107458005B6A826D0B401370836D01338365B0F8EE
:107468005E30013B9BB2A0F85E30B0F85E309BB254
:10747800002B42D1026852E8003F23F4907342E89F
:10748800003103680029F5D103F1080252E8002F02
:1074980022F0010203F1080C4CE800210029F3D185
:1074A8002022C0F88C20184A41679342016705D111
:1074B800C26E012A0ED0FBF7EBFD1EE05A681102DE
:1074C800F6D553E8002F22F0806243E80021002916
:1074D800F7D1EDE70022C26653E8002F22F0100230
:1074E80043E800210029F7D1DA69B0F85C10D20628
:1074F80044BF10221A62FFF725FE08BD9A6942F0C0
:1075080008029A61F9E700BF00800040D0F88C209B
:10751800B0F86010222A08B5036852D15A6A11409F
:10752800826D22F8021B8265B0F85E20013A92B2A1
:10753800A0F85E20B0F85E2092B2002A40D153E84D
:10754800002F22F4907243E800210029F7D103F1BB
:10755800080252E8002F22F0010203F1080C4CE85F
:1075680000210029F3D12022C0F88C20174A416756
:107578009342016705D1C26E012A0ED0FBF788FD40
:107588001EE05A681102F6D553E8002F22F08062F7
:1075980043E800210029F7D1EDE70022C26653E84D
:1075A800002F22F0100243E800210029F7D1DA6900
:1075B800B0F85C10D20644BF10221A62FFF7C2FD71
:1075C80008BD9A6942F008029A61F9E70080004014
:1075D8002DE9F74F0368B0F86080DF691A689D6885
:1075E800D0F88C1001922229044640F0B480B0F8FB
:1075F8006890DFF86CA1DFF86CB10026B9F1000FD4
:1076080001D0BB0621D4B4F85E309BB2D3B1B4F834
:1076180068209A4216D9226802F1080353E8003F0D
:1076280023F08053083242E8003122680029F2D161
:107638004D4B636752E8003F43F0200342E80031B6
:107648000029F7D103B0BDE8F08F2368A26D5B6A0B
:1076580003EA08031370A36D0133A365B4F85E3021
:10766800013B9BB2A4F85E302368DF6978072CD011
:10767800F9070AD5019AD20507D501211962D4F86C
:10768800901041F00101C4F89010B80709D5E90736
:1076980007D502211962D4F8901041F00401C4F80A
:1076A80090107A0709D5E80707D504211962D4F89C
:1076B800903043F00203C4F89030D4F8903023B1EE
:1076C8002046FFF710FDC4F89060B4F85E309BB216
:1076D800002B93D1216851E8003F23F4807341E8DF
:1076E800003023680028F5D103F1080252E8001F92
:1076F80001EA0A0142E800100028F5D120215B4583
:10770800C4F88C10606720670AD05968090207D549
:1077180053E8001F21F0806143E800100028F7D1EA
:10772800E16E012913D1E66653E8001F21F010012C
:1077380043E800100028F7D1D969CA0644BF1021D0
:1077480019622046B4F85C10FFF7FCFC56E72046A7
:10775800FBF79EFC52E79A6942F008029A6171E7CA
:10776800FEFFFFEF00800040497400082DE9F74F45
:107778000368B0F86080DF691A689D68D0F88C10DB
:1077880001922229044640F0B280B0F86890DFF8F0
:1077980068A1DFF868B10026B9F1000F01D0BB0677
:1077A80021D4B4F85E309BB2D3B1B4F868209A42C1
:1077B80016D9226802F1080353E8003F23F08053EA
:1077C800083242E8003122680029F2D14C4B636745
:1077D80052E8003F43F0200342E800310029F7D186
:1077E80003B0BDE8F08F2368A26D596A08EA010169
:1077F80022F8021BA265B4F85E20013A92B2A4F8FE
:107808005E20DF6978072CD0F9070AD5019AD205DE
:1078180007D501211962D4F8901041F00101C4F88C
:107828009010B80709D5E90707D502211962D4F8DD
:10783800901041F00401C4F890107A0709D5E807C0
:1078480007D504211962D4F8903043F00203C4F834
:107858009030D4F8903023B12046FFF744FCC4F8A8
:107868009060B4F85E309BB2002B95D1216851E846
:10787800003F23F4807341E8003023680028F5D1E5
:1078880003F1080252E8001F01EA0A0142E8001069
:107898000028F5D120215B45C4F88C10606720676B
:1078A8000AD05968090207D553E8001F21F0806102
:1078B80043E800100028F7D1E16E012913D1E666EC
:1078C80053E8001F21F0100143E800100028F7D109
:1078D800D969CA0644BF102119622046B4F85C1061
:1078E800FFF730FC58E72046FBF7D2FB54E79A69CC
:1078F80042F008029A6173E7FEFFFFEF0080004044
:107908001575000838B5044603682169A2681D6822
:10791800C0690A4361690A437D49024329400A4311
:107928001A605A68E16822F440520A435A60794A58
:10793800A16993421CBF226A11439A6822F06E42E1
:1079480022F430620A439A60DA6A616A22F00F020E
:107958000A43DA62704A93421CD14FF0B043D3F81D
:10796800883003F0030343F44033A3F54033013B6D
:10797800022B00F2C780694A9B5CB0F5004F40F0CB
:107988008980082B24D8DFE803F061C08323802393
:1079980023236500624A934209D14FF0B043614AFC
:1079A800D3F8883003F00C0343F44023E4E7594A42
:1079B80093420DD14FF0B043D3F8883003F44063BD
:1079C800B3F5006F1AD005D853B1B3F5806F12D054
:1079D800012009E0B3F5406FFAD14FF400400EE002
:1079E800FEF7D2FC58B900204FF00113A36600231C
:1079F800C4E91D3338BDFEF7CFF8F3E74A48656898
:107A08004A4B626A05EB450133F81220B0FBF2F3EA
:107A18009942DDD8B3EB053FDAD800231946FAF7C7
:107A280073F8090241EA10616B080002C0182A467F
:107A38004FF0000341F10001FAF766F83C4BA0F55E
:107A480040729A42C4D82368D860CCE7FEF79CFC01
:107A58000028C8D06168354B626A33F81220B0FB41
:107A6800F2F24B0803EB42034FF6EF72B3FBF1F36C
:107A7800A3F110019142ABD823F00F02216892B212
:107A8800C3F342031343CB60ADE7FEF785F8DFE7A6
:107A98002548DFE7082B9BD801A252F823F000BF46
:107AA800F17A0008FD7A0008097B0008D9790008F6
:107AB800037B0008D9790008D9790008D97900082A
:107AC800CD7A00084FF400406368616A174A32F8BB
:107AD8001120B0FBF2F000EB5300B0FBF3F04FF6CF
:107AE800EF73A0F11002ACE7FEF74EFC00283FF45C
:107AF8007AAFE9E7FEF758FCF8E7FEF74DF8F5E747
:107B08000948E1E7B0F5004FF4D1FEF74DFC9FE7D7
:107B1800F369FFCF00800040003801402C1D0108A8
:107B2800004400402F1DF5070024F4003C1D010807
:107B3800FFFC0F00836ADA0710B506D50168C46A2E
:107B48004A6822F4003222434A609C0706D501683D
:107B5800046B4A6822F4803222434A60590706D5EA
:107B68000168446B4A6822F4802222434A601A075B
:107B780006D50168846B4A6822F4004222434A60B1
:107B8800DC0606D50168C46B8A6822F48052224359
:107B98008A60990606D50168046C8A6822F4005246
:107BA80022438A605A060FD50168446C4A6822F459
:107BB80080122243B4F5801F4A6005D14A68846C5C
:107BC80022F4C00222434A601B0606D50268C16C33
:107BD800536823F400230B43536010BD2DE9F04193
:107BE800DDF8188004460E4615461F462268D369FC
:107BF80036EA03030CBF01230023AB4201D0002067
:107C080027E0B8F1FF3FF2D0FAF76AFFC01B404502
:107C1800206802D8B8F1000F1DD150E8003F23F4C6
:107C2800D07340E80032002AF7D100F1080353E886
:107C3800003F23F0010300F1080141E80032002A67
:107C4800F3D12023C4F88830C4F88C3084F8842019
:107C58000320BDE8F08103685A07C7D5C3691B052F
:107C6800C4D54FF40063036250E8003F23F4D07397
:107C780040E80032002AF7D100F1080353E8003F3A
:107C880023F0010300F1080141E80032002AF3D192
:107C98002023C4F88830C4F88C30C4F89030D5E775
:107CA80073B504460026C0F89060FAF719FF2368F8
:107CB8001B681A07054619D423681B685B070AD591
:107CC8006FF07E43009300222B464FF4800120463C
:107CD800FFF784FFB0B900202023C4F8883084F867
:107CE8008400C4F88C30E06620670CE06FF07E43B7
:107CF8000093324603464FF400112046FFF76EFF0B
:107D08000028D9D0032002B070BD10B5044650B386
:107D1800D0F888301BB980F88430FBF797F82268D0
:107D28002423C4F88830136823F001031360204625
:107D3800FFF7E8FD012816D0A36A13B12046FFF724
:107D4800F9FE23685A6822F490425A609A6822F031
:107D58002A029A601A6842F0010220461A60BDE8B9
:107D68001040FFF79DBF012010BD000030B58165B0
:107D78008168A0F85C200023B1F5805FA0F85E2040
:107D8800436735D10369002B40F2FF1318BFFF2367
:107D9800A0F860300023C0F890302223C0F88C305F
:107DA800016801F1080353E8003F43F0010308317B
:107DB80041E800340368002CF2D1456E84680169FB
:107DC800B5F1005F34D1B0F86850954230D8B4F5B9
:107DD800805F1DD1254A264C002918BF22464267DC
:107DE800C1B153E8002F42F4807243E80021F7E75D
:107DF80029B90369002B14BF7F23FF23C8E7B1F11A
:107E0800805FC5D10369002B0CBF7F233F23BFE7E9
:107E1800174AE4E703F1080252E8002F42F08052C3
:107E280003F1080040E800210029F3D1002030BD0B
:107E3800B4F5805F0FD10F4A0F4C002918BF2246B6
:107E4800426751B153E8002F42F4907243E8002191
:107E58000029F7D1EAE7084AF2E753E8002F42F091
:107E6800200243E800210029F7D1DFE775770008F1
:107E7800D97500081575000849740008D0F88C30C9
:107E8800202B30B415D1B9B1B2B100230468C36650
:107E98000A4B9C420AD063681B0207D554E8003F8E
:107EA80043F0806344E80035002DF7D130BCFFF77C
:107EB8005DBF022030BC70470120FBE70080004016
:107EC800436E30B52BB90123A0F86A30A0F86830AA
:107ED80030BD0368094D9A689968094C490FC2F387
:107EE80042626B5C615CDB00B3FBF1F3A0F86A30C3
:107EF800AB5CA25CDB00B3FBF2F3E7E75C1D0108B7
:107F0800541D01087047704770471FB504AB03E95B
:107F1800060090F88430012B04463AD0012380F8FB
:107F280084302423C0F8883003681A6822F00102DC
:107F38001A609A6822F440120A439A6071B95A6822
:107F4800BDF80C009DF80E1022F0100202435A6092
:107F58005A6822F07F4242EA01625A601A6842F087
:107F680001021A60FAF7BCFD6FF07E4203460092E8
:107F78004FF4800100222046FFF730FE38B9202355
:107F8800C4F88830002384F8843004B010BD03207E
:107F9800F8E70220F9E790F88430012B0FD001238D
:107FA80080F88430016851E8002F42F0020241E86D
:107FB8000023002BF6D180F8843018467047022041
:107FC800704710B590F88430012B044617D024234D
:107FD800C0F8883003681A68196821F0010119602F
:107FE80042F000524FF0005141661A60FFF768FFF7
:107FF8002023C0F88830002084F8840010BD0220B7
:10800800FCE770B590F88430012B044617D005685A
:108018002423C0F888302E682B6823F001032B60D6
:10802800AB6823F060431943A960FFF749FF202399
:108038002E60C0F88830002084F8840070BD0220CB
:10804800FCE770B590F88430012B044617D005681A
:108058002423C0F888302E682B6823F001032B6096
:10806800AB6823F060631943A960FFF729FF202359
:108078002E60C0F88830002084F8840070BD02208B
:10808800FCE7000038B5084D052455F8043B2BB92A
:10809800013C14F0FF04F8D1204638BDDB6898474E
:1080A8000028F5D0F9E700BF38080020034BD87046
:1080B800034B1B681B6C03B1184770474C08002022
:1080C80034080020034B1874034B1B685B6C03B126
:1080D800184770474C08002034080020F0B5314D8F
:1080E800314B95F90420314E91B00C46012795F992
:1080F80005108DF8047002288DF809208DF80A10F3
:1081080010D18DF80800D8711C7202F09FFD3378E9
:1081180003B114B101A803F003FA254B059A1A60BC
:1081280011B0F0BD59714FF480711A71D9801C7269
:1081380033788DF8087053BB1F2306A88DF81C20D0
:108148008DF8183002F064FF20238DF8183006A847
:108158002B798DF81C3002F05BFF22238DF8183044
:1081680006A86B798DF81C3002F052FF21238DF898
:10817800183006A86B798DF81C3002F049FF2923C6
:108188008DF8183006A80B4B079302F041FF02F058
:108198005DFD012306A88DF818308DF81C3002F01B
:1081A80037FFB4E74C080020C00000202808002052
:1081B8002C080020000400017FB5092301A88DF8D0
:1081C800043003F0ADF90038044B059A1A6018BF63
:1081D8000120404207B05DF804FB00BF2C080020D6
:1081E80070B504460B46134962784A700020A2789D
:1081F8000A7208701A884A729A788A72DB780B7445
:108208006368CB600C4B1B68DA6A2AB1237803F0E9
:10821800FB030A2B00D09047084E052556F8043B6F
:108228001BB15B6A0BB120469847013D15F0FF056D
:10823800F4D170BDCC00002034080020380800209C
:1082480070B5044610480123037063784370A3781F
:108258008372E368C360E3780376236943762379FE
:1082680043720A4B1B689B6A03B19847084E052561
:1082780056F8043B1BB19B690BB120469847013D5A
:1082880015F0FF05F4D170BDE0000020340800208F
:1082980038080020014B1868704700BF2C080020E0
:1082A80000B58BB0012368468DF8003002F088FDD8
:1082B80038B99DF80400003818BF01200BB05DF8EC
:1082C80004FB0020FAE7000008B501F073FE48B986
:1082D800FFF7E6FF012806D0054BD879197AFFF792
:1082E800FDFE012008BDBDE80840FFF7CBBE00BF7A
:1082F800C00000202DE9F04186B005460E4617461D
:1083080001F058FE00287FD101F06CFE044640B908
:10831800FFF7C6FF012807D03D4B197AD879FFF738
:10832800DDFE6FF0020462E0DFF8E88088F808609C
:10833800003E18BF01268DF80460374E68783379FF
:108348008DF81230694602F0D9FC00283ED08DF82D
:1083580004400394ADF810406FF0060495E803005C
:108368002E4B83E80300337988F80A30394601A890
:1083780003F0DAF92A4B059A1A60112841D801A3AB
:1083880053F820F0EB830008118400080B840008E0
:108398000B8400080B8400080B8400080B84000879
:1083A8002B8300080B8400080B8400080B8400084A
:1083B800058400080B8400080B8400081184000859
:1083C8001184000811840008FF8300082B788DF8B9
:1083D80008306B78ADF810306B6803934FF0FF34BA
:1083E800BCE7104B00221A70E31D18BF1446204644
:1083F80006B0BDE8F0816FF00404F8E76FF00504FB
:10840800F5E74FF0FF34F2E76FF00104EFE700BF44
:10841800C0000020E00000204C080020F0000020F0
:108428002C0800203008002037B501F0E5FD144D78
:10843800052455F8043B5BB11B694BB155F8043C66
:108448009B682BB1984718B155F8043C1B699847AD
:10845800013C14F0FF04ECD1FFF714FE68B9094D94
:108468002B7853B1084BADF80040D97801942246D7
:108478006846FFF73FFF00B92C7003B030BD00BF5E
:1084880038080020300800204C08002030B58BB098
:10849800054601F08FFD0446002839D1FFF700FF9B
:1084A800012838D168468DF8004002F089FC10B1E7
:1084B8004FF0FF3004E09DF80430AB4202D10020B9
:1084C8000BB030BD012DF3D0022D11D0002DF7D106
:1084D800002BF4D068468DF8045002F099FD00286E
:1084E800E6D10E4B1B681B6B002BE8D09847E6E7DC
:1084F800002BDDD168468DF8045002F089FD002874
:10850800D6D1064B1B681B6B002BD8D02846EDE74D
:108518006FF00100D4E76FF00200D1E734080020C3
:1085280010B504468AB018B94FF0FF300AB010BD34
:10853800002368468DF8003002F042FC0028F3D191
:108548009DF804302370F1E77FB500220B462049DF
:108558008DF8072001220A7042784A700446002AE2
:1085680033D102790A721A884A729A788A72DB7849
:108578000B740369CB60C378164D8DF80830037B04
:108588008DF80930836803932B68DB6A0BB102A866
:1085980098472B689B6B13B1227E02B198470E4E09
:1085A800052556F8043B1BB1DB690BB120469847FB
:1085B800013D15F0FF05F4D10DF10700FFF7B0FFFD
:1085C800637913B1054B01221A7004B070BD00BF66
:1085D800CC00002034080020380800203008002093
:1085E80010B504468AB018B94FF0FF300AB010BD74
:1085F800202368468DF8003002F0E2FB0028F3D112
:10860800024A9DF9043023701371EFE74C080020EB
:1086180000B58BB02323019068468DF8003002F036
:10862800F7FC003818BF012040420BB05DF804FB8E
:1086380070B5654C01468EB01822204606F0ECF85D
:10864800624B00221A70FBF759FF23784068012219
:1086580002FA03F1014004D15D4B084608F0D2F854
:10866800FEE75C495C481A4602F032F918B14FF04F
:10867800FF300EB070BD272304A88DF8103002F02B
:10868800C7FC564E564D002870D1012333702B6815
:10869800DB690BB100209847272304A88DF8103018
:1086A80002F08EFB059B93F84820227093F818215E
:1086B80093F81A316270A370464BD3E9020105F0B2
:1086C8009DFF05460028D2D1464E062304A88DF802
:1086D800103002F075FB059B736104A802F098FC4A
:1086E800022304A88DF81030059602F069FB0836BD
:1086F800032304A88DF81030059602F061FB0F26BD
:1087080006F040F8012304A88DF814308DF81060A5
:1087180002F07EFC10230DEB03008DF810308DF86D
:10872800145002F075FC04238DF8103004A8A378C7
:108738008DF8143002F06CFC3A238DF8103004A840
:108748006369059302F064FC02A920788DF808603B
:1087580004F0E4F8003818BF0120E0711420FFF796
:1087680057FFE07903F0A4F9284682E728238DF81B
:1087780010302B681B6943B104A802F021FB2B6859
:1087880005981B6940F2C4519847272304A88DF81F
:10879800103002F03DFC50B9012304A88DF81030C8
:1087A80002F00EFB9DF81430002B7FF46EAF337887
:1087B800002B7FF46CAF052204A88DF810200593D8
:1087C80002F026FC78E700BF4C08002030080020A3
:1087D800641D0108740800208C0800202808002067
:1087E800340800201008002037B500230D460193F7
:1087F8000446D0B900F0A8FB0190019BD3B10F4A01
:1088080042F824300E4A9A620E4A1268916B196334
:10881800916C596392690C49D9625A6128465B6820
:108828000A49F2229847002006E001A900F092FBCD
:108838000028E2D04FF0FF3003B030BD38080020E8
:10884800E580000834080020C18100081C070020CA
:10885800194B07B51860194B194A1A60194A5A601A
:10886800194A9A60194ADA60194B02681A60426814
:108878005A6082689A60C268DA60164A1A61826928
:108888005A61154BC26B5A60144A019119609A607B
:108898001946134ADA600020FFF7A6FF48B901A875
:1088A80000F056FB003818BF0120404203B05DF8C5
:1088B80004FB4FF0FF30F9E7340800208C08002053
:1088C800498200085185000869890008E981000883
:1088D80074080020D5C8000864080020B580000886
:1088E800CD80000851B118B1012804D0002070478C
:1088F800044B0B607047044B0B60F7E74FF0FF30F9
:10890800704700BF000400010100010208B503F030
:10891800EBF8002814BF6FF00100002008BD08B56F
:1089280002F0BCF9002814BF6FF00100002008BD58
:1089380010B504468AB018B94FF0FF300AB010BD20
:10894800212368468DF8003002F03AFA0028F3D166
:10895800024A9DF9043023705371EFE74C08002058
:108968002DE9F0412E4D2F4F00232B7043786B706B
:108978003B689B6A8AB004460BB128469847DFF8E3
:10898800A880052658F8043B1BB11B6A0BB120468A
:108998009847013E16F0FF06F4D12378052B2FD017
:1089A8000B2B35D0012B25D1204C062368468DF89A
:1089B800003002F005FA0199E07905F065FE10B97A
:1089C8001B4B019A5A611B48FFF70AFE1A48FFF72A
:1089D800AFFF6B788BB9A371184B5878FFF756FD2A
:1089E8003B685B6A0BB1114898476B7813B9E0791B
:1089F80005F0DAFE0AB0BDE8F081FF23A371EFE7C6
:108A08000F4B01225A74227A9A74627ADA74F1E767
:108A18006378002BEED00AB0BDE8F041FFF7CCBB7D
:108A2800E00000203408002038080020C0000020A2
:108A380010080020C4000020C50000204C080020B9
:108A4800CC00002030B58BB0FFF769FF0446F0B9C1
:108A580003F044FF831C1DD0F8B9134D2B685B69E4
:108A6800DBB1272368468DF8003002F0A9F92B689E
:108A780001985B694FF4B961984703F041FF78B9F1
:108A88002CB9094B1B68DB690BB1012098472046BC
:108A98000BB030BD6FF00704EFE74FF0FF34ECE7A1
:108AA8004FF0FF34F3E700BF34080020014B18787B
:108AB800704700BFA0080020014B5878704700BFDE
:108AC800A008002070470000044B9A7A0AB10122DE
:108AD8005A70034B5B6903B118477047A008002020
:108AE800FC00002073B5224C6378002B33D008F0CB
:108AF80073F966680546FFF7CDFB0644AE4214D20B
:108B0800A37A93B1E0228DF800208DF80130217A04
:108B1800E368019301226846FFF7ECFB08B10730D0
:108B280010D100236370A372656094F83430EBB100
:108B3800002384F834300F4B5B6BBBB102B0BDE847
:108B48007040184740F2DC510B4808F011FA0A4807
:108B580008F0D4F9E8E794F83520002AE5D094F82D
:108B6800360084F83530FFF791FCDEE702B070BDBF
:108B7800A0080020FC000020D808002037B5104DC0
:108B8800104CC8B1C1B10123627200222860E160B3
:108B980023700D480D4B00924FF0FF3108F002F999
:108BA80000250B4825822022294605F049FE6570DC
:108BB800A574A58603B030BD00232B602370EFE7B2
:108BC8009C080020A0080020D8080020D18A0008AE
:108BD800B40800202DE9F0478E4C23788CB0002B88
:108BE80056D0C2780AB9837B13B1238A0133238212
:108BF800437B002B4CD0E02A4AD10023A37287681C
:108C080097F80080B8F1220F27D8B8F1220F30D892
:108C1800DFE818F04100FB0052005A0061006E00C6
:108C280075008E009D00B400C7002F002F002F0094
:108C38002F002F002F002F002F002F002F002F00B4
:108C48002F002F002F002F002F002F002F002F00A4
:108C58002F002F00C900D000D400B8F17E0F00F01B
:108C6800CC80B8F17F0F00F0DF80B8F17D0F00F005
:108C7800AB80A57A002D00F05B81674C637A3BB925
:108C88004FF47A71204608F073F9204608F036F957
:108C98000CB0BDE8F087E36801220021A2721970C8
:108CA800A37AE1689818A0720620C854A37AE168EC
:108CB8009818A072CA54DCE7584B9B6A002BD8D08E
:108CC800012102209847D4E77B7884F836300123C5
:108CD80084F83530CDE704238DF804307B78003BE9
:108CE80018BF012301A88DF8083002F091F9C0E7F8
:108CF8007878003818BF012002F0DAFEB9E7484E4C
:108D08000FCE01AD0FC50FCE0FC596E8070085E859
:108D180007007B780A2BACD8424A12685268002AAE
:108D2800A7D00CA901EB830353F82C0C9047A0E7BC
:108D38007878431E012B9CD83A4B01381B6818BF22
:108D4800012020729B68002B93D0984791E7E26836
:108D580001230821A3721170627A057BA17AAA42C5
:108D680028BF2A46934284D285685A1CEB5CE56882
:108D780001334E1CA6726B54D3B2EDE7E3680122AF
:108D8800A27209221A70A37AE268218A581CA0727A
:108D9800D154A27A238AE1681B0A501CA0728B5412
:108DA80067E7238265E705238DF8043001A802F000
:108DB800B7FB5EE7194BDB6A98475AE7194B787897
:108DC8001B686075DB68BEE7037B072B7FF451AF38
:108DD80006238DF80430B7F80130ADF808307B79F8
:108DE8003A791B0443EA0223FA7813436422534373
:108DF8000393BB798DF81030D8E73B2201A88DF892
:108E080004208DF8083002F003F9012384F8343087
:108E18002FE700BFA0080020D8080020FC00002091
:108E28003C1401089C0800202A2301A88DF804306E
:108E380001F0C6FF94F80A90E6689DF808009DF8CE
:108E480009509DF80A709DF80BC09DF80D309DF8EB
:108E58000E209DF80F109DF80CE009F1010A84F826
:108E68000AA006F80980354E94F80A903668D4F8B6
:108E78000C8009F1010A84F80AA096F803A008F802
:108E880009A094F80A90D4F80C8009F1010A84F832
:108E98000AA096F802A008F809A094F80A90D4F855
:108EA8000C8009F1010A84F80AA096F801A008F8D4
:108EB80009A094F80A9009F1010A84F80AA096F822
:108EC8000080E66806F8098094F80A80E66808F1E8
:108ED800010984F80A9006F808C094F80AC0E66800
:108EE8000CF1010884F80A8006F80C70A77AE66885
:108EF80007F1010C84F80AC0F555A57AE6686F1CDD
:108F0800A7727055A07AE568461CA6722954A17A02
:108F1800E0684D1CA5724254A27AE168501CA07208
:108F28008B54A37AE268591CA17202F803E0A0E608
:108F3800034807F095FF6570AAE600BF9C0800206B
:108F4800D80800207047000000487047FC00002047
:108F5800002070474FF0FF3070470000044B054A6F
:108F680093F81831022B18BF062382F89034704703
:108F7800B40E00207C140020034BD3F8483313B1FF
:108F88005B6903B1184770477C140020034A1378C3
:108F980043F004031370FFF7EFBF00BF78140020FD
:108FA8001FB50A4B8DF8090093F87C208DF80A202C
:108FB80093F88C2093F848000D3202A98DF8082008
:108FC80003F0ACFCC0B205B05DF804FBB40E0020A1
:108FD80010B5074C04F5806007F042FF94F81A3486
:108FE80013B1012384F81934BDE81040FFF7C4BF5A
:108FF8007C14002010B50C4CD4F8403343F08003A7
:10900800C4F8403394F81A3413B10020FFF7E0FF96
:1090180094F8913423F0120343F0120384F8913446
:10902800BDE81040FFF79ABF7C1400202DE9F041FD
:10903800DFF8AC8098F81831022B06460D4602D0AE
:10904800284BDB6A984702F0E9FD044628B1022064
:1090580002F0DAFD002002F0DCFD98F81831012B4F
:1090680017D102F0DDFD074630B1002002F0CDFD3A
:10907800002002F0CFFD3C4602F0D4FD48B10020AC
:1090880002F0C4FD002002F0C6FDBDE8F041FFF784
:1090980065BF002CF9D1144C94F8902494F81A3434
:1090A800BAB90BB184F84164304602F065FFD8F8CC
:1090B8002C0007F09BFED4F8B4339842E5D30B4854
:1090C80007F0CEFE94F8913443F0100384F89134FD
:1090D800DBE70BB184F84154284602F04DFFF1E775
:1090E800B40E0020E42401087C1400201418002089
:1090F80073B5164C164D04F57A76EB6C95F850203E
:1091080095F9781095F84800009603F02DFC95F82D
:10911800303184F8FC3395F8480040F2012304F21A
:1091280024423146A4F8FA3303F02AFC58B194F8E3
:10913800243484F86A34074B00205B6B984794F812
:10914800FB3384F8903402B070BD00BF7C1400205B
:10915800B40E0020E4240108074A10B5137843F040
:1091680002031370FFF708FFBDE81040034B01220C
:109178000021022007F046BB78140020AD1D01082D
:10918800074A10B5137843F008031370FFF7F4FE8D
:10919800BDE81040034B01220021022007F032BB3A
:1091A80078140020BD1D01082DE9F0410F46164630
:1091B8001D46804607F010FE0B4A0C4C1378278199
:1091C80023F0110343F011031370C4E9000866810A
:1091D8002573FFF7D1FEBDE8F041054B01220021C0
:1091E800022007F00FBB00BF78140020281A0020C7
:1091F800CD1D010813B507F0EFFD0D4B6C46186047
:10920800204607F03DFD94E803000A4A0A4B83E82C
:109218000300137843F020031370FFF7ADFE074BEC
:1092280001220021022002B0BDE8104007F0EABA8E
:10923800381A002078140020B4170020DA1D01081D
:10924800F8B5334D95F81841012C06464BD0022C41
:1092580051D064B938B9D5E91B0105F1740383E825
:1092680003002046F8BD01283DD0022801D0032480
:10927800F7E7284F85F8180107F5747EBEE80F0058
:1092880007F57A7CACE80F009EE8030095F8E93012
:109298008CE8030087F8FB63E3B195F80031022BF3
:1092A80018D1D5F804316B67C7F8EC3395F87D30E1
:1092B80095F8082187F8F83395F88C3085F87820E8
:1092C80087F8F93397F81B2487F8E82340F201332D
:1092D800A7F8FA33002387F81A340F4BDB6A98474C
:1092E800FFF706FFBDE702F0A4FC04460028B8D14A
:1092F80085F81861B5E70028B9D1064B85F818013B
:10930800062283F89024044BDB6A98473446A8E782
:10931800B40E00207C140020E42401082DE9F0415B
:1093280092B0064602F07AFC002840F05981AD4D13
:1093380095F81831012B09D02B6BAB4C93B194F8ED
:109348000431BBB1042B6FD0032003E002F068FCAA
:1093580018B10F2012B0BDE8F08102F063FC0028BC
:10936800EAD0F6E7B5F82031D4F81C24013B534382
:109378002B63E4E79D4803F008FA002840F02C81AD
:1093880094F80C3123802B6B0C930DF1180895F889
:1093980039308DF83830404695F81C318DF83A3020
:1093A80007F094FCD5F82831009302AF98E806003E
:1093B800D5F82431384607F020FC97E803000FABB6
:1093C80083E80300EB6A0D9300238DF8443023886B
:1093D800ADF8463095F8303101228DF839201BB9A7
:1093E8008DF844208DF83930814B0093814B95F8E6
:1093F8004800A3F179020CA903F005FBC0B10B28C2
:10940800A8D1D4F8941499B1002EA3D0D4F840333D
:10941800794843F02003C4F8403307F0A9FD7648A3
:1094280007F06CFD002095E7704803F0E2F9A4E727
:1094380095F8487095F9693095F9392095F87D10B7
:109448006E4E384603F0ECFA009641B2EB6C95F894
:1094580050203846183603F087FA0096EB6C95F8DA
:10946800502095F9701095F8480003F07DFAD4F86B
:10947800C413AB6DD4F8DC230B44C4F8B033EB6DE4
:109488001344C4F8B43394F80431042B07D02B6E7A
:109498000B44C4F8B0336B6E1344C4F8B4330023E0
:1094A800089395F8303183B108A802F095FC00289C
:1094B8004ED195F9390094F837629DF82070FFF77E
:1094C8006FFD3E4480B2B04240D300238DF8133084
:1094D80095F839308DF8213095F838308DF82230EC
:1094E800D5F880300993D5F884300A932388ADF8ED
:1094F8002C3095F8303194F81B648DF82E3095F89F
:1095080048003F4B8DF820600DF1130208A903F0C5
:109518003FFA012384F8413495F8393084F842340D
:109528009DF8133084F84334D4F81C34C4F85064DC
:10953800C4F84834C4F8583402F076FB50B1D4F873
:109548001C0402F083FB28B1102003E7082001E780
:109558001320FFE695F81831012B01D102F078FBB2
:1095680002F065FB0023059394F8043195F939500E
:1095780094F81B649BB1042B7FF4E6AE05A802F0B7
:1095880067FE58BB94F8183413B1059B013B05934B
:10959800164B05983246E9B202F0BCFE02E01348C9
:1095A80002F090FEC0B9D4F8403394F80C11218031
:1095B80043F00203C4F8403394F8183411480133D7
:1095C800DBB284F8183484F845340F4B00259B6AC5
:1095D800C4F89854984725E71120BBE61220B9E64D
:1095E8000E20B7E6B40E00207C140020841500205D
:1095F800E40E002010190020E41700203418002081
:10960800981800207E140020E4240108F0B5504C7E
:10961800504EB4F8DC202287D4E92D0194F8B1200B
:1096280084F8692004F16C0282E80300D4E92F0170
:1096380004F1740282E80300B4F8C420A4F87C2082
:1096480091B0D4F8CC20D4F8C810C4F884200025F0
:10965800D4F8D020C4F888200123A4F82031C4F815
:10966800801084F83051A56284F81B5184F83A5070
:1096780084F81D5184F81E51C4F83451C6F8985422
:10968800A6F8185486F81A54A4F838518DF81830EA
:1096980004F50973039304F50A7394F84800A4F8D1
:1096A8004651049303A92C4B84F84551C4E94F55FE
:1096B800059303F041F9E36EC6F8D43394F87D308E
:1096C80086F8E03394F88C3086F8E1334FF48073F1
:1096D800A6F8E23386F8D05394F8303186F8E433AC
:1096E80006F574770FCF06F57A740FC497E8030070
:1096F80040F2012384E80300A6F8FA33D6F8483389
:1097080086F81B54CDE901551BB15A685B69019273
:109718000293124B0793A3F148020892A3F1140293
:1097280009920F4A0B9229330A93A2F19C030C93D6
:10973800A2F198030D93131D0E9301A902F14C0396
:1097480007A802F599620F9302F05DFA11B0F0BD17
:10975800B40E00207C14002098190020E418002082
:10976800980F0020F8B50D4F0D4C0E4E0D4607F022
:1097780077FB3B6B984796F8480004F22442294649
:1097880003F0FEF848B194F8243484F86A34706D14
:109798007B6B9847EB7C84F89034F8BDE42401088F
:1097A8007C140020B40E00200F4890F81B3480F879
:1097B800B8330E4B93F8692080F8BB2393F87D20CB
:1097C80080F8C82393F88C2080F8C92393F83031A7
:1097D80080F8CC330022A0F8CA2300F56E7100F59A
:1097E8006070FFF7BFBF00BF7C140020B40E0020DC
:1097F800114890F89034EBB190F81B3480F8D033CE
:109808000E4BDA6EC0F8D42393F87D2080F8E0235D
:1098180093F88C2080F8E12393F8303180F8E43312
:109828004FF48072A0F8E22300F5747100F56670B9
:10983800FFF798BF704700BF7C140020B40E0020CB
:1098480070B5344C2421204604F0FCFF636A98422A
:1098580018BF60624FF01C012F4814BF0125002576
:1098680004F0F0FF636C984218BF60644FF4807195
:109878002A4818BF45F0020504F0E4FFD4F848313F
:10988800984218BFC4F848014FF0D401244818BFC3
:1098980045F0040504F0D6FFD4F82032984218BFEA
:1098A800C4F820024FF000011E4818BF45F0080513
:1098B80004F0C8FFD4F82432984218BFC4F8240230
:1098C8004FF46071184818BF45F0100504F0BAFF4E
:1098D800D4F8A835984218BFC4F8A8054FF0140169
:1098E800124818BF45F0200504F0ACFFD4F8C03585
:1098F80098420F4B18BFC4F8C005D3F8483318BFB7
:1099080045F040052BB11B691BB12846BDE87040E6
:10991800184770BDB40E0020DC0E0020FC0E00209D
:1099280000100020D8100020DC1000206014002057
:109938007C1400202DE9F04F91B04FF00008012B66
:1099480005460F4602928DF81580ADF8188003D8A9
:10995800C84EC146B94502D311B0BDE8F08F15F81D
:10996800090002F077FA4844B842F5DC15F80930E6
:1099780009F10104023BE4B2112BEDD801A252F81F
:1099880023F000BFD5990008079A0008079B000834
:10999800319B0008B99B0008E19B0008539C000814
:1099A800859C0008019D00086199000861990008DC
:1099B8005F9D000861990008619900081D9E0008D4
:1099C800459E0008899E0008C79E0008052002F0F1
:1099D800EDFA90B10521002002F0ACFA2A5DA64B01
:1099E80009F1030409F102095FFA89F983F85C2493
:1099F80015F8092083F85D24E4B2A146AAE70023FC
:109A08008DF816308DF817308DF81C308DF8203011
:109A1800B8F1000F6CD14FF0050896F87C208DF84E
:109A28003920631E96F839208DF83B202B4496F890
:109A380038200D938DF83C2096F81A3196F8682056
:109A48008DF83D20D6F82C218DF83A300C9273B35E
:109A58007B1C1B1BDBB28DF8383008AB019307ABBE
:109A6800009396F848000DF117030DF116020CA9A2
:109A780002F09AFF8DF8150000F00700072813D1AF
:109A880096F939209DF9163086F839309A429DF8B2
:109A9800173086F83830B8BF01229DF81C30B8BF9F
:109AA80086F81D2186F868304FF0000909E0052383
:109AB800D1E701220DF11501032002F0DBF809F1CD
:109AC80001095FFA89F29DF82030B3FBF8F1914261
:109AD800EFD82344DCB2631EDBB29F420DD9EA5CA7
:109AE800032A9AD0A74288BF1C464FF0010884E792
:109AF80009F105095FFA89F4F7E71C46F5E72B5DDC
:109B0800012203F00F0309F1020986F81B3102FA5A
:109B180003F35FFA89F9A6F82031002206A9042088
:109B280002F0A8F84C4668E707238DF815302B5D3E
:109B380096F84800C3F3021203F00F038DF8303093
:109B480009F10303DBB28DF83120EA5C09F1040363
:109B5800DBB209F10504EB5C09F102095FFA89F946
:109B68001B0443EA022315F80920134364225343D4
:109B78000CA90D9302F027FF00F00703072BE4B2AE
:109B88008DF815000CD19DF8303086F8703086F8C5
:109B980078300D9BF36673679DF8313086F869302D
:109BA8008DF81800012206A9052002F063F824E7C1
:109BB800314BD3F848336BB11B685BB19847029BB4
:109BC8008DF8180003F03F038DF81930022206A91A
:109BD8000620EAE7FF20F2E703238DF815302B5D16
:109BE8008DF824300CAB089309F10303DBB209F1BB
:109BF8000604EA5C96F8480009F10403DBB208A9F8
:109C0800EB5C1B0443EA022309F10202D2B209F118
:109C18000509AA5C1343642253435FFA89F90C933C
:109C280000230D9315F809308DF8383002F0D1FE75
:109C3800C3B20028E4B28DF81530FFF6DEAE8DF819
:109C48001830012206A90720AFE72B5D03F00F03A8
:109C5800012B4FF47A7238BF0123534309F10209EB
:109C6800B36513445FFA89F9F365002206A9082051
:109C780056E700BFB40E00207C1400202B5D96F838
:109C88004800C3F340128DF81D2007A9C3F3001242
:109C980003F00F038DF81C208DF81E3002F09FFE94
:109CA80009F1020901305FFA89F93FF43BAFBDF8C9
:109CB8001C30914AA6F87C309DF81E309DF81C4057
:109CC800D05CF7F7A3FE0223C6F880000CA996F82B
:109CD80048008DF830308DF8324002F01FFE96F9BA
:109CE8003930089040B29842B8BF184686F8390013
:109CF800002206A9092013E703238DF815302B5DF0
:109D08008DF8303009F10303DBB209F10504EA5C90
:109D180096F8480009F10403DBB209F10209EB5C8B
:109D28005FFA89F91B0443EA022315F80920134353
:109D3800642253430CA90D9302F057FEC3B20028C6
:109D4800E4B28DF81530FFF658AE8DF818300122C0
:109D580006A90A2029E7092002F028F9DFF89CA1C2
:109D6800002854D00921002002F0E4F80023ADF8BF
:109D7800263009F10203DBB24FF47A71EA5C09F18B
:109D88000303DBB20DF1300BEB5C1B0443EA022347
:109D98002A5D134309F10402D2B209F1060409F15C
:109DA8000509AA5C5FFA89F943EA026315F80920F4
:109DB80003934A4312125846ADF8242006F060FF78
:109DC800039B03F1965303F5A91303F5EC5308938A
:109DD800DAF83C3300930DF1200999E80600DAF827
:109DE80038330AA806F009FF0B9B00939BE806008E
:109DF8000A9B484606F0E6FE99E8030006F018FFBD
:109E080001F021FF0123E4B28AF83834F5E58AF835
:109E18003804F2E50C2002F0C9F800283FF4EDAD53
:109E28000C21002002F086F8344B93F89034043B60
:109E3800012B7FF6E2AD01F002FFDEE509F1020336
:109E4800DBB22A5DE95C09F10303DBB209F1050421
:109E5800EB5C09F104095FFA89F91B0415F809009C
:109E680043EA012313436421594300F00F0001F032
:109E7800E7FEE4B28DF81800012206A9112094E645
:109E88000D2002F093F800283FF4B7AD0D21002013
:109E980002F050F809F10203DBB2194AE85C2B5DC5
:109EA800126809F1040409F103095FFA89F943EA20
:109EB800002015F80910E4B201F0C4FE9DE52A5D02
:109EC80009F1020309F1040409F10309DBB25FFA9D
:109ED80089F9E95C15F809301B0443EA01231343A7
:109EE8006420584301F0B0FEE4B28DF81800012256
:109EF80006A9132059E600BFE71D01087C140020BD
:109F0800281A00200E4B93F89124920703D593F852
:109F18008F24012A08D90B4991F81A2122B18A6A9B
:109F2800501C18BF01328A620022A3F8182483F853
:109F38001A24D3F8402322F00202C3F840237047C2
:109F48007C140020B40E002070B5184C184D04F590
:109F58005A7006F085FFD4F84033D4F89804D5F841
:109F6800906023F02003C4F8403338B106F03EFF78
:109F7800864203D2002385F83A3070BD0120FFF7EE
:109F8800CDF90028F9D00B28F7D095F8393084F8A6
:109F98004234092094F8183484F8453484F841048C
:109FA80001F0EAFFBDE87040FFF7ACBF7C14002069
:109FB800B40E0020094BD3F84023012A0AD00849DF
:109FC8000978C90708D43AB993F89204013818BF38
:109FD8000120704700207047012070477C14002042
:109FE80078140020034BD3F84003431E58425841CD
:109FF800704700BF7C1400202DE9F04FA9B0EFF3A3
:10A00800108272B6DFF8F4820021D8F80030C8F860
:10A01800001082F31088BA4C002B00F0E480DAB20A
:10A028009B06039264D5B74D95F81831022B02D0E0
:10A03800B54BDB6A9847EFF3108972B6B34F06F059
:10A04800CBFE3E68D4F8B013361A3144B04806F057
:10A058008FFFAF4806F052FFD4F8B413AD4831442F
:10A0680006F086FFAB4806F049FF89F3108894F89C
:10A078001A34002B00F06D81152312A995F84800B9
:10A088008DF8483002F04AFCD4F8B4130F9001441C
:10A09800A14806F06DFFA04806F030FF3B6894F831
:10A0A8001B24EB620DAF38468DF870201D9306F027
:10A0B8000DFED5F82831009306AE97E80600D5F8CE
:10A0C8002431304606F099FD96E803001FAB83E87B
:10A0D8000300D4F81C341E9395F8303195F84800E5
:10A0E800003B18BF01231CA98DF8713002F01FFC3A
:10A0F800039BDF064BD5834DDFF820A2D5F8E4207B
:10A10800BAF90A30059298F800200493002363F303
:10A1180000020A9388F8002084F84434049AA4F8CA
:10A12800223484F82534C4F82834A4F82C3484F86C
:10A138002E34C4F8303484F82034C4F8343484F825
:10A148003834C4F83C34704B9AF90C90A4F88C2439
:10A1580094F89024DB6A84F88E9484F88F24DAF8D3
:10A168000470BAF80860984794F88F3413B96948AE
:10A1780006F076FE3146384601F04EFD834600284B
:10A1880000F0EA80049BA4F87E3484F88094039B52
:10A1980019071AD55B4B93F81831022B02D05A4B8A
:10A1A800DB6A98470220FEF7D9FE84F8410401F0E3
:10A1B800E3FE94F81A3413B1012384F8193494F89F
:10A1C800913443F0100384F89134039B5A0703D564
:10A1D80006210520FEF72AFF039B9B0703D50421D0
:10A1E8000320FEF723FF01F035FD94F89124D706EC
:10A1F8005FD5002384F89234D4F840331E0644BF58
:10A2080023F08203C4F8403312F0050F00F0FC82FB
:10A218000B2001F0CBFE002800F0F68294F8913470
:10A22800DD0700F1F182580740F10883D4F8403384
:10A2380023F00203C4F84033D4F8402382BB94F8D7
:10A24800915415F001011EBF2B4662F3000384F8F8
:10A25800913494F891345E0744BF6FF3820384F815
:10A268009134012384F8923421B1D4F844332C4832
:10A278001B6898476D070BD52A4801F0A3FE01F02B
:10A28800D1FE28B194F8913443F0040384F8913452
:10A2980001F0CEFC94F891346FF3041384F89134F0
:10A2A800012384F8923494F8913443F0200384F81D
:10A2B800913494F8913418070AD56FF3C3031A49F7
:10A2C80084F89134D4F84433A1F12400DB6898472A
:10A2D80094F8913499070AD56FF34103124984F829
:10A2E8009134D4F84433A1F16C005B68984794F832
:10A2F8009034022B1AD1FEF7FBFE17E078140020E9
:10A308007C140020B40E0020E4240108381A002030
:10A31800FC170020141800207C180020281A0020A0
:10A32800BC180020D01800200819002094F8913497
:10A338009A0640F1C6826FF3451384F89134D4F835
:10A348004033002B40F0BD8229B0BDE8F04FFFF745
:10A3580077BA84F84134A1E695F81821012A0CD17E
:10A3680001F05EFC804668B1584601F04EFC584644
:10A3780001F050FC042384F88F347EB9012384F85B
:10A38800213450E101F04EFC0028F6D0404601F09F
:10A398003DFC404601F03FFC0523ECE73B78049385
:10A3A8005B09013B062B00F21882DFE813F0070077
:10A3B800160295001602920016020702102EDDD929
:10A3C80095F830311297F6B28DF84C60002BD5D144
:10A3D8001CA804F04BF912AA1CA9FF2002F0AEF841
:10A3E8009DF85830C3F3030307468DF82C3095F8D1
:10A3F800480095F87D308DF82D3007220BA902F022
:10A40800A0FA002F5DD100285BD09DF853309DF84D
:10A4180052201599C5F8E4101B0443EA02239DF85D
:10A42800512002201343C5F8E03004F02DF99DF8BF
:10A43800583095F8480085F82E71C3F30212C3F31B
:10A44800030385F8703085F878309DF8593085F821
:10A458006920012B38BF01234FF47A725343AB654F
:10A468001344EB650DF15A034FF001081093113EA8
:10A4780094F81B348DF83C300FA985F868808DF866
:10A48800446002F066FA0223404685F8303101F054
:10A498008DFD18B14146384601F04CFD94F88F34D3
:10A4A800012B00F2A88194F81A34002B40F09B810C
:10A4B80094F8913443F0100384F89134FEF74EFD7C
:10A4C80065E6012001F072FD0028E7D00121072090
:10A4D800E2E7012384F8203495F87D308DF82E309A
:10A4E80094F824348DF82D3095F88C3095F8480080
:10A4F8000D330BA98DF82C3002F010FAA6F10D03DC
:10A508001BB2099023EAE37300B283423FF736AFE8
:10A518000B2E7FF633AFBB4B25931CA8FF231C974C
:10A528008DF874608DF8983002F0D4F8074600284A
:10A538007FF424AF95F81831012B13D101F070FB8B
:10A54800002873D0384601F060FB384601F062FB02
:10A5580004239DF87C101E9884F88F34C1F30011F1
:10A5680001F077FB9DF87C301E99C4F8341413F081
:10A578000F0203D09DF89000002863D19DF8980041
:10A58800002862D0002A7FF4F9AE9DF89020002AB6
:10A598000CBF4FF002084FF0030800220A92D5F8CA
:10A5A800EC20914254D195F8E910002950D0D5F803
:10A5B8000C1195F8EAB009680A9195F81811022962
:10A5C80002D1032184F88F14B8F1030F7FF4D6AEBB
:10A5D80013F0600F7FF4D2AE0592012795F82E3163
:10A5E800BBF1000F37D0BBF1010F38D1012B34D1AB
:10A5F8006FF0090646FA08F606F00106C6F10206EB
:10A60800F6B2BDF87E100AAA304601F02DFE40B31E
:10A6180007280CBF0823012384F821340A9BC4F8B7
:10A628003034C4F86C34FEF7E5FCB0E501F0FAFA12
:10A63800002897D0384601F0E9FA384601F0EBFADD
:10A64800052386E74FF00008A7E74FF00108A4E7C5
:10A658004FF0010BC2E70426D3E70326D1E7012315
:10A66800DAE71CAB009305990A9B3246584601F07D
:10A67800B7FE20B102280CBF0A230B237FE60A9BF2
:10A68800C4F83034C4F86C349DF87C3084F8210464
:10A69800C3F3401384F82E3484F8443494F88F3488
:10A6A80084F82274012B9EBF0122A86285F81E211E
:10A6B800012FC4F8280484F82C0484F8410438D104
:10A6C800022284F8202495F83A20002A4AD19DF8DD
:10A6D8007C20D60646D4012B94F840149DF87C20A3
:10A6E80005D8012901D1900601D501F05FFBB8F129
:10A6F800020F94F88F3443D0B8F1030F0AD09DF8B5
:10A708007C10B8F1010F4A4601F00F0120A83BD098
:10A71800FFF710F99DF8903084F82334259BC4F88E
:10A7280028349DF8983084F82C34012384F82D348B
:10A7380030E0049A02F0E002A02A1BD195F82E110D
:10A74800012285F83A2009B927996963012B84F811
:10A75800202407D9D5F89020C4F83C24DAF8002042
:10A76800C4F8982495F81821002AB4D1012284F855
:10A778002524B0E7002285F83A2084F82024A6E7AB
:10A788009DF8981025984A46FFF7D4F89DF8903020
:10A7980084F823349DF89020E02A08D195F81F31D9
:10A7A8002BB984F82324C4F82834A4F82C3494F85A
:10A7B800913443F0020384F891346FE6114D013E61
:10A7C800B2B2791C284604F027F80323A4F82034F1
:10A7D800C4F8285484F82C64E9E7012384F8213468
:10A7E800FEF708FC5AE694F84434002B3FF460AEB8
:10A7F8000020FEF7EDFB94F88F34022B3FF45EAE99
:10A8080056E600BFB416002094F89134590715D5C0
:10A81800012001F0CBFB60B1012001F09DFB08B9DC
:10A8280084F81804D4F8403323F00203C4F8403302
:10A8380004E0062001F0BAFB0028F3D194F8913423
:10A84800DA077FF5F9AC94F840240AB1032A18D145
:10A858001D4A94F8181492F86820914205D29B0773
:10A8680023D594F88F34012B1FD8184806F0F8FA2E
:10A87800D4F8403323F02003C4F84033FFF742FBF9
:10A88800DAE4012A11D194F81924002A3FF4D4AC4F
:10A898000D4A94F8181492F868209142E5D29F075F
:10A8A80003D594F84434002BDFD194F89134002078
:10A8B8006FF3041384F8913484F81904FFF744FB08
:10A8C800BAE429B0BDE8F08FB40E0020E4170020E8
:10A8D8002DE9F04F89468DB090460746002800F0D4
:10A8E8008F81002900F08C810368002B00F088819B
:10A8F8004368002B00F084818368002B00F080817E
:10A90800C368002B00F07C81104602F003F8002891
:10A9180000F07881BD4CBE4D384601F0C1FA40F2D6
:10A92800C4520021204603F08BFF40F21C52002144
:10A93800284603F085FFB74BC4F82C3104F509739A
:10A94800089304F50A7300264046099308A9B24BF8
:10A9580084F848800A9384F8186184F88C608DF82C
:10A968002C6001F0E9FF0F2306A994F848008DF840
:10A97800183001F0D3FF801B18BF01204FF00A0BDD
:10A9880084F81C0106A994F848008DF818B001F065
:10A99800C5FF4FF0060A84F8DC0006A994F84800C1
:10A9A8008DF818A001F0BAFF102384F8DD0006A97D
:10A9B80094F848008DF8183001F0B0FF1123C4F85E
:10A9C8009C0006A994F848008DF8183001F0A6FFFD
:10A9D8001223C4F8A00006A994F848008DF818308E
:10A9E80001F09CFF1323C4F8A40006A994F84800BA
:10A9F8008DF8183001F092FF1423C4F8A80006A9B6
:10AA080094F848008DF8183001F088FF1623C4F830
:10AA1800AC0006A994F848008DF8183001F07EFFC4
:10AA2800172384F8B10006A994F848008DF8183067
:10AA380001F074FF18230DEB0301C4F8B400C4F847
:10AA4800BC0094F848008DF8183001F067FFC0B2D8
:10AA58001D2384F8B80084F8C00006A994F84800BB
:10AA68008DF8183001F05AFF1E2384F8C40006A997
:10AA780094F848008DF8183001F050FF1F2384F82F
:10AA8800C50006A994F848008DF8183001F046FF73
:10AA98002023C4F8C80006A994F848008DF8183097
:10AAA80001F03CFF0B23C4F8CC0006A994F8480039
:10AAB8008DF8183001F032FF0C2306A9A4F8D00055
:10AAC80094F848008DF8183001F028FFD4F89C302D
:10AAD8006365D4F8A030A365D4F8A430E365D4F84E
:10AAE800A83023664FF00108D4F8AC300590A4F8DC
:10AAF800D200636684F8B080C4F894B084F898A053
:10AB0800C4F84CB084F850A084F8688084F81F8199
:10AB1800C5F84893FEF77AFD404B009632464FF051
:10AB2800FF3105F55A70C5F84473C4E90B6684F81B
:10AB3800198185F89164C5F8408306F033F9384BDC
:10AB4800009632464FF0FF3105F5607006F02AF99D
:10AB5800344B009632464FF0FF3105F5667006F02B
:10AB680021F902AF304B009632464FF0FF3105F520
:10AB7800806006F017F9384606F0A8F897E8030051
:10AB880004F5927383E80300284B294F1E60294B74
:10AB9800C5F84C33284BC5F85433284BC5F85C33FB
:10ABA800274BC5F85033274BC5F8583305F5537074
:10ABB8003B68984704F5A67003F084FB20B1112682
:10ABC80030460DB0BDE8F08F204601F01DFB00288F
:10ABD800F5D101F041F8B8B91B4801F067FB06460A
:10ABE8000028ECD17B69984703F0F4FDBB6D94F81D
:10ABF80019019847FB6A9847012385F89234DFE7E3
:10AC08000326DDE70926DBE71326D9E7B40E002083
:10AC18007C1400200004000198190020519F0008AE
:10AC2800B1970008F9970008D98F00087814002018
:10AC3800E4240108FD910008B1910008958F0008EF
:10AC480089910008619100089C0F002008B5034B0A
:10AC58000020C3F84003FEF781F908BD7C140020EA
:10AC680010B5FFF7A7F90A4C60B90A4B93F81831E9
:10AC7800022B02D1084BDB6A98470123C4F8403302
:10AC8800002010BDD4F84003013818BF0120F8E7B0
:10AC98007C140020B40E0020E424010838B5134CBD
:10ACA80004F55A7006F0DCF804F5607006F0D8F880
:10ACB80004F5667006F0D4F804F5806006F0D0F864
:10ACC80000F0B5FF0A4B0025DB6A9847C4F84053EB
:10ACD800FEF7B6FD0749084840F2C45203F09CFD50
:10ACE8000123C4F84033284638BD00BF7C14002037
:10ACF800E4240108B40E0020F008002070B52E4BA3
:10AD08008AB0054693F8DD008DF8090093F8DC0059
:10AD18008DF80A0029489A6A90F8180403920026C8
:10AD28008DF80B0004960C46002940D00692D3F803
:10AD3800882007921A8F93F81A118DF8151052BAB5
:10AD4800ADF8202093F87C2093F848308DF8243013
:10AD580003AB8DF822008DF8232000930DF10A0231
:10AD68000DF10B030DF1090105A88DF8146000F031
:10AD7800DDFE9DF90900FEF713F9607004A801F0E3
:10AD88002BF8B0B9049A0F2A0DD863789A420AD8DA
:10AD98001544AB42A3EB02012CBF00200120217017
:10ADA800C0000AB070BD002323700820F9E7032013
:10ADB800F7E71320F5E700BFB40E00207C1400204D
:10ADC8001FB50446002800F012810078412800F2DF
:10ADD8000881DFE810F0420048004D00520056009C
:10ADE8005A005F0006010601060106010601060178
:10ADF8000601060166006A006E0079008000830083
:10AE080086008B0089008D009100940097009A00BD
:10AE18009D00A000AF00B300BB00B700BF00C20098
:10AE2800C600CF00CB00CD000601D3000601060105
:10AE380006010601060106010601060106010601D2
:10AE480006010601060106010601DB00DF00E3003A
:10AE5800E800EC00F000F400FD00674B93F81831AF
:10AE6800237104B010BD644B93F83031237102E0B4
:10AE7800606803F0B5FB0020F3E7606803F0F6FBB9
:10AE8800F9E75D4B93F81A31F0E75B4BD3F8E03004
:10AE98006360F0E7584B211D93F8300103F0FEFB87
:10AEA800E9E7554B93F81931E0E7534B93F88C30A9
:10AEB800DCE71C238DF808304F4B02A993F84800B3
:10AEC80001F02CFD6060D6E74C4B043493E8030096
:10AED80084E80300CFE74A4B0434F7E7494B0434CE
:10AEE800F4E7494B0434F1E71A23E3E71923E1E7D0
:10AEF800414B93F86830B9E73F4B5B6DC8E73E4B71
:10AF08009B6DC5E73C4BDB6DC2E73B4B1B6EBFE758
:10AF1800394B5B6EBCE702238DF80830364B02A92B
:10AF280093F87C2093F848008DF80A2001F0F6FC8D
:10AF38002071A0E7304B93F8DD3097E72E4B93F85C
:10AF4800393093E72C4B93F8DC308FE72A4B93F892
:10AF580038308BE7284BDB6C9AE7274B93F8503057
:10AF680084E7254BD3F88430636084E7224B8FE76E
:10AF7800264B8DE7204BD3F8CC30F5E71E4BD3F8A2
:10AF88002C31636001F058FDA06074E71A4BD3F8C8
:10AF980090307DE7184B93F81F3167E7164BB3F8ED
:10AFA8008830A38067E7144BB3F88A30F9E7124B6F
:10AFB800B3F8D030F5E7104BB3F8D230F1E70E4BC9
:10AFC80093F848200AB1062A13D1B3F8A035E8E768
:10AFD800094B93F848200AB1062A0AD1D3F8A435B8
:10AFE80056E7204604B0BDE8104000F024BE032018
:10AFF80037E7182035E700BFB40E0020200F0020E7
:10B00800680F0020280F0020700F0020F008002093
:10B018007FB5044610B9032004B070BDA44DD5F81F
:10B0280040339A0700F171820278412A00F26A825D
:10B03800DFE812F04200480056005C00600065003E
:10B048006A007700820088008E0094009A00A000B1
:10B05800A600AC00B6006802BB00DD00F0001701D6
:10B0680039012A0144014D015101550159015D0180
:10B078006802610173019B018901AD01B301BA0145
:10B08800BF01C40168022A026802680268026802F5
:10B098006802680268026802680268026802680258
:10B0A800680268026802680236023B0240024502F2
:10B0B8004A024F0254025E020079FEF7C1F80028E6
:10B0C800AAD105E00379022BA5D07A4A82F830315B
:10B0D80095F8913443F0200385F8913400209BE7DC
:10B0E800406803F06FFA0028F2D094E7406803F054
:10B0F800ADFAF8E76F4B027983F81A21E8E76D4B50
:10B108004268C3F8E020E3E76A4E416896F83001E8
:10B1180003F0BAFA00287FF47EAF6368C6F8E4301B
:10B12800D6E7416800293FF476AF002001F0EAF93C
:10B138000028CDD011206FE7416800293FF46BAF9C
:10B148000120F3E7416800293FF465AF0820EDE7E7
:10B15800416800293FF45FAF0920E7E7416800290B
:10B168003FF459AF0C20E1E7416800293FF453AFA1
:10B178000D20DBE7416800293FF44DAF0E20D5E7ED
:10B18800416800293FF447AF0F20CFE74A4C494BAD
:10B19800007983F81901A36D9847E36A984797E700
:10B1A800444B027983F88C2092E7424E037A8DF85B
:10B1B800043096F8480096F87D308DF8053007225F
:10B1C80001A901F0BEFB00283FF425AF636896F89B
:10B1D80048000193002201A901F0B3FB00283FF4C5
:10B1E8001AAF6C36D4E9010186E8030070E7314EE6
:10B1F800037A8DF8043096F8480096F87D308DF87B
:10B208000530072201A901F09CFB00283FF403AF99
:10B21800B436E7E7274E037A8DF8043096F84800ED
:10B2280096F87D308DF80530072201A901F089FBD9
:10B2380000283FF4F0AED4E9010106F1740383E875
:10B24800030096F81831022B7FF442AF96F830319C
:10B25800002B3FF43DAF184BDB6A9847FDF748FFDA
:10B2680036E7144E037A8DF8043096F8480096F8BD
:10B278007D308DF80530072201A901F062FB002816
:10B288003FF4C9AEBC36ADE74368029301238DF89D
:10B298000C30084B02A993F8480001F05FFB002826
:10B2A8007FF416AFB7E6436802930023EFE700BFC9
:10B2B8007C140020B40E0020E424010803795A1EEF
:10B2C8000E2A3FF6A8AE934A82F8683000E7914B01
:10B2D80042685A65FCE68F4B42689A65F8E68D4BE2
:10B2E8004268DA65F4E68B4B42681A66F0E6894BE9
:10B2F80042685A66ECE6874C037994F848008DF862
:10B308000430062201A901F01CFB00283FF483AE9B
:10B318009DF8043084F8DD30DAE67E4C03798DF848
:10B32800043094F8480094F87C308DF806300522F3
:10B3380001A901F006FB00283FF46DAE9DF804302A
:10B3480084F83930C4E6734C037994F848008DF8D2
:10B3580004300A2201A901F0F4FA00283FF45BAE98
:10B368009DF8043084F8DC30B2E66A4C037994F82E
:10B3780048008DF80430092201A901F0E2FA0028FA
:10B388003FF449AE9DF8043084F83830A0E6614BAC
:10B398004268C3F89420DA649AE65E4B027983F82F
:10B3A800982083F8502093E65A4B4268C3F88420CB
:10B3B8008EE6584B4268C3F8CC2089E6012B40F052
:10B3C800A480554C2421204603F03CFA636A984235
:10B3D80001D0172020E61C2104F1280003F032FADE
:10B3E800636C9842F5D14FF4807104F1480003F082
:10B3F80029FAD4F848319842EBD1D42104F5A67043
:10B4080003F020FAD4F820329842E2D1002104F562
:10B41800097003F017FAD4F824329842D9D14FF4BE
:10B42800607104F50A7003F00DFAD4F8A835984253
:10B43800CFD1142104F2AC5003F004FAD4F8C0358B
:10B448009842C6D1334E2146304640F2C45203F0EA
:10B45800E3F9204640F2C452002103F0F1F995F8CF
:10B468001B3485F8E833736FC5F8EC3396F87D30F4
:10B4780085F8F83340F20123A5F8FA33274B96F8FC
:10B4880019019B6D984723E68379012B3FF6C3ADDD
:10B49800204B42684068C3F82C2100F0D1FE47E6F3
:10B4A8001C4B4268C3F8902012E61A4B027983F8C5
:10B4B8001F210DE6174B8288A3F8882008E6154B54
:10B4C8008288A3F88A2003E6124B8288A3F8D0204A
:10B4D800FEE5104B8288A3F8D220F9E50D4B93F8CE
:10B4E80048200AB1062A12D1A288A3F8A025EFE5C0
:10B4F800084B93F848200AB1062A08D16268C3F8B5
:10B50800A425E5E500F099FBD9E5012084E518209C
:10B5180082E500BFB40E0020F0080020E4240108F2
:10B528002DE9F04387B00023ADF800300646002827
:10B5380000F0ED800361FEF73DFD20B101242046B7
:10B5480007B0BDE8F08300F073FD0028F6D100F0E5
:10B5580069FD014618B96F48142203F071F96E4D60
:10B5680095F89134012243F0040385F8552485F8B1
:10B57800913433788DF804300021013B8DF8052093
:10B58800ADF806100C2B00F2BA80DFE803F007B81C
:10B59800B8B87881B8B88FB8AC99A800D5F8407316
:10B5A80017F02007CAD196F80480B8F1020F45D1E8
:10B5B800DFF868815A4CFEF729F896F9051098F8D3
:10B5C80048003A4601F017FA88F83900B37988F844
:10B5D8003830384607238DF80530FDF731FEFF2354
:10B5E80004F58670A5F80C31C5F8084185F8047192
:10B5F80003F03CF804F58A7002F0F2FF3846FDF7D4
:10B608008DFE044640B196F9051098F848000122CD
:10B6180001F0F1F988F83900D5F894343361002C39
:10B6280071D000F0FFFC002889D195F8913485F895
:10B638001A0460F3820385F8913480E7B8F1010FAA
:10B648004FF00204E8D1DFF8D4908DF8144099F84F
:10B65800480089F81D7102A901F06EF9337989F85B
:10B6680030318DF805708DF80680FDF785FC95F86A
:10B67800913443F0100385F891340024CCE700227C
:10B688006946022000F0F6FA0028F6D01324C3E732
:10B69800244BB288DB6B96F90C10B0689847D5F844
:10B6A800403343F00203C5F84033E6E702A90D2012
:10B6B80000F060FB0028E0D0002269460D20E1E799
:10B6C800164B93F81831D3B9347904F0070000F019
:10B6D800ADFA8DF80040012269461020D2E7002219
:10B6E80069461220CEE78DF8072000F090FA04464C
:10B6F80038B900F089FA204600F08BFA8CE702246A
:10B708008AE7012488E701A800F0DEFB17E7032495
:10B7180015E700BFD01800207C140020B40E0020CC
:10B728007E140020E42401082DE9F04F99B08046EA
:10B73800059118B9032019B0BDE8F08F0023036103
:10B74800FEF738FC0646002840F0AB8045460FCD92
:10B758000EAC0FC45A4C98F800A0B8F80C7098F9C1
:10B768000EB0142204F58860314603F069F801220E
:10B7780084F84124534C94F83021022A35460BD1E1
:10B7880094F81821022A07D194F81E2122B9BAF197
:10B79800010F38BF4FF0010ABAF1010F2DD0BAF1ED
:10B7A800030F2CD0BAF1000F35D102229DF83C309E
:10B7B800DDF84090029362F34715012694F87C1057
:10B7C8008DF8321002220CA994F848008DF8302028
:10B7D80001F0A4F894F81A3194F830C194F81D11C6
:10B7E80040B20222002B6FD0BCF1010F65D10029B5
:10B7F80063D1002E6DD1104627E00422D6E700233E
:10B80800DDF83C90BDF840709DF942B0029365F0B8
:10B818001F050126D2E74FF0000BD946CDF808B036
:10B82800CCE74FF0010084F81A04DDE005F29A42F3
:10B838000BA900F0DDFA002800F020811320049BFA
:10B8480033871F4B002283F81A241D4BD3F89434F6
:10B85800C8F810306FE705F29A452A460BA900F0A0
:10B86800C7FA0028EAD10B9B84F82801C4F82C51A8
:10B8780084F8303102E1B9F1000F00F0FF80002AAE
:10B8880000F0FC804946E01C02F0C6FF94F837320D
:10B8980001332380F2E01220D1E70220CFE707200E
:10B8A800CFE7012047E7064B93F8912483F840A49B
:10B8B80042F0010283F89124C7E7EEB90220C4E7F9
:10B8C8007C140020B40E0020002E94D05845B8BF38
:10B8D800584694F87C308DF82000052294F84800EA
:10B8E8008DF8223008A901F02CF800283FF422AF87
:10B8F8009DF8203084F83930694A6A4BD2F89804A8
:10B90800D3F8904038B105F071FA664B84423CBFD9
:10B91800002283F83A20198F1A8F93F83001049186
:10B92800996A099152BA0028B9D093F81B0100B955
:10B93800186393F81801ADF85820013893F87C2063
:10B9480093F81A411491D0F1000BD3F888108DF8B0
:10B958005B204BEB000B93F8482093F83A0093F8E0
:10B9680068308DF85A3009AB00934F4B03904FF075
:10B9780001008DF84C0015918DF85C20A3F12F0182
:10B98800A3F1300213A88DF84D4000F0CFF8039BC7
:10B998004FEA0B1B4BEA431B00264BEA801B4BEA82
:10B9A800C413B1453E4C039308BF37463A4649464F
:10B9B80004F59C70CDE90A669B46268084F81A64D3
:10B9C80002F02AFFE9B2A570C5F34215FAB2042DB8
:10B9D800344E039B84F837223FF423AF072D3FF4FE
:10B9E8004AAF022D7FF459AF304D84F80D11042071
:10B9F800029984F80401FF2084F80C0184F82811C6
:10BA080084F81431D6F8E410C4F8085105F59B738E
:10BA18000AA8C4F8101184F83021C4F82C3100F0B9
:10BA280017FC00287FF437AF0A9BA4F844040BA83E
:10BA3800A4F81631C4F84C3400F0CEF900287FF48D
:10BA4800FDAE0B9BD3B196F93900FDF7A9FA94F82E
:10BA58003732002B3FF4FFAE0B9B0F2B3FF6E6AEC1
:10BA680005F58B720BA90F2000F0C2F900287FF4AE
:10BA7800E5AE0B9B63F3030B84F814B10598FDF74F
:10BA88004DFC00287FF4DBAE099B86F83A00B362D0
:10BA980000F07EF900283FF406AF1320D1E600BF7E
:10BAA8007C140020B40E00201C0F00207E140020FF
:10BAB80037B50B4D8DF8040004460F2295F8480061
:10BAC80001A900F03EFF40B1064A85F81C4192F8F2
:10BAD800913443F0200382F8913403B030BD00BFA5
:10BAE800B40E00207C14002010B5FFF7B9F8044606
:10BAF80088B90A4805F0B4F9094805F0B1F90948C8
:10BB080005F0AEF900F093F8FDF780FD064BDB6A0F
:10BB18009847204610BD0124FBE700BFE41700202A
:10BB2800FC17002014180020E42401082DE9F04F28
:10BB38008BB047780093149B90F90C8090F90D60B6
:10BB480090F80E908B464168196004469246002F83
:10BB580057D002238DF8103004A9C37B007C8DF8E0
:10BB6800123000F0DBFEB4F808C0618943B26068A7
:10BB7800984545466144B8BF1D46604534BF002717
:10BB88000127884209D30A218DF81010207C0193DF
:10BB980004A900F0C3FE019B46B2B4F808C060894E
:10BBA80061680CEB400E714520D3A1EB0C01B1FB91
:10BBB800F0FC00FB1C11C9B998450ADC237833B1A5
:10BBC8000223207C8DF8243006A900F0B5FE4FF042
:10BBD800010921238DF81030207CE37B8DF811506A
:10BBE80004A98DF8123000F099FE45B2009B8BF83D
:10BBF800005038468AF8006083F800900BB0BDE822
:10BC0800F08F4546F2E7704770477047704700204D
:10BC18007047704770477047002070470020704792
:10BC28000020704700207047002070477047704719
:10BC38007047022070470220704702207047704703
:10BC480000207047704770470020704700207047F9
:10BC5800704770477047000010B5054C4FF40372E9
:10BC68002046002102F0ECFD0020C4E9000010BDD0
:10BC78003C1A00202DE9F8438146174600293FD099
:10BC8800244B002503F1010C1A462801103312F841
:10BC9800018FB8F1000F36D19A42F8D11E4E3368A1
:10BCA8000BB9C6F800C073680BB1C3F800C03318ED
:10BCB800002401359C6083F80C900D302B01BAB23A
:10BCC80006EB05153044F750C6F804C002F0A4FD91
:10BCD800B9F1110F4FF0000398BF104C6B71D6F8F3
:10BCE800083298BF24FA09F403F1010398BF04F05D
:10BCF80001043B442C71C6F808324046BDE8F8837D
:10BD08004FF00108F9E70135202DBBD14FF00208AB
:10BD1800F3E700BF431A00203C1A00202007020066
:10BD280010B510B3124A1368984204D1036813601F
:10BD3800002304E00B4613B119688842FAD1516810
:10BD4800884208BF53600BB101681960D2F8083205
:10BD58008168013B00245B1A04602146C2F808325E
:10BD6800102202F06DFD204610BD0120FCE700BF47
:10BD78003C1A0020054B1B6813B11A798242FAD18C
:10BD8800002B0B600CBF0320002070473C1A0020DA
:10BD980010B5054B186800B910BD037B04680BB9D2
:10BDA800FFF7BEFF2046F6E73C1A002038B5084BDF
:10BDB800084C186800B938BD03790568112B05D8F7
:10BDC80024FA03F3DB0701D5FFF7AAFF2846F1E7BA
:10BDD8003C1A00202007020028B1044BD3F808328F
:10BDE8000360002070470120704700BF3C1A002004
:10BDF8002DE9F04107460E4615463AB331B3144BC8
:10BE08001C6800232CB93046FFF7E6FF0020BDE888
:10BE1800F081A268F91A0132914210D32279EA54CA
:10BE2800581C22895FFA80F8611D55FA80F002F0EB
:10BE3800F3FCA368246898445FFA88F3E2E7204695
:10BE48002468FFF76DFF002CF9D1DCE70120DEE75D
:10BE58003C1A00200238C0B211289ABF014B185C66
:10BE680000207047F71D010830B50B4B93F82020D0
:10BE78000446084672B100211C330578A54208D053
:10BE880001319842CDB20CBF04480430AA42F4D81C
:10BE9800002030BD1046FCE7481C0020541C002040
:10BEA80010B5084C00232060142204F10C00FF2177
:10BEB80084F82030C4E9010002F0C2FC012384F8B0
:10BEC800213010BD481C002010B50E4A92F82010F1
:10BED800042915D8936804781C7044785C70C47879
:10BEE800807898700131DC7082F8201002F11C0112
:10BEF8008B4214BF043302F10C039360012010BD80
:10BF08000020FCE7481C0020094B93F8200068B18A
:10BF18005A6803F11C018A4200F1FF3014BF043251
:10BF280003F10C0283F820005A600120704700BF1B
:10BF3800481C002010B5074B93F8202004460846FB
:10BF480032B15968FFF790FF10B101234470837034
:10BF580010BD00BF481C002008B5064B93F82020F0
:10BF68002AB15968FFF780FF08B1407808BD012061
:10BF7800FCE700BF481C002030B50A4A92F82010A0
:10BF8800536882F8210061B1916801241C32DD7880
:10BF9800587005B99C7093420CBF034B0433994207
:10BFA800F5D130BD481C0020541C002008B5044BB6
:10BFB8005968FFF759FF003818BF012008BD00BFB6
:10BFC800481C00202DE9F3410422154E04460021A7
:10BFD8000DEB020096F8208002F032FC0025EBB24F
:10BFE800984502D802B0BDE8F081736819782170CD
:10BFF8005A7862709F785FB1336820469B6898478B
:10C00800FFF782FF17B901A8FFF75EFF0135E6E7E2
:10C01800DB788DF804108DF805208DF80730EFE7F0
:10C02800481C0020014B93F820007047481C002052
:10C03800034B93F82000042894BF00200120704788
:10C04800481C00201FB50024CDE90244C41F8DF808
:10C0580000408DF801100C0AADF80420090C120CF0
:10C068008DF803108DF806208DF8073002461B0A5C
:10C07800012168468DF802408DF8083002F04BFA2D
:10C08800002818BF0E2004B010BD2DE9F04188B07B
:10C0980017460D460F9A064600284DD00024012168
:10C0A800CDE904448DF810109DF838108DF815105E
:10C0B800ADF81630190CCDE900441B0ECDE9024449
:10C0C8008DF81930ADF81A20130C120E07948DF85C
:10C0D80018108DF81C308DF81D20E3B24FEA0318B4
:10C0E800002D5FFA88F803DC002008B0BDE8F08175
:10C0F800013310218DF81F303A466B460DEB0100D5
:10C1080002F09FF90346C8B9102DAC46A8BF4FF0FE
:10C11800100CDAB2624503F1010303DB103D2DB2C6
:10C128000134DAE708EB020020326A44315C12F885
:10C13800202C4A403254ECE70920D6E70E20D4E7F9
:10C148000138032815D8DFE800F002080C100A4B64
:10C158001B681B690B6000207047074B1B685B69F5
:10C16800F8E7054B1B689B69F4E7034B1B68DB6921
:10C17800F0E70520704700BF6C1C00202DE9F04156
:10C18800C4B00C464A9E17461D468046B8B3B1F562
:10C19800807F36D84FF488720021684602F050FB41
:10C1A800492300934FF48073ADF804302B0C8DF8BD
:10C1B8000830330CADF80650ADF80A608DF80C3035
:10C1C80022460023414604A82D0E360E8DF80E3067
:10C1D8008DF809508DF80D608DF80F4002F01CFBAA
:10C1E80004F110014B9A3B4689B2684602F013F9F4
:10C1F80010B1012818BF0E2044B0BDE8F081092015
:10C20800FAE70D20F8E7000010B590B10A4C282293
:10C218000021206002F014FB2368084A1A600020FD
:10C228004FF0FF32C3E90302C3E90522C3E907223D
:10C2380010BD0820FCE700BF6C1C002000010101B4
:10C24800024B1B6818600020704700BF6C1C002060
:10C2580030B1044B1B68DB68013303600020704772
:10C26800092070476C1C002013B500230C4601936D
:10C27800D2B101A9FFF764FF18B9019B591C02D17B
:10C28800146002B010BD99B2611A002902DD0B4496
:10C298001360F6E702D113600720F2E71B0C1B04BA
:10C2A80003F580332344F3E70920EAE728B1044B78
:10C2B8001B681C334362002070470920704700BF89
:10C2C8006C1C002013B50446D8B1114B1A6893882A
:10C2D80001339BB29380C38200F057FA98B904F1F6
:10C2E8001803009321680123132202F08BF860B928
:10C2F800204600F04AFA003818BF0120000102B0B9
:10C3080010BD0920FBE71020F9E70E20F7E700BF72
:10C318006C1C0020F0B5054687B01C463BB32F4E79
:10C328003368DB68834257D894F82020002A14BF6A
:10C3380009220822834205D3204600F05AFA70B138
:10C3480010200AE0002301900093A36894F82810B5
:10C35800606AFFF79AFE0028EED007B0F0BD237997
:10C368002168B4F808C0A768043B9AB209B9092043
:10C37800F3E7B2F5807F2DD8ADF80EC08DF81730F1
:10C388004FEA174C04F12C033F0E8DF811700093FF
:10C398002F0C08234FF0490EADF80C008DF81470DF
:10C3A8008DF816002F0E0DEB0300CDF808E08DF880
:10C3B80010C0ADF812508DF8157002F023F808B1CE
:10C3C8000E20CAE7204600F014FA0028B8D13368D6
:10C3D800DD60C2E70D20C0E70620BEE76C1C002028
:10C3E8002DE9FF410A9D80460F4616461C46002D42
:10C3F8005AD0002303A910460393FFF7A1FE18B1F2
:10C40800062004B0BDE8F081039B9C4201D80133AB
:10C41800F6D1284600F05EF9002847D1264B1A7855
:10C42800424503D01A79424542D10120AA68BA424E
:10C4380040D103EB8002EB6A92F801802979CDE9BB
:10C4480000430439927828683B4689B2FFF796FE84
:10C458000028D6D195F820300194002B4FF0010325
:10C46800009314BF4246082295F82810686A3B4694
:10C47800FFF70BFE0028C4D1013E032EC1D8DFE828
:10C4880006F002070B0F0D4B1B681C611C62B8E716
:10C498000A4B1B685C61F9E7084B1B689C61F5E770
:10C4A800064B1B68DC61ACE70920AAE70F20A8E768
:10C4B8000B20A6E70220A4E7340100206C1C002012
:10C4C8001FB50A460B2A4FF00001CDE90011CDE94E
:10C4D800021107D00C2A13D00A2A0FD00A2005B05F
:10C4E8005DF804FB012802D120238DF8003068464E
:10C4F80002F011F8002818BF0E20F0E73023F4E707
:10C508000B21F4E738B5054602F000F8044678B97F
:10C518007DB9094B1B680B219878FFF7D1FF38B913
:10C528000C21FFF7CDFF18B90A21FFF7C9FF00B1A9
:10C538000E24204638BD00BF6C1C00202DE9F043B6
:10C5480080468FB00C461746002A6BD0002969D068
:10C55800002529461D2206A8059504F093FE8DF8AE
:10C568001350344D2B680DF114099E88CDF80490B2
:10C578000DF1130302933B7900933B683246214641
:10C58800404601F0E4FF00284ED138683A79494620
:10C5980002F042F9384600F04FF8002846D13C7ABC
:10C5A800FA79BB79240444EA02241C432B689A686C
:10C5B80094423DD99C609DF813000B21FFF780FF42
:10C5C800034658BB0C21FFF77BFF034630BB0A210B
:10C5D800FFF776FF034608BB7B7ABA7AFF7A3F04F7
:10C5E80047EA02271F433A46334621460920FFF708
:10C5F80029FD034690B933463A4621460820FFF7FD
:10C6080021FD034650B92A689DF813109170002146
:10C61800D1604FF0FF31C2E90411916118460FB0A3
:10C62800BDE8F0830923F9E70E23F7E70F23F5E7C1
:10C638000323F3E76C1C002010B50446002845D0FE
:10C648000168002942D011F8013B437103220630EA
:10C6580002F0E2F82046032250F8091B043102F0E8
:10C66800DBF82168CB79E3600A7A43EA0223E360C6
:10C678004A7A43EA0243E3608A7A43EA0263E36060
:10C68800CB7A23740B7B63742379212B1AD1102264
:10C698000D3104F1120002F0BFF81D222168501C70
:10C6A8008B5C6362085C43EA0023901C6362085C4D
:10C6B800033243EA004363628A5C43EA02636362CB
:10C6C800002010BD112B03DC0D22E7E70220F8E75C
:10C6D8000120F6E710B50446002854D00168002967
:10C6E80051D00B7843714B7883608A7843EA0223F0
:10C6F8008360CA7843EA024383600A7943EA0263A3
:10C7080083604B7903738B79C381CA7943EA022327
:10C71800027BC38102F00F020831103002F07CF86E
:10C72800237B002203F00F0384F8202084F82820BC
:10C73800227903F10800111A04290DDD2168093353
:10C74800043AD21A085C84F82000D2B2606A84F8ED
:10C758002820194402F060F8237922681A4400203E
:10C7680012F8043CE36212F8031C43EA0123E36273
:10C7780012F8021C43EA0143E36212F8012C43EA6F
:10C788000263E36210BD0220FCE710B5044660B303
:10C79800036853B30279162A29D942791A700146D7
:10C7A800082251F8060B013002F040F82146082211
:10C7B80051F80E0B093002F039F82368E28A5A74EE
:10C7C800E38A22681B0A93742368A269DA74A3694E
:10C7D80022681B0A13752368628B5A752368E27EE8
:10C7E8009A7517232371002010BD0120FCE7022051
:10C7F800FAE738B50446002863D00168002960D0FC
:10C80800037B90F8282003F00F03002A57D1083340
:10C81800207904321344984255D363790B70236806
:10C82800A2685A70A36822681B0A937023686289F9
:10C83800DA702368E27A1A712368227B5A712368B6
:10C84800E2899A71E38922681B0A2146D371227B07
:10C8580051F8100B02F00F02083001F0DDFF237BC6
:10C8680094F8282003F00F0303F108052AB1226881
:10C8780094F82010515503F10905206894F82820F0
:10C88800616A284401F0C8FF94F828302268E16AF8
:10C898002B44D1545A1CE16A206892B2090A815487
:10C8A8009A1C2168E08D92B28854DA1C216894F8A9
:10C8B8002F0092B2043388542371002038BD093305
:10C8C800A6E70120FAE70220F8E70000024B1A88E1
:10C8D80010431880704700BF701C002008B5074B34
:10C8E8001B883BB1FEF7BCF900280CBF00206FF095
:10C8F800020008BD6FF00100FBE700BF701C0020BC
:10C9080010B5034B00241C80FEF7A0F9204610BD8B
:10C91800701C0020B0FA80F04009704782B018B946
:10C92800084602B000F0CAB8002002B0704710B93B
:10C93800084600F077B9704710B9084600F08EB97C
:10C9480070470346084611460BB900F0E5B90020C8
:10C95800704710B9084600F071BD704710B9084615
:10C9680000F006BA0020704710B404460846114685
:10C978001A46019B14B910BC00F018BA10BC7047D5
:10C988000346084611460BB900F042BA002070472A
:10C9980010B40446084611461A4614B910BC00F0F3
:10C9A800AFBA002010BC704730B40546084611469F
:10C9B8001A46DDE902341DB9029430BC00F02EBBE2
:10C9C800002030BC704710B9084600F0DFBB0020DB
:10C9D800704710B9084600F06FBD0020704710B9C5
:10C9E800084600F0EEBB0020704710B9084600F07A
:10C9F800EBBB002070470346084611460BB900F010
:10CA080005BC0020704710B40446084611461A4673
:10CA1800019B14B910BC00F0FBBB092010BC704787
:10CA280010B40446084611461A4614B910BC00F062
:10CA380063BDC8B210BC70470048704701000102CE
:10CA4800064B10B51B6A0446984730B10448054B9D
:10CA5800204498428CBF0020012010BDE424010826
:10CA680040C220C980B92A00F0B5114B85B00C46E8
:10CA780010491F56054601F049F80F4BE4B25E6AAB
:10CA8800072D4FF00103CDE9024301460AD10522E3
:10CA98000023CDE900234FF47A727A431846B04751
:10CAA80005B0F0BD08220020CDE900203A46F5E7A0
:10CAB800331E01080C1E0108E42401081FB50023D9
:10CAC80000930378013B372B21D8DFE803F01C24BF
:10CAD8002020201E202020204143454E2055585B11
:10CAE8005E6164206C1E6E73787A20207D8126201A
:10CAF80020202020202020202020202083858A20FC
:10CB080020838A208C90C3780BB10223009300986D
:10CB180005B05DF804FB8378F6E743788DF80430B8
:10CB280005238DF805308378003B18BF01235B008F
:10CB38008DF8063010238DF80730304B1B6801A89C
:10CB480003F55872CDE9022300F0C0FF0090DEE73C
:10CB58004023DBE72023D9E7827890F9013012B926
:10CB6800274AD35CD2E7274AFBE7827890F901305D
:10CB7800002AF8D1244AF4E740F6B833C6E74FF460
:10CB88007A73C3E74FF4FA63C0E741F28833BDE72D
:10CB980041F27073BAE71D484FF47A7101F020FE34
:10CBA80000F5FA60D2E71A4BB0E7144B1B6803F59F
:10CBB8005873ABE7114B1B6803F55B73A6E71023AB
:10CBC800A4E70E4B1B68A1E74FF0834300939EE751
:10CBD800104BFBE7104B99E740F21113ADF800300A
:10CBE80095E7032392E790F901300C4AB9E70C491D
:10CBF80090F9010000F08AFFA8E700BF781C002028
:10CC0800BB1E0108C31E0108CB1E010818FCFFFF4C
:10CC180000EA06379A99094040F70937331E010898
:10CC28000C1E010837B50B4B02781B680C2101FB61
:10CC380002335B7A03EB4304074B1D6803690093D7
:10CC4800C3684278816805EBC40000F0DFFC03B0DC
:10CC580030BD00BF781C0020741C002070B586B061
:10CC6800027B6423ADF80030012A4FF00003CDE9C0
:10CC78000133CDE903338DF802308DF8143030D00C
:10CC8800022A39D05ABB03684BB343683BB31F4DE4
:10CC980080682B601E4B18226946186001F0BCFDA5
:10CCA8001C4B2C6893E807000C3384E8070093E8D2
:10CCB800070004F10C06032386E80700A4F86C3388
:10CCC800012204F55B7104F5587000F090FC2B68A4
:10CCD8004FF6B072A3F878230522C3F87C2306B078
:10CCE80070BD0A4908684360036100F55B7100F58F
:10CCF800587000F07CFCF2E7044B1B68B3F8602323
:10CD0800B3F86C130A43A3F86023E8E7781C002003
:10CD1800741C00206814010808B503460A2924D8A1
:10CD2800DFE801F006232323230B161B2321210010
:10CD3800BDE808400068FFF783BE90F900009978C5
:10CD4800052271B900F013FC003818BF012008BD96
:10CD5800052293F900000021F4E790F900005978C2
:10CD6800EEE70221EEE70722F3E70020EFE70000F5
:10CD780010B504791CB1012C0BD0002010BD0A4B52
:10CD880001681B68012203F5587000F030FC01208F
:10CD9800F4E7054B01681B68224603F55B7000F059
:10CDA80026FC2046EAE700BF781C0020F7B50528D6
:10CDB800144D1C46A8BF052058700E462946174634
:10CDC80000F0A4FE94F90130A070072B13D1322093
:10CDD80000F09CFD0C4BDB6D0546984704F10C02F6
:10CDE80008340346019200943A463146284600F03A
:10CDF80092FD03B0F0BD054A55F82310D05C00F051
:10CE08007DFDE7E70C1E0108E4240108331E010834
:10CE18002DE9F04F344F90F901607B68D0F8049009
:10CE28008BB00446884698470546002859D1E37CCC
:10CE380073B92E4A2378126803EB4303990002EB77
:10CE48008303D3F80490B9F1000F01D152F801908F
:10CE5800274B484613F906B0FB689847A37CD7F8D8
:10CE680018A022890993072E28D100230121CDE992
:10CE78000223204A0693CDE90431CDE90733052181
:10CE8800CDE900214FF47A7202FB0BF24CF25031DB
:10CE98001846D047637C13B3174B995D7B6D0D31F2
:10CEA800C9B228469847E07C3246494600F040FE21
:10CEB80088F8006001200BB0BDE8F08F0021012543
:10CEC8000823CDE90013CDE90715CDE90511CDE912
:10CED80003110292A1782B465A462846D9E7074BF8
:10CEE800DBE70020E7E700BFE4240108781C002006
:10CEF800331E010885450100CB1E0108BB1E010831
:10CF08002DE9F04F8DB090F90130DFF8FCA0DFF883
:10CF1800FC90CDE90A123E4A12F903B00278DAF819
:10CF280000300C2505FB02333A4A5B7A126803EBA2
:10CF3800430302EBC303044693F9021090F902007D
:10CF480000F0DFFD3449064694F9010000F0DEFDEB
:10CF5800A26861688046304600F005FD2178DAF85D
:10CF68000020D9F80C306943074650589847D9F83B
:10CF78001C309C4694F901300025072B4FF47A6346
:10CF8800CDE90753CDE905552DD10123CDE903534B
:10CF98000523CDE901534FF47A7303FB0BF3009398
:10CFA8003946434646F2A81228466746B8472378CA
:10CFB800DAF800200C214B4394F90110D05800F006
:10CFC800D9FDA18994F90100FFF74EFD0B9B217B48
:10CFD8001860D9F85430284698470A9B01201E70DB
:10CFE8000DB0BDE8F08F01200823CDE90350CDE94D
:10CFF80001032A46CDF800B0654643463946A8479E
:10D0080001200546D3E700BF781C0020E42401086E
:10D01800331E0108741C00200C1E01082DE9F04F76
:10D028008FB0002405468A46914698460494ADF888
:10D038001440ADF8024007264FF0010B2B7AA342AB
:10D0480006D9686804A9204400F0F2FB00285ED1E4
:10D0580002238DF8083002A86B7A8DF80A30FFF7A2
:10D068002DFDAB7A8DF81D309DF811308DF81E30EE
:10D078009DF812308DF81F309DF810308DF8203053
:10D08800EB7A8DF821302B7B8DF822306B7B8DF875
:10D09800233010238DF81C608DF824303A4E8DF81B
:10D0A8002C000DF102030A9305238DF82D30336807
:10D0B8000C930723ADF834302B6806930DF1120258
:10D0C80004AB0DF1110106A800F0CCFB07280546BA
:10D0D8000BD130680C22002100F5587001F0B0FB2C
:10D0E8003368BDF80220A3F860239DF811308AF850
:10D0F80000309DF8123089F800309DF8103088F81B
:10D108000030189B28461C700FB0BDE8F08F9DF8C2
:10D118001330BDF81470ADF802702044C4B2F3B9EE
:10D1280017B3194A00201168072602464FF00C0C65
:10D13800062B1BD10CFB00FE51F80EE0BEF1000FD0
:10D1480004D00BFA00F23A4397B2012201301028BA
:10D15800EED1002A3FF472AFADF802706EE75A1EA6
:10D16800042A01D9062BDCD0062667E747FA00FE19
:10D178001EF0010FEAD00CFB00FE51F80EE0BEF1E4
:10D18800000F08BF0626E1E7781C002038B50546E1
:10D198004068FFF755FC0522841D002195F9000021
:10D1A800E4B200F0E4F908B904F0FD0495F90100CF
:10D1B8000722002100F0DBF908B904F0FB0420463F
:10D1C80038BD00207047000010B503780F2B0446C7
:10D1D80018D84068FFF734FC22780B4902EB42026A
:10D1E8000968831C01EB820051F82220DBB21AB9CE
:10D1F80003F0FD0358B210BD032B06BF62684260FE
:10D208000223F7E70020F6E7781C00200220704789
:10D218002DE9F04FDFF838810446D8F8000099B0BE
:10D228008946174600211E460122032300F558703F
:10D23800CDE90611CDE908118DF814108DF81510F7
:10D24800ADF8163000F0B5F938B9D8F80020B2F8C2
:10D25800603343F00303A2F86033D8F80020637A00
:10D268008DF8283002F55871CDE90B12394A94F936
:10D27800083012680D920DF116020F922268109272
:10D2880062681192D4E90301A27A8DF8482001223C
:10D298008DF8492013AA82E803001025227DE18A2F
:10D2A8008DF8293018468DF85420ADF83850FFF71E
:10D2B800DBFB0AAB17930DF115031690009331466B
:10D2C800019705AB06AA10A800F0BCFB064698BB60
:10D2D8009DF81410204F013901F082FA1F4B1B6989
:10D2E8000393C4B24FF00C0B04F160036B44D8F8FD
:10D2F800000013F848AC9DF814300BFB0AFC01340D
:10D308003946B4FBF3F203FB1244D0F87C33B0F98E
:10D31800782350F80C00DDF80CC0E4B2E04728B1DF
:10D3280089F800A0304619B0BDE8F08F013D15F02E
:10D33800FF05D9D10D26F5E70C2801BFD8F8002044
:10D34800B2F8603343F00303A2F86033EAE700BFA2
:10D35800781C0020741C0020400D0300E424010800
:10D36800F8B50679012E054601D80620F8BD0F2E1E
:10D378002BD80368187A40F303000522002140B235
:10D3880000F0F5F82B680446187A40F303100522DC
:10D39800002140B200F0EBF8A8B1B4FA84F46409B3
:10D3A80029680B7A086843F3030243F3031352B264
:10D3B8005BB29A42C8BF0124FFF742FB48B9002C70
:10D3C800D3D10420D2E70124EAE70320CEE70520E1
:10D3D800CCE7002CFBD10C4F29683B6806EB4600D4
:10D3E80003EB80000C2201F017FA3A680C2303FBC8
:10D3F800062320465C72B2F860130123B3400B4346
:10D40800A2F86033B2E700BF781C002010B401789E
:10D4180001290ED9084B18680C234B43C418002265
:10D42800C250C4E9012200F5587010BC102200F067
:10D43800A7B8002010BC7047781C00202DE9F041E7
:10D4480086B050238DF81430037A102B074630D15C
:10D458004368DD7B6DBB0224A8466426062C14D8DD
:10D468007A68535D03932A44517843EA012303936E
:10D47800927843EA02437343CDE9033863B96846B7
:10D488008DF80040FFF7C2FF0DE0CDF80C808DF855
:10D498001480CDF81080F2E703AB01A801938DF852
:10D4A8000840FFF75DFF0134E4B2102C05F10305D5
:10D4B800D4D106B0BDE8F0811FB5026803791168C0
:10D4C80051B901A88DF80430FFF7A0FF78B9002002
:10D4D80040B205B05DF804FB02A802928DF80C304A
:10D4E800FFF73EFF0628F2D8024B185CF0E703204E
:10D4F800EEE700BF2C1E0108C90020B9034B0B44FE
:10D508009856C0B27047024BF9E700BF3B1E0108AE
:10D518007B1E0108F0B59A42069D03DB9DF9143085
:10D528009A4220DD0020F0BD03EB430331F814C01C
:10D5380005EB830300264CFA06F7FF0707D51F7A89
:10D5480007F00F0E724502DBB2EB171F0DDD013637
:10D55800102E03F10C03EED10134E4B22301DBB247
:10D568009842E1D8DEE70024F8E70120DBE78842AB
:10D5780004DB9042CCBF0020012070470020704798
:10D5880010B51409B4EB111F03464FEA11100ED35E
:10D5980091420CD202B201F00F0133F8124001207F
:10D5A80000FA01F124EA010123F8121010BD00204D
:10D5B800FCE7F0B528B100EB4105012700209142B6
:10D5C80000D3F0BD002435F802CB234607FA04F651
:10D5D80036EA0C0608BF013304F1010408BFDBB2C8
:10D5E800102CF3D118440131C0B2C9B2E7E710B525
:10D5F80000B149B910BD31F8134020F81340013388
:10D60800DCB2A242F7D8F5E70023F9E782B030B5DB
:10D61800048804936AB9B3F5616F18D349F6AF2546
:10D6280042F21072AB4298BF4FF47A72944238BFFC
:10D638001446012C38BF01246143BDE83040C3685B
:10D648008B428CBF5B1A0023C36002B07047642210
:10D65800ECE700002DE9F04F91B01546DDF86C803D
:10D6680004939DF8683009930C46064603F0B4FB12
:10D67800684ADFF8A4B10590A8F5F633303BB3FB50
:10D68800F2F3534303F5F63203F5A83303F5C073F9
:10D698000393182313FB05433032069208930025A1
:10D6A8004FF0FF3A089BA34207D1002D14BF504604
:10D6B8004FF0FF3011B0BDE8F08FBDF97030ADF814
:10D6C8002C300B99CDF86C804046CDF8288003F0BB
:10D6D80013FBB4F800906EB9B8F5616F5BD349F6E7
:10D6E800AF2242F21073904598BF4FF47A73994570
:10D6F80038BF99464B46012B38BF01230793002EAC
:10D7080052D1B9F1640F48D1A0605F46A1680EA854
:10D7180003F014FB0F9B0093DDE90A120E9B0CA883
:10D7280003F06BFA049B0C9A0BB9099B2BB1236984
:10D73800BB4202D1394B9A420DD9394BE760984523
:10D7480009D90023ADF83430069B0D990C9318467F
:10D7580003F0D2FAA060606800B9E760276126B1DB
:10D7680003F044FBE3680344E360D4E903329342E3
:10D77800059B1D996360079B88BFE2604B43E16886
:10D78800994202D20498A8B9A6B101231D44237571
:10D79800EDB2183486E76423A9E7B9F57A7F0ABFA2
:10D7A800204F214FA060B1E7049B0BB9C4F80CB01F
:10D7B8005F46D0E700209342207506D85B1A9A4549
:10D7C80005F1010528BF9A46EDB2002EE1D1B9F165
:10D7D800640F164AADF8346019D049F6B023B9F58C
:10D7E8007A7F18BF1346904584BF039A9B180C9301
:10D7F8001C9B00930CAF97E806001B9B384603F070
:10D80800FCF997E8030003F077FA8246C1E74FF482
:10D818006163E8E78051010040771B007F510100F8
:10D828002FEC010080A81201002E930230EC0100B9
:10D838000378032B14D1437803F00F021B098A7075
:10D848004B7083788B80C27843EA02238B800379FC
:10D85800C3F3021203F00F03CA700B700520704760
:10D86800002070472DE9F34798464379057990F9E8
:10D8780007609146044690F906208A4683B190F9DC
:10D88800087075B30F2A12D194F909200F2E1ED1F2
:10D8980094F90A60072D24D1002F08BF012720E042
:10D8A80090F90B7090F9092090F90A60E9E7A369EB
:10D8B800019394F915300093216994F91430207B71
:10D8C800FFF728FE0028E1D105F0FD05DEE794F911
:10D8D8001D30B3420FDC94F91C30B342DADA05F09C
:10D8E800FB0528468AF8002089F8006088F800704F
:10D8F80002B0BDE8F0871E46CCE70000024B03FAF1
:10D9080000F0B0FBF1F0704740420F004FF4FA53BB
:10D91800B3FBF0F0704730B54FF47A750C1F6A43CB
:10D9280000FB042252001EBF00F1FF341219B2FBA3
:10D93800F0F2914238BF1146039A116082004843C1
:10D948001CBF013040084FF47A71121A01FB1323EF
:10D95800002BCABF03F2E73393FBF1F1B3FBF1F1FC
:10D96800049B196030BD38B5400014460D46F4F7E5
:10D978004DF801462846F3F797FF2146F3F794FF41
:10D98800F3F786FE03F0C4FCF3F762FF40B238BD3C
:10D998002DE9F74F019300231F469C461C01058A79
:10D9A8005FFA84FE04F0F004A54206D8019B82F8D1
:10D9B80000C01F7003B0BDE8F08F0EEB4E054FEAB4
:10D9C8004309AD000024466836F809602641F60789
:10D9D80027D5866806EB050A765916B3067836B950
:10D9E800466926B136F809602641F60719D59AF82E
:10D9F800086090F901B046F303084FFA88F8D84553
:10DA08000FDC46F3031676B25E450ADB9AF8096026
:10DA180006EB4608C66806EBC806367D4EB90137E0
:10DA2800FFB20134102C05F10C05CCD10133DBB267
:10DA3800B4E70CF101060EEB040801F80C805FFA5C
:10DA480086FCEEE72DE9FF4704464068DDE90C67F0
:10DA58001D468A46914603F0C9F923681B1A3B60A4
:10DA68004FF000080123337085F80080636813B114
:10DA78002368834224D8CAF80080D4F81CC0A3695C
:10DA88009CF800E00393D4E9030101AB83E80300A9
:10DA9800237D0093DCF80C10237A627A7046FFF736
:10DAA800D9FD334638602A46E0694946FFF770FFDA
:10DAB8002B782BB1C7F80080002004B0BDE8F087B0
:10DAC8003378002B14BF0B200C20F6E737B590F9FC
:10DAD800002090F90250954204460FD0013A52B204
:10DAE80095420BD0A368019394F9013000936168C3
:10DAF800E0782B46FFF70EFD0028EFD0104603B064
:10DB080030BD8842B8BF08467047000051F8200071
:10DB1800054B984205D0054BC31A5842584140005E
:10DB280070470120704700BF90D0030020A1070074
:10DB380005281FB50ED80C4B53F820300093CDE9BB
:10DB480001120A4B01220021022002F05BFE05B0FF
:10DB58005DF804FBCDE90012054B012200210220EB
:10DB680002F050FEF3E700BF3C1F0108D31E010876
:10DB7800F21E010807B5054BCDE90001012200217D
:10DB8800022002F03FFE03B05DF804FB0E1F0108FF
:10DB980010B5102204460021F13000F051FE00219A
:10DBA800C4F814112046F022BDE8104000F048BE29
:10DBB80002460846102100F0A5B92DE9F0430446B5
:10DBC800D0F8140185B00E46154604F2011988B341
:10DBD800C0F110089045474628BF1746BAB24844D6
:10DBE80000F01AFED4F814313B440F2BC4F814315A
:10DBF8002DD9A8452BD204F1F00304F5807113F850
:10DC0800012F187C8B4282EA00021A70F7D104F1C6
:10DC1800F10810224146684600F0FEFD224669469A
:10DC2800684600F0E9F910226946404600F0F4FD24
:10DC38003E44ED1B04F5807804F1F107102D09D856
:10DC4800AAB23146484600F0E7FDC4F8145105B0C1
:10DC5800BDE8F08304F1F003711E13F8012F11F8E9
:10DC6800010F434582EA00021A70F6D110223946A4
:10DC7800684600F0D1FD22466946684600F0BCF9C6
:10DC880010226946384600F0C7FD1036103DD5E72A
:10DC9800F0B589B00C46102200210546684600F010
:10DCA800CFFD22466946684600F0A6F99DF9003086
:10DCB800002B6A464FF0000143DA137812F8010F7F
:10DCC80001315B0043EAD0130F2902F8013CF4D17B
:10DCD8009DF80F305B0083F08703D4F81401DBB2A2
:10DCE80010288DF80F303BD104F58073694604F590
:10DCF800887013F8016F11F8012B984282EA060226
:10DD08001A70F6D104F1F00304F5807113F8012FAD
:10DD1800187C8B4282EA00021A70F7D110220DEBB0
:10DD2800020004F1F10100F077FD2246294604A81B
:10DD380000F062F910220021684600F081FD09B068
:10DD4800F0BD137812F8010F01315B0043EAD013DC
:10DD58000F2902F8013CF4D19DF80F305B00BCE7B5
:10DD68009DF90030002B6A464FF0000137DA13782E
:10DD780012F8016F01315B0043EAD6130F2902F84C
:10DD8800013CF4D19DF80F305B0083F08703471CFA
:10DD9800DBB28DF80F30102F04EB0003C0F10F0633
:10DDA8004FF0800288BF002600F5817083F80121BA
:10DDB8000021324620443E4403F064FAC4F814615A
:10DDC80004F58073694604F5887013F8016F11F83B
:10DDD800012B984282EA06021A70F6D192E713786C
:10DDE80012F8016F01315B0043EAD6130F2902F8DC
:10DDF800013CF4D19DF80F305B00C8E70A7803783E
:10DE0800534003704A784378534043708A78837844
:10DE180053408370CA78C3785340C3700A79037932
:10DE2800534003714A794379534043718A7983791E
:10DE380053408371CA79C3795340C3710A7A037A0C
:10DE4800534003724A7A437A534043728A7A837AF8
:10DE580053408372CA7AC37A5340C3720A7B037BE6
:10DE6800534003734A7B437B534043738A7B837BD2
:10DE780053408373CA7BC37B5340C373704710B549
:10DE88000B7814786340037054784B786340437080
:10DE980094788B7863408370D478CB786340C37070
:10DEA80014790B796340037154794B79634043715A
:10DEB80094798B7963408371D479CB796340C3714A
:10DEC800147A0B7A63400372547A4B7A6340437234
:10DED8008B7A947A63408372D47ACB7A6340C37224
:10DEE800147B0B7B63400373547B4B7B634043730E
:10DEF800947B8B7B63408373CB7BD27B5340C37310
:10DF080010BD0000A1F11003DBB2102B2DE9F04782
:10DF180004D8374C24FA03F3DB0705D4002382F82E
:10DF2800F030FF20BDE8F087531E4418A0424ED1C0
:10DF380001F11C039B005FFA83F9C3F30313013B50
:10DF48002C4D82F8F03001240B46D618B3FBF1F0C3
:10DF580001FB103010F0FF0016F804AC16F803ECC3
:10DF680016F802CC16F8017C36D115F80E8015F893
:10DF78000CE015F807C015F80A70E00900EB40003E
:10DF880084EA080800EBC0006400C0B2E4B2444070
:10DF9800C246581AC0B212F800808AEA080A02F883
:10DFA80003A01044043390F801808EEA080E86F826
:10DFB80001E090F802E08CEA0E0C86F802C0C07806
:10DFC800DBB247409945F770BFD80020AAE710F8A0
:10DFD800015B03F8015FA9E71829DAD9102801BF06
:10DFE80015F80AA015F80EE015F80CC0EF5DD0E79B
:10DFF80001010100542101082DE9F04FA3B092F866
:10E00800F0301D911B920193002B00F053810146C3
:10E018001EA8FFF734FF1B9BA74CA84DA84E103332
:10E028000293002303939DF87C0004909DF88600DA
:10E038000590205C06909DF87B000790205C089076
:10E0480004989DF881C0205C099014F80C000A908F
:10E058009DF880000B909DF885009DF878809DF8CC
:10E068007DE09DF882A09DF887900C909DF87A003D
:10E07800029B1C9314F80A2014F8093014F80810AD
:10E0880014F80E700D90205C0E909DF87F000F9094
:10E09800205C10900B98205C11900C98205C1290DA
:10E0A8009DF8840013909DF8790014909DF87E00E7
:10E0B8001590205C16909DF883001790205C1890AE
:10E0C8001398205C19901498205C1A9003980130DA
:10E0D80003900298DDF804B0103002909DF80C000F
:10E0E800834536D88DF878108DF87A2009990E9ADC
:10E0F8008DF87C108DF882201199069A8DF8801081
:10E108008DF87E201999169A8DF884108DF886203E
:10E118000A99189A8DF87D108DF887201299109A0F
:10E128008DF87B301B9B8DF881108DF883201A9910
:10E13800089A1D988DF885108DF87F201EA903EB8D
:10E148000B128DF87970FFF79AFE002023B0BDE816
:10E15800F08F15F808B082EA03008BEA000016F881
:10E168000EB080EA0B008DF8780015F80E004B40D1
:10E17800434016F80A0043408DF8793081EA0703D6
:10E1880015F80A10594016F80930594016F80830A1
:10E198008DF87A107A40534015F8092053408DF8CD
:10E1A8007B30089A069B5340049AAA5C534016F8A1
:10E1B8000C2053408DF87C30DDE908325A4015F8C0
:10E1C8000C305340059AB25C53408DF87D30DDE940
:10E1D80009325A40059BEB5C5340079AB25C5340A6
:10E1E8008DF87E30069B0A9A5340049AB25C5A40D6
:10E1F800079BEB5C5A408DF87F200E9B109A53408A
:10E208000B9AAA5C53400C9AB25C53408DF880304C
:10E21800DDE910325A400C9BEB5C53400D9AB25C1E
:10E2280053408DF88130DDE911325A400D9BEB5C8B
:10E2380053400F9AB25C53408DF88230129A0E9B6D
:10E2480053400B9AB25C5A400F9BEB5C1C995A40A6
:10E258008DF88320169B189A5340139AAA5C534052
:10E26800149AB25C53408DF88430DDE918325A4074
:10E27800149BEB5C5340159AB25C53408DF8853083
:10E28800DDE919325A40159BEB5C5340179AB25C92
:10E2980053408DF886301A9A169B5340139AB25CF5
:10E2A8005340179AAA5C1EA853408DF88730FFF791
:10E2B800A5FDB8E6FF2049E754210108541F0108CD
:10E2C8005420010808B538B1044A05491060D8221D
:10E2D80000F0A2FA002008BD0220FCE77C1C002008
:10E2E800842601080A4B1A6870B5002302F1180544
:10E2F80003EB03142E5D864204D1183422440A60CD
:10E30800002070BD01330B2BF2D10320F9E700BFC9
:10E318007C1C00202DE9F041CCB00646DDF8488190
:10E3280017461C460D4631B3B8F1000F23D006A896
:10E33800FFF72EFC204601A9FFF7D4FF0446B0B929
:10E34800019906A80131FFF733FC26B110223146A6
:10E3580006A8FFF732FC3A46294606A8FFF72DFC27
:10E3680006A902A8FFF794FC029BC8F800302046D3
:10E378004CB0BDE8F0810224F9E7000030B595B053
:10E3880013A90446FFF7AEFF002830D11B490C2320
:10E3980003FB00F2555CA5422BD1139B187C10900F
:10E3A800D87B0F90987B0E90587B0D90187B0C9023
:10E3B800D87A0B90987A0A90587A0990187A089027
:10E3C800D87907909879069058790590187904902B
:10E3D800D8780390987802900A445B780193936800
:10E3E80000930022064B1146022002F00BFA15B0EA
:10E3F80030BD01300B28CBD1F9E700BFCC23010891
:10E40800542201080B2B10B402D810BCFFF782BFAE
:10E41800032010BC704730B50D4685B01446014640
:10E4280068B103AA002000922A460390FFF772FF02
:10E4380018B90398001B18BF012005B030BD022091
:10E44800FBE72DE9F0430D46BFB0144699468046D8
:10E4580020B31BB311F00F0122D1F02201A800F064
:10E46800EFF920466946FFF73DFF044648B9009892
:10E4780001AA10210130FFF745FD2E46AF1BFFB260
:10E488001EB920463FB0BDE8F08301AA09EB070199
:10E4980008EB0700FFF7B0FD103EEFE70224F0E7B6
:10E4A8000524EEE7F0B5184E3468024685B00846F4
:10E4B800002304F1180103EB03154F5D97421ED1A9
:10E4C8000D2A05F1190513D10023CDE90033CDE953
:10E4D80002330C2210216B46FFF7B3FF0446306865
:10E4E80010226946284400F097F9204605B0F0BD8F
:10E4F80001461022601900F08FF90024F5E7013376
:10E508000B2BD8D10324F0E77C1C002009B1FFF7BE
:10E51800C9BF022070471FB51446A0B10C2A01D10B
:10E528000B2912D10023CDE90033CDE902330A4685
:10E538006B461021FFF785FF18B969462046FFF79B
:10E54800B1FF04B010BD0220FBE70320F9E7F8B5DE
:10E558001E46DDE907479DF818505BB354B34FB327
:10E56800212D29D819462A46204600F055F90122BE
:10E57800631C691EB018FFF764FFF8B9E37ADB097A
:10E588003B70EBB96319204613F8012C13F8021CF1
:10E59800120642EA014213F8041C0A4313F8031C4A
:10E5A800012342EA0122291FFFF735FF003818BF6F
:10E5B8000120F8BD0220FCE70520FAE70720F8E76C
:10E5C8000420F6E708B5014630B1044B0822186864
:10E5D80000F022F9002008BD0220FCE77C1C002086
:10E5E80008B530B1044B0822196800F015F900206D
:10E5F80008BD0220FCE700BF7C1C00207FB5124E3E
:10E608000023044602A801930D46FFF7E9FF33688B
:10E618005B6901936CB102AA082312F8011B41B986
:10E62800013B13F0FF03F8D102A8A04702A8FFF7A7
:10E63800C9FF35B1019B23B901A8A8473368019ADE
:10E648005A61002004B070BD7C1C002008B501464A
:10E6580038B1054B18680822104400F0DDF8002096
:10E6680008BD0220FCE700BF7C1C002008B538B1BB
:10E67800044B19680822114400F0CEF8002008BDA8
:10E688000220FCE77C1C0020034B1B6802280CBFFF
:10E6980019615961002070477C1C002041B1054B6D
:10E6A8001B6802280CBF1B695B690B600020704760
:10E6B800022070477C1C002030B58FB0002405462E
:10E6C8000CA80994FFF78CFF9DF8373007939DF845
:10E6D800363006939DF8353005939DF83430049311
:10E6E8009DF8333003939DF8323002939DF8313012
:10E6F80001939DF830300093224621461E4B02209C
:10E7080002F080F80AA8FFF7B1FF9DF82F300793B1
:10E718009DF82E3006939DF82D3005939DF82C30EA
:10E7280004939DF82B3003939DF82A3002939DF8AB
:10E73800293001939DF82830009322460F4B21463B
:10E74800022002F05FF809A92846FFF7A7FF9DF805
:10E75800243003939DF8253002939DF826300193C9
:10E768009DF8273000932246054B2146022002F0EF
:10E7780049F80FB030BD00BFB0220108EE220108F1
:10E788002C23010808B50020FFF7F8FD0120FFF74A
:10E79800F5FD0920FFF7F2FD0820FFF7EFFD002047
:10E7A800FFF78AFF002008BD10B504460B20FFF7CD
:10E7B800E5FD0C20FFF7E2FD0920FFF7DFFD08204B
:10E7C800FFF7DCFD0A20FFF7D9FD2046FFF774FFAD
:10E7D800002010BD014B1860704700BF3C010020AD
:10E7E8000B4A30B514680B4D43F2390305FB04336B
:10E7F8001360091A6FF00042B3FBF2F2C2EBC27267
:10E8080001319B1A93FBF1F201FB1233184430BD1E
:10E818003C0100206D4EC64101380A44914200D1A6
:10E82800704711F8013B00F8013FF7E710440A442C
:10E83800914200D1704711F8013B00F8013DF7E71C
:10E8480002F020BD30B530B10A4D01444FF0FF331E
:10E85800814201D1D84330BD10F8012B5340082222
:10E8680043F30004013A2C4092B284EA5303002A8D
:10E87800F6D1EDE72083B8ED01207047054B4FF442
:10E8880000529A62044B1B6813B15B6803B11847C6
:10E89800704700BF00040048801D0020054B4FF45E
:10E8A80080529A62044B1B6813B1DB6803B11847A6
:10E8B800704700BF00040048801D002001207047F9
:10E8C8000120704701F048B901F036B910B501F0E0
:10E8D80019FE0E21044640F61F1001F02DF92046BE
:10E8E800012101F0F9FDBDE8104001F0D7BA0000A0
:10E8F80070B50C4E01EB40030D46B3654FF6FF7142
:10E90800002304461A46084601F05EFB96F85600B6
:10E91800002101F0E1FD29462046BDE8704001F0E4
:10E9280095BA00BF9C1D002010B5044601F0AAFE50
:10E9380001281CD101F0AEFE34B11248214602F084
:10E9480017FB104802F0DAFA0F4C104B00214FF475
:10E958008052A1659A6194F8560001F0BDFD637874
:10E968006BB16FF07F40BDE8104001F053BA00234F
:10E9780040F262211A46084601F026FBDCE7A0684F
:10E988008001F0E7841D00209C1D00200004004841
:10E99800002001F0BFB9000008B501F0C7F804383D
:10E9A800C0B2032896BF024B0020185C08BD00BF08
:10E9B800E024010808B501F0BAFD033008BD01F0F4
:10E9C80049B901F009B908B501F000FD00B208BD68
:10E9D80038B50D46144601F05DFB284601F092FD5E
:10E9E8000E21054640F61F1001F0A6F82846012121
:10E9F800074D01F071FD01F051FA4FF47A7161434E
:10EA0800284602F0B5FA2846BDE8384002F076BA42
:10EA1800F81D002001F03EBB08B5084B002193F813
:10EA2800560001F059FD00234FF4C0711A460846FC
:10EA380001F0CAFABDE8084001F024BA9C1D002084
:10EA480010B5044601F01EFE01281CD101F022FE7B
:10EA580034B11248214602F08BFA104802F04EFAFF
:10EA68000F4C104B00214FF48052A1659A6194F825
:10EA7800560001F031FD63786BB16FF07F40BDE85F
:10EA8800104001F07DB9002340F262211A46084681
:10EA980001F09AFADCE7A0688001F0E7841D002005
:10EAA8009C1D00200004004808B54FF0040001F048
:10EAB80017F9BDE808400220F4F71AB808B5002392
:10EAC8001A461946184601F07FFABDE8084001F0D9
:10EAD8006DB900001D4B73B51D4D186000241D480D
:10EAE8006C70C5E90144AC6501F098FAAC8101F09D
:10EAF80003FA2146204601F04BFC2146042201205E
:10EB080001F0FCFA144E154D4FF6FF7123462246CC
:10EB1800084601F059FAFFF7C7FF2246104B009448
:10EB28004FF0FF31304602F03DF90E4B009422467B
:10EB38004FF0FF31284602F035F9304602F090F9DF
:10EB4800284602B0BDE8704002F08AB9801D002056
:10EB58009C1D002025FB0008F81D0020841D0020B6
:10EB680085E80008A5E800080128084805D1084BF1
:10EB7800C17719700E3001F0A7BB437D012B03D17B
:10EB8800034B81751970F5E7704700BF9C1D002085
:10EB9800400100200D4B10B504461873587301202E
:10EBA80000F016F85CB134214FF4E86000F0C4FFBF
:10EBB8004421BDE8104040F2417000F0BDBF14216F
:10EBC8004FF4E86000F0B8FF2421F2E79C1D002014
:10EBD80038B5114C0546207001F061FD052D04D8AB
:10EBE800DFE805F0090B03171709032001F070FA95
:10EBF8000023637338BD0020F8E7012001F068FAAC
:10EC0800207B637B8342F5D06073BDE83840FFF713
:10EC1800C1BF0220EAE700BF9C1D00202DE9F04398
:10EC28001E4687B000230546CDE901330C4617463A
:10EC380001F027FD032D61D8DFE815F07B00C30044
:10EC48000E010400A27C082A04D94FF0FF3007B057
:10EC5800BDE8F083A16801A801F0DCFE2168002965
:10EC6800F3D042F210729142E37C864D51D80322D0
:10EC7800AA7385F83820E96385F844304FF0020814
:10EC88006368A17DDB002B820423AB74A37CDB00CB
:10EC9800EB7402294FF000032B75637D02D0227DAF
:10ECA800022A42D103F10F02D2B2012A01D9012B63
:10ECB800CBD1754B754A196803944FF0010903A825
:10ECC8008DF8149001F0DAFC0028BED1287685F87A
:10ECD80017906875FFF75CFE4046FFF779FF6C48B0
:10ECE80001F086FA6B4801F0EFFA01A800F084FF02
:10ECF800208A00F055FFA08900F09AFF384601F0FD
:10ED080001FC604C84F8560001F0C0FC66600020ED
:10ED18009DE74FF00008E963890885F80E8085F8BB
:10ED2800388085F844302964AAE7EB7529766A7536
:10ED3800D0E72368002B88D0A27C082A85D8514DBB
:10ED4800A16801A801F066FE002385F83830226822
:10ED5800EA63E27C85F84420A269AB732A6462689E
:10ED6800A17DD2002A820422AA74A27C2B75D2002B
:10ED78000229637DEA7402D0227D022A1DD103F1A3
:10ED88000F02D2B2012A02D9012B7FF45EAF3E4BAB
:10ED98003E4A196803944FF0010803A88DF81480BF
:10EDA80001F06CFC00287FF450AF287685F81780B6
:10EDB8006875FFF7EDFD00208FE7EB7529766A751A
:10EDC800F7E7304D012185F83810227885F8502072
:10EDD800637885F85130A37885F85230E3788B4210
:10EDE80002D0022B03D03BB985F8533004E00B3A2C
:10EDF800012A29D885F853104FF0010885F80E80AC
:10EE0800A388AB83A379AB77E37985F82030237A9D
:10EE180085F82130FFF7BCFD4046FFF7D9FE1C48B6
:10EE280001F0E6F91B4801F04FFA95F85130062B2E
:10EE380040F689000AD100F08FFE00F0FB0140F691
:10EE4800890000F079FE59E70023CDE700F084FE41
:10EE580040F00401C9B2F2E72368013BB3F57A7FB9
:10EE6800BFF4F3AE0320FFF7B3FE0648022380F891
:10EE7800383023688364162380F84C30383001F02A
:10EE8800B7F93BE79C1D0020801D0020F81D0020DD
:10EE9800D41D0020AA1D00202DE9F041002686B0CF
:10EEA8001F461446CDE9016680460D4601F0E9FB90
:10EEB800B442764C16BF0123334637466370B8F127
:10EEC800000F06D0B8F1010F7CD0002006B0BDE8D5
:10EED800F081AB68002B00F0D680EB68002B00F0C7
:10EEE800D280AA7F082A00F2CE80296901A801F001
:10EEF80091FD2868003818BF012000F0D9FF84F878
:10EF08003880AB68E36395F8203084F8443068684B
:10EF180001F05AFB84F80E8084F84500EB68DB00AA
:10EF28002382EB7FA374AB7FDB00E37495F8213079
:10EF3800237595F82230002B3ED12A7D95F82410B0
:10EF4800A275022995F8232001D0022B36D102F1AF
:10EF58000F03DBB2012B02D9012A40F09480002371
:10EF68008DF814304A4B4B4A1968049503A801F0F0
:10EF780085FB002840F0878001232076E3756075C3
:10EF8800FFF706FD0020FFF723FE434801F030F9A4
:10EF9800424801F099F901A800F02EFEA88B00F074
:10EFA800FFFD288B00F044FE4FF4FA53AA687B4318
:10EFB800B3FBF2F3A36088E7FF22BFE7E27521768F
:10EFC8006375DDE72B8E002B5DD095F83230A86A8B
:10EFD800012B0CBF95F814804FF0FF08003818BFBC
:10EFE800012000F065FFF8B200F06EFF012184F8FF
:10EFF800381095F82C2084F8502095F82D3084F896
:10F00800513095F82E3084F8523095F82F308B42D5
:10F0180002D0022B03D03BB984F8533004E00B3AFA
:10F02800012A28D884F853102B8EA38395F8323000
:10F03800A377AB8E23840126A67384F81F80FFF77D
:10F04800A7FC3046FFF7C4FD134801F0D1F8134878
:10F0580001F03AF994F82130B34240F236700CD1FD
:10F0680000F07AFD00F0FB0140F2367000F064FD1C
:10F078004FF6FF739EE70023CEE700F06DFD40F0EA
:10F088000401C9B2F0E74FF0FF301FE79C1D0020D4
:10F09800801D0020841D0020D41D0020AA1D0020F2
:10F0A8002DE9F04F85B082460E9DBDF840B09DF821
:10F0B80044709DF84890019288461E4601F0E1FA96
:10F0C800BAF1010F524C54D0BAF1040F00F09180FC
:10F0D800BAF1000F3AD10B22304684F8442084F864
:10F0E80038A0E56301F070FA019B23644FEACB0373
:10F0F800B9F1000F238241F60403638214BFF2239F
:10F108000123E37587F001070123237684F845007E
:10F1180084F80EA084F814A06775FFF739FC5046F0
:10F12800FFF756FD04F1380001F062F804F10E0013
:10F1380001F0CAF8374A1068516802AB03C302A845
:10F1480000F05AFD40F2FF1000F02AFD404601F0A1
:10F15800D9F90E2184F8560040F61F1000F0ECFC97
:10F1680094F8560001F092FA169B636005B0BDE86A
:10F17800F08F294984F838A0EAB2895D84F85020D4
:10F1880076BB0B3D012D8CBF00250125053A012AD0
:10F1980004D8BBF10C0F38BF4FF00C0B1F4B9DF878
:10F1A8003C201B7884F85350E37701259DF85430B0
:10F1B80084F8511084F8522084F82130A573A4F8FB
:10F1C8001CB0A77784F82090FFF7E2FB2846FFF7EA
:10F1D800FFFC134801F00CF8124801F075F8B5E788
:10F1E800012E04D1A5F10C035D425D41CEE7002557
:10F1F800CCE75046FFF7ECFC022384F8383004F1E2
:10F2080038001623A56484F84C3000F0F1FF9DE720
:10F218009C1D002080140108AE2401084001002034
:10F22800D41D0020AA1D00202DE9F04F87B0DFF87B
:10F23800B4B29DF864A09DF84C90029314469DF8D2
:10F2480054309DF85020BDF84880039205468BF84D
:10F2580001A0BDF8446001930F4601F012FABAF11B
:10F26800000F18BF4FF00008DFF87CA2039AB9F12D
:10F27800000F08BFFF22012D8AF8002000F0C88087
:10F28800052D48D0002D40F0C080284600F010FE23
:10F298000B2238468BF844208BF83850CBF83C408A
:10F2A80001F092F9019B8BF8450041F60402002B0E
:10F2B800ABF812209AF800208BF8162014BFF2221F
:10F2C80001228BF81720F600012289F001098BF83A
:10F2D80018208BF80E50ABF810608BF814508BF890
:10F2E8001590FFF755FB2846FFF772FC0BF1380025
:10F2F80000F07EFF0BF10E0000F0E6FF7B49086886
:10F30800496804AA03C204A800F076FC40F2FF1082
:10F3180000F046FC71E0012000F0CAFD09224FF020
:10F3280000098BF8442038464FF44872CBF8402047
:10F338008BF83890CBF83C4001F046F94FF48052F6
:10F34800ABF812209AF800208BF845008BF81620AD
:10F3580028460122F6008BF817208BF80E90ABF8A0
:10F368001060ABF814908BF81890FFF731FC0BF194
:10F37800380000F03DFF0BF10E0000F0A5FF5B49DF
:10F388008868C96804AA03C204A800F035FC40F2E2
:10F39800FF1000F005FC40F6B80000F0DDFB00F0BF
:10F3A800EF0140F6B80000F0C7FB042140F6B900B1
:10F3B80000F0C2FB40F69B0000F0CEFB00F0E3013A
:10F3C80041F0080140F69B0000F0B6FB40F2D16026
:10F3D80000F0C2FB40F01801C9B240F2D16000F061
:10F3E800ABFB40F2AC6000F0B7FB00F08F0141F0DE
:10F3F800500140F2AC6000F09FFB4FF4FA5202FB60
:10F4080008F2B2FBF4F2CBF8082007B0BDE8F08FA1
:10F41800002000F04DFD36498BF83850E2B2C95D46
:10F428008BF85020002F4DD10B3C012C8CBF0024B1
:10F438000124053A012A02D80C2E38BF0C26029B5B
:10F448009AF800208BF852308BF85340019B8BF8C8
:10F458001F2001249DF860208BF821208BF8511083
:10F468008BF820308BF80E40ABF81C608BF81E90A0
:10F47800FFF78EFA2046FFF7ABFB1E4800F0B8FEF8
:10F488001D4800F021FF5FFA88F000F01DFD40F6EE
:10F49800A30000F061FB00EA040140F6A30000F0BD
:10F4A8004BFB9BF82120A24240F2367013D100F0AA
:10F4B80053FB00F0FB0140F2367000F03DFB4FF6C5
:10F4C800FF72A0E7012F04D1A4F10C035C425C4158
:10F4D800AFE70024ADE700F03FFB40F00401C9B2FC
:10F4E800E9E700BF9C1D00204001002080140108AE
:10F4F800AE240108D41D0020AA1D0020F0B58BB051
:10F508000D46044617461E46FFF742FA0020FFF74D
:10F518005FFB204600F0BEFD00240123CDE908432F
:10F5280003234FF4167229462046CDE90644CDE957
:10F538000444CDE90244CDE900532346FFF774FEA5
:10F548002046FFF77DFAFFF735FAF3F7D1FA01F015
:10F5580043FC0446204601F049FCB04205D301248F
:10F56800FFF716FA20460BB0F0BD00F02FFF00B2EF
:10F578008742EFDA0024F3E7F7B500230C4640F2A0
:10F5880001211A460646084600F01EFD644B654DEB
:10F598004FF400529A6195F85600012100F09CFF43
:10F5A8002B78012B40F6890013D195F85130062BA2
:10F5B8000FD100F0D1FA00F0FB0140F6890000F00D
:10F5C800BBFA2B78042B6CD8DFE803F0524B527F40
:10F5D800090000F0C1FA40F00401C9B2EDE7524A4F
:10F5E800731E1046C6F101074FF0000CF9188C4243
:10F5F8006FDC0022E7001346BA4271D19A0142EA51
:10F60800C3125B0183F020031343661C0355F6B253
:10F6180002234648AB73AE7600F056FE0021F12077
:10F6280000F08AFA0021F02000F086FAAB6C642B17
:10F6380070D17021F32000F07FFA1D21F22000F034
:10F648007BFAE1008C1CF420090A00F075FA04F03A
:10F65800FE01F52000F070FA33486FF07F42314622
:10F668001DE0EC77314800F02FFE0022214615E01E
:10F6780001F008F80128074625D121460DF10702B7
:10F68800304601F004F80446A0B99DF80730274831
:10F69800AB7500F019FE9DF807102246304600F0C1
:10F6A80065FB6968224801F063FC214801F026FCEB
:10F6B800002006E01F4B3A460021022001F0A2F884
:10F6C800032003B0F0BDAC75CCE70223AB73AC7676
:10F6D800C8E713F8011FC943197002F801CB85E781
:10F6E800D1106FEA020C715C0CF0070C013241FA80
:10F6F8000CF101F001014FEAE20C4B40D14310F844
:10F708000CE001F0070103FA01F141EA0E0100F8EB
:10F718000C1071E7E121F32000F00EFA04218DE7C7
:10F72800000400489C1D0020801C0020AA1D002009
:10F73800F81D002050240108F0B5BDF814409DF8CC
:10F7480018709DF81CE09DF8205040B1012814D095
:10F758000122002398180138B0FBF2F0F0BD87F0C1
:10F768000107E30003EBC70318330EEB450503EB72
:10F77800C5034FF47A714B43ECE7501F012803F19E
:10F78800040302D80C2C38BF0C24D1B9A2F10B0CFD
:10F79800BCF1010F8CBF4FF0000C4FF0010C280199
:10F7A800002F00EBCE0014BF00251425A0EB82002B
:10F7B800062A4FEA82062844A2F102070DD83546E8
:10F7C80010E0012906D1A2F10C00D0F1000C4CEB9D
:10F7D800000CE4E74FF0000CE1E70830BCF1000F43
:10F7E800EDD0BD000028ACBF2E182E1C701E90FB5B
:10F7F800F5F003FB0044094B062A5A5C8CBF0C3415
:10F808000E340A2A09D8A30001334FF47A71BB4099
:10F818004B43034951F822209CE7FFDEAE24010840
:10F82800B424010808B5094B012193F8560000F0EB
:10F8380053FE4FF4D7602D2100F07EF900F033FB22
:10F84800BDE80840024800F07BBA00BF9C1D0020BC
:10F85800FFFF0F0073B5A44CB4F854300025202BDB
:10F868008DF80350019500F01B8114D8082B0DD892
:10F878007BB1013B072B0CD8DFE813F042005B009B
:10F888000B00CD000B000B000B00FD00102B00F04F
:10F89800008102B070BDB3F5807F00F0988011D868
:10F8A800402B00F01081802BF3D1284600F032FA6B
:10F8B8008E4B1B68002BECD09B69002BE9D02846A7
:10F8C8009847E6E7B3F5007FE3D1894B0122294643
:10F8D800022000F097FF00F029F9042840F0858005
:10F8E800844B85484FF400529A6201F0B9FA2846D1
:10F8F80000F010FA7D4B1B68002BCAD05B6814E03F
:10F908007C4B7D484FF400529A6201F0A9FA00201E
:10F9180000F000FA00F0B8FE012801D100F0BDFEA9
:10F92800724B1B68002BB4D01B68002BB1D09847D2
:10F93800AFE7704B71484FF480529A6201F090FA29
:10F94800657895B9284600F0E5F9294640F6021091
:10F9580000F0F2F840F6441000F0FEF840F0020122
:10F96800C9B240F6441000F0E7F8FF220DF1030198
:10F9780063485E4D00F05AFD624800F071FD2B6847
:10F98800002B86D09E68002E83D094F82430012B5B
:10F9980008D194F9313094F930209DF80310584873
:10F9A800B04776E7E06B01A900F022FE019B9DF8C5
:10F9B800031053484FF47A7203F5FA7393FBF2F38A
:10F9C8002A685BB2956894F92920A84761E7284618
:10F9D80000F0A0F9454B1B68002B3FF45AAF9B6918
:10F9E800002B3FF456AF01206AE700F09FF8052886
:10F9F8007FF44FAF3F4B41484FF480529A6201F079
:10FA08002FFA284600F086F9384B1B68002B3FF484
:10FA180040AFDB6889E700213B4B0122022000F060
:10FA2800F1FEA16D00293FF434AFC1F3074140F660
:10FA3800031000F081F894F8591040F6041000F013
:10FA48007BF894F8581040F6051000F075F840F669
:10FA5800021000F081F840F00101C9B240F602102E
:10FA680000F06AF8002340F262211A460846A365AE
:10FA780000F0AAFA0DE7254B01220021022000F030
:10FA8800C1FE00F0FFFD01287FF403AF00F006FE81
:10FA9800FFE61F4B01220021022000F0B3FEF8E62A
:10FAA800164801F0DDF9607808B900F033F90F4B1A
:10FAB8001B68002B3FF4EDAEDB68002B3FF4E9AE8A
:10FAC8009847144BE6E7144B01222946022000F020
:10FAD80099FE607808B900F01DF9044B1B68002BEB
:10FAE8003FF4D7AE1B6920E79C1D0020801D002035
:10FAF8006524010800040048F81D0020841D00202A
:10FB0800801C0020C01D00207924010882240108DF
:10FB18008C240108952401089E240108024BA3F8AF
:10FB28005400FFF797BE00BF9C1D0020014B1878BA
:10FB3800704700BF161E002007B501238DF8071077
:10FB48000DF1070201460348F7F786F803B05DF8A0
:10FB580004FB00BF4C03002007B5012301460DF14B
:10FB680007020448F7F7B1F89DF8070003B05DF8FD
:10FB780004FB00BF4C03002010B50446F4F728FD31
:10FB880001280CD140F62310FFF7E6FF00F0F90139
:10FB9800214340F62310BDE81040FFF7CDBF10BD4C
:10FBA80010B50C4B1B7804469BB94FF4D760FFF790
:10FBB800D3FFC4F3002100F0FE0001434FF4D760E7
:10FBC800FFF7BAFFE1B240F2B960BDE81040FFF7B5
:10FBD800B3BF10BD171E002010B51346EFF31084F5
:10FBE80072B60A4601460348F7F736F884F31088D8
:10FBF80010BD00BF4C03002008B5014608224FF491
:10FC0800D860FFF7E9FF002008BD000007B5074BE3
:10FC18001B7840BAADF804002BB9022201A940F2C2
:10FC2800BC60FFF7D9FF03B05DF804FB171E002086
:10FC380007B5074B1B7840BAADF804002BB9022270
:10FC480001A940F2BE60FFF7C7FF03B05DF804FBEF
:10FC5800171E002010B51346EFF3108472B60A463B
:10FC680001460348F7F731F884F3108810BD00BF48
:10FC78004C03002010B51346EFF3108472B60A4601
:10FC880001460348F7F713F984F3108810BD00BF45
:10FC98004C0300200A4601460020FFF7EBBF000096
:10FCA80010B51346EFF3108472B60A4601460348AE
:10FCB800F7F730F984F3108810BD00BF4C0300201B
:10FCC80010B51346EFF3108472B60A46014603488E
:10FCD800F7F736F884F3108810BD00BF4C030020F6
:10FCE80013B504460020F4F74DFC0220FFF744FF4B
:10FCF80004F0070401220DF1070184208DF8074064
:10FD0800FFF7DEFF024B00221A7002B010BD00BFE1
:10FD1800161E002007B501228DF807000DF1070116
:10FD28008020FFF7CDFF9DF80730002B034B0CBF59
:10FD3800012202221A7003B05DF804FB161E00208F
:10FD480007B5094B8DF8060004221A70030C8DF8CC
:10FD580004300322030A01A983208DF80530FFF738
:10FD6800AFFF03B05DF804FB161E002010B5144663
:10FD7800FFF790FF2046BDE81040FFF7E1BF000005
:10FD880007B5094B8DF8060005221A70030C8DF88B
:10FD980004300322030A01A982208DF80530FFF7F9
:10FDA8008FFF03B05DF804FB161E002073B5002614
:10FDB80040F6E2000196FFF7CFFE00F0FE0105468F
:10FDC80040F6E200FFF7B8FE40F6E500FFF7C4FE94
:10FDD80000F07F01044640F6E500FFF7ADFE6FF046
:10FDE8007F40FFF7CDFF04220DEB020140F619001A
:10FDF800FFF730FF3046FFF78DFF294640F6E20057
:10FE0800FFF79AFE214640F6E500FFF795FE0198B8
:10FE180002B070BD13B50C4B04460522972140F67D
:10FE2800AC001A70FFF788FE230C8DF8043003220B
:10FE3800230A01A982208DF805308DF80640FFF7C6
:10FE48003FFF02B010BD00BF161E002007B5030C0F
:10FE58008DF80030030A8DF801300B0C49BA8DF883
:10FE68000200ADF804100622694694208DF803308C
:10FE7800FFF726FF024B06221A7003B05DF804FB59
:10FE8800161E0020002208B51146C520FFF718FFEE
:10FE9800014B07221A7008BD161E002000221146C9
:10FEA800D120FFF70DBF00221146D220FFF708BF6F
:10FEB80007B501228DF807000DF107019F20FFF714
:10FEC800FFFE03B05DF804FB07B501228DF80700BB
:10FED8000DF10701A020FFF7F3FE9DF807103F2959
:10FEE80007D901F0F8010131C9B240F20670FFF7F5
:10FEF80023FE03B05DF804FB07B5F4F769FB431E66
:10FF0800584258418DF8070001220DF1070196204B
:10FF1800FFF7D6FE03B05DF804FB07B500F07F00DD
:10FF28008DF8070001220DF107018920FFF7C8FEAF
:10FF380003B05DF804FB0000154B984207B51BD8C9
:10FF4800144B98421BD8144B98421BD8134B984219
:10FF58001BD8134B984295BF29226B222B236F2362
:10FF68008DF8042001A9022298208DF80530FFF7AA
:10FF7800A7FE03B05DF804FBE122E923F0E7D722EE
:10FF8800DB23EDE7C122C523EAE775228123E7E7F2
:10FF980000E9A43580F8A9328044E52D000B6B1BDD
:10FFA80040FC541907B58DF8062004228DF804008A
:10FFB8008DF8051095200DEB02018DF80730FFF73D
:10FFC8007FFE03B05DF804FB07B552BAADF8042014
:10FFD80040BA082249BAADF80000ADF802105BBA81
:10FFE80069461046ADF80630FFF76AFE03B05DF8C3
:08FFF80004FB07B50B0C042209
:020000040801F1
:1000000000F0070049BA8DF80400ADF806109720FB
:100010000DEB02018DF80530FFF756FE03B05DF8D9
:1000200004FB000010B508B1194B1860F2F764FC2E
:100030000220FFF7A5FD0024164B20461C70FFF799
:100040006DFEF4F7C7FA012817D14FF42071FFF7BE
:10005000D4FF40F611102146FFF772FD4FF07F00EC
:10006000FFF75FFF0E2140F61F10FFF769FDF4F761
:1000700059FA094B01221A7010BD102140F61110D7
:10008000FFF75EFD102140F61210FFF759FDE9E77A
:10009000181E0020141E0020161E002037B50C4D1F
:1000A0002B7804461BB9FFF74BFF01232B7000236D
:1000B000084A6006E109F1F72BFD042200BA01901D
:1000C0000DEB02018620FFF7FFFD03B030BD00BF3E
:1000D000141E00200048E80107B5094B8DF8070001
:1000E0000146187018B940F2AC60FFF729FD0122F3
:1000F0000DF107018A20FFF7E7FD03B05DF804FB6F
:10010000171E0020012873B50C46164637D1002073
:10011000F4F764FAA042B8BF44B20E2805461AD1DB
:1001200001231A4600210420FFF740FF6FF010035F
:100130009C42B8BF1C46182140F6E700FFF700FDBF
:10014000022201A98E208DF804408DF80560FFF78A
:10015000BBFD02B070BD01230A28E4B21A464FF07D
:10016000000105D11846FFF721FF033464B2DDE733
:100170000720C5F10E05FFF719FF2C44F6E740F6FE
:10018000D800FFF7EDFC40F01E01C9B240F6D800E0
:10019000FFF7D6FC0120F4F721FAA042B8BF44B221
:1001A000142805464FF001034FF000020CD1052141
:1001B0000320FFF7FBFE023464B26FF008039C4299
:1001C000B8BF1C463821B7E7112805D1032102200A
:1001D000FFF7ECFE0534EFE70E2804D102210846B4
:1001E000FFF7E4FEE9E7C5F11605072104202544E1
:1001F000FFF7DCFE6CB2E0E713B5314A0446516804
:1002000010686B4603C32F4B20781B78834201D0C4
:10021000FFF762FF2378032B27D8DFE803F00239CA
:10022000283C6268284BB3FBF2F31A0CA1688DF8E6
:1002300000208DF802301A0A237B8DF80330637B8F
:100240008DF801208DF80430204A00234806C909A2
:10025000F1F75EFC030C40BA8DF80530ADF80600EE
:10026000082269468B20FFF72FFD02B010BD2269DE
:10027000154BB3FBF2F31A0C8DF800208DF8023009
:100280001A0A237D8DF801208DF803300422E8E757
:10029000A3690093FAE762680B4BB3FBF2F31A0C05
:1002A0008DF800208DF802301A0A237B8DF8033078
:1002B000637B8DF801208DF804300522D1E700BF63
:1002C00090140108171E00200000093D0048E801B5
:1002D0001FB52E4A0446D1689068127C01AB03C357
:1002E0001A702B4B20781B78834201D0FFF7F4FE65
:1002F0002378032B26D8DFE803F002383302637A31
:10030000F12B21D14FF6FF70FFF784FC48F2050076
:10031000FFF792FC02236288A188ADF8061052BA5A
:10032000E188ADF804208DF80B30227AA37A8DF89D
:100330000A20ADF808108DF80C30092201A98C2094
:10034000FFF7C2FC04B010BDF22BE4D141F60F5010
:10035000FFF760FC41F22100FFF76EFC0623DAE7AD
:10036000237B8DF804300122E8E7E389094A5BBA70
:10037000ADF80430237C13708DF80630637C8DF863
:100380000730638AADF808300622D7E790140108D9
:10039000171E0020151E002007B502228DF804004C
:1003A0008DF805108F2001A9FFF78EFC03B05DF8D2
:1003B00004FB000010B51346EFF3108472B60A4632
:1003C00001460348F6F7F8FC84F3108810BD00BF1F
:1003D0004C03002007B5012201A91520FFF7EAFF11
:1003E0009DF804004042401003B05DF804FB00009B
:1003F00037B505460C46022201A91320FFF7DAFFA4
:100400000A4B1B78012B0DD1094B1B78012B09D10D
:1004100040F20270FFF7A4FB9DF8053028702370AE
:1004200003B030BD9DF80400F6E700BF171E0020A2
:10043000151E0020F7B50D46064600240DF10701F4
:10044000284617468DF80740FFF7D2FF2A78BA42B0
:1004500007D89DF807003146FFF726FC204603B079
:10046000F0BD0120FBE7000013B50322044601A9FB
:100470001420FFF79FFF184B1A7822704AB1012A07
:1004800017D014220021204600F0D2FA0F23237047
:100490000DE09DF8043023719DF80530A2605B42A9
:1004A0005B10A3719DF806305B425B10637102B074
:1004B00010BD9DF804305B425B1023739DF905303D
:1004C00002339B1063739DF806305B425B10A3738D
:1004D000024B1B682361EAE7171E0020101E002054
:1004E000012908B5034608460ED1012B07D1042087
:1004F000FFF746FB0220BDE80840F4F747B8022B9F
:1005000014BF08460320F6E70120F4E738B5044697
:10051000F4F75EF850B1022814BF012502252846E1
:1005200002222146FFF7EEFD284638BD0F2CCCBF36
:1005300002250125F3E70A2070470000014B012046
:100540001B681847181E0020014B02201B68184723
:10055000181E0020014B40201B681847181E002061
:1005600011B1012904D07047044B1B688020184743
:10057000024B4FF480701B68F9E700BF181E002083
:10058000024B4FF400701B68184700BF181E002074
:10059000014B20201B681847181E0020014B042027
:1005A0001B681847181E0020014B08201B681847BD
:1005B000181E0020014B10201B681847181E002031
:1005C000024B4FF480401B68184700BF181E0020E4
:1005D00068B1084A002352F83310814203D902EB74
:1005E000C302107970470133162BF4D1FEE71F20A8
:1005F000704700BF7025010873B51D4B0193044679
:1006000040F607000D46FFF7ABFAC0F3C10308330D
:100610006B4413F8042C00F00703013302FA03F3D0
:10062000144AB2FBF3F2B2FBF4F007281ED84000E4
:1006300003288CBF022304234FF4D66002FB03F48B
:10064000FFF78EFA060240F2B160FFF789FA06F46E
:1006500070663043030544BF6FEA00506FEA1050E4
:1006600063094343DB112B6002B070BD0123E3E754
:1006700004080A0C0048E8014FF0FF3070474FF0C3
:10068000FF3070474FF0FF307047704700207047D1
:100690000020704770474FF0FF3070474FF0FF3039
:1006A000704770477047704770B5EFF3108672B6A9
:1006B000144B5C8A1A8A944213D1C4F5806292B2B8
:1006C000904206D3844218D901229A7000221C80DD
:1006D0005A825A8A0A800244C2F309025A820020CE
:1006E0000DE006D9C4F58065ADB28542F1D88242ED
:1006F000E9E7121B92B28242EBD84FF0FF3086F34B
:10070000108870BD1C220020EFF3108172B6034ADE
:10071000D38A0133D38281F3108870471C220020D2
:10072000EFF3108172B6034AD38A013BD38281F37F
:10073000108870471C22002010B50848182200219C
:1007400000F076F906484FF48062002100F070F95D
:10075000044B05481B68BDE8104018471C220020C8
:100760001C1E002050150108D9080108014B5860D3
:10077000704700BF1C220020014B1872704700BF59
:100780001C22002073B5EFF3108572B61C4CE08A72
:1007900000282FD1FFF7B8FF218A628A914227D023
:1007A000A378012B12D1238820805B1A9BB20221EF
:1007B000A382A17063B9A3702382238A9A428BBF5C
:1007C000D21AC3F58063A282A38201E0002BF4D089
:1007D000238A0C4E1E4485F31088F2F77BF90A4BEE
:1007E000A18ADB680193304602B0BDE8704018472B
:1007F000FFF796FF85F31088002002B070BD00BFA0
:100800001C2200201C1E00205015010808B4F0B561
:1008100086B00023ADF800302C4B0B9C1D7A85422E
:100820004DD3D86881434DD15B681BB112B1694685
:1008300002A898470CAB22464FF40071244801935C
:1008400000F0F6FBFFF760FFBDF8003018440DF133
:10085000020180B2FFF728FF01302BD00022BDF843
:100860000030BDF802701B480DF1080C164691B21D
:1008700017FA82F58B42ADB216D83B449BB20EB14B
:10088000ADF80230BDF80250019B22464FF40071D2
:10089000284400F0CDFBFFF743FFFFF773FF06B0DE
:1008A000BDE8F04001B070471CF8011B4155013212
:1008B0000126DCE7FFF734FF6FF00200EFE76FF08F
:1008C0000400ECE76FF00500E9E700BF1C22002000
:1008D000342200201C1E002013B5EFF3108472B6E2
:1008E000204B9A78588A022A1DBF1A8A998A521870
:1008F000002214BFC2F309029A7090421A8228D0D3
:10090000D98A012925D19978012913D119888A1A00
:10091000022192B2997000219A82198062B99A706C
:100920001A821A8A90428BBF801AC2F5806298821E
:100930009A8201E00029F4D01A8A0B48104484F30B
:1009400010880A4A998AD368019302B0BDE8104022
:10095000184784F31088F2F7C1F802B0BDE81040E0
:10096000FFF7DEBE1C2200201C1E002050150108CF
:10097000024A00231360024A1360704738240020A3
:100980003424002010B5EFF3108472B641B1012970
:1009900003D1064A13680343136084F3108810BD23
:1009A000024A136823EA0003F6E700BF3824002058
:1009B00010B5EFF3108472B641B1012903D1064A94
:1009C00013680343136084F3108810BD024A136850
:1009D00023EA0003F6E700BF3424002038B5EFF324
:1009E000108572B60A4B0B4C1B6833B123689847CD
:1009F0006368984785F3108838BD074B1B681BB1A7
:100A0000A3689847E368F4E7236998476369F0E7C8
:100A100038240020BC1401083424002001380A4482
:100A2000914200D1704711F8013B00F8013FF7E710
:100A300000F02CBC10B5EFF3108472B6064A1368B0
:100A400003431360054A52F83130034342F8313012
:100A500084F3108810BD00BF88240020802400206B
:100A600070477047030C1B04C3B90004102310F037
:100A70007F4F02BF08330002DBB210F0704F08BF97
:100A800000014FEA1070064A08BF0433125C08BF29
:100A9000DBB2C3F11F03981AC0B270470023E6E728
:100AA000202601082DE9F84F384D394ED5F8008041
:100AB000DFF8E0B0DFF8E0A0DFF8E090D6F800C0A3
:100AC000374FDBF80010374CDAF80020D9F8003047
:100AD00008EA00002860286800EA020E1EEA0C0FEF
:100AE00001D019421ED04FF0FF333B60FFF7B8FF33
:100AF000EFF3108472B63368DBF80020DAF80010E8
:100B00000B4029680B4205D1D9F80030134201D1BE
:100B1000F1F76EFF84F31088FFF7A3FFC5F800809C
:100B2000BDE8F88F236823680340134062681A42C7
:100B300004BF4FF0FF32626060681840FFF792FF19
:100B400062683860012303FA00F022EA0002626062
:100B5000EFF3108172B63A689340326822EA0302DA
:100B60003260226822EA0303236081F310880E4A70
:100B70003B6852F823309847D6F800C0DBF80010E5
:100B8000DAF80020D9F80030A5E700BF44010020C2
:100B90008824002040240020480100204424002014
:100BA0003C240020802400204824002010B5114659
:100BB000EFF3108472B6FFF755FF034B43F8201094
:100BC00084F3108810BD00BF4824002082B082B09A
:100BD0000DF1080C0CE90600BDF8042003930B444A
:100BE000BDF810100A4491B212B2B2F57A7FA2BFDA
:100BF000A1F57A72013312B20360828002B002B0B2
:100C0000704782B082B00DF1080C0CE90600BDF807
:100C100004200393CB1ABDF81010521A91B212B2ED
:100C2000002ABEBF01F57A7203F1FF3312B20360EE
:100C3000828002B002B0704730B585B0114D6B466E
:100C400083E8030000230293ADF80C3003A82B695E
:100C50009847009BBDF804400290181ABDF80C306C
:100C6000E41AA3B224B2002CBEBF03F57A731CB2FF
:100C700000F1FF302B689847AB682046984705B0D5
:100C800030BD00BF1015010873B5114E0023054695
:100C90000093ADF8043001A833699847F3680090D9
:100CA0009847736804469847009B1844BDF8043081
:100CB00023449AB21BB2B3F57A7FA2BF0130A2F5EA
:100CC0007A731BB228602846AB8002B070BD00BFAB
:100CD0001015010837B500230093ADF80430074B19
:100CE00004461B6901A898476D46009095E80300EB
:100CF00084E80300204603B030BD00BF1015010892
:100D000037B50F4D02AB03E90300EB6898476B68FA
:100D100004469847BDF80430009A1B1B99B21BB2D9
:100D2000002BA2EB0002BEBF01F57A7102F1FF3287
:100D30000BB24FF47A7000FB023003B030BD00BF3D
:100D4000101501082DE9F0414FF47A75B1FBF5F566
:100D5000C5EB4513DFF83C8005EB8303A1EBC30330
:100D60009CB2D8F80C3006469847D8F804300746AD
:100D70009847E31999B21BB2B3F57A7F2844A2BF12
:100D8000A1F57A7301301BB23060B3803046BDE804
:100D9000F08100BF10150108024B00221A60024BBF
:100DA0001B6818478C24002024150108F8B5044658
:100DB000174608461E467CB173B1084B00255B6A96
:100DC00025609847069B60602581A572E6602361D7
:100DD000E77265612846F8BD0120FCE7241501088B
:100DE00010B5034CE3699847A36ABDE81040184763
:100DF0002415010870B5064DEB69064698476B6AE5
:100E0000044630469847AB6A201ABDE87040184740
:100E100024150108054B1B680BB91846704783421F
:100E200001D05B69F8E70120704700BF8C240020E7
:100E30002DE9F3410B4E336A044698470123B76905
:100E40002372D4F800800546B8472844804502D272
:100E5000B84728442060B3682068019302B0BDE819
:100E6000F04118472415010870B520B3EFF3108640
:100E700072B6124D2B680122827253B10022427267
:100E800098425C690ED102723CB120462C60FFF79B
:100E9000CFFF86F31088002070BD094BDB689847B0
:100EA0002C60F6E71A465B69002BF2D09842F9D124
:100EB00043695361EDE70120EEE700BF8C24002079
:100EC00024150108084B10B51A685369516911B906
:100ED0005061416110BD046819688C4202D91A46FC
:100EE0005B69F3E71946F3E78C240020044A136892
:100EF0000BB10021197243611060FFF799BF00BF69
:100F00008C2400202DE9F041044600282DD0FFF765
:100F100081FF50BB657A45BBEFF3108872B6144E63
:100F20006768336A984787422CBF27602060114F5B
:100F3000A5724FF4807323813B684BB9336998479E
:100F40002046FFF7D3FF88F310882846BDE8F081DC
:100F5000B3699847236818443B6820601B6898422F
:100F60002046EED3FFF7AEFFEDE70125EDE700BF2A
:100F7000241501088C24002010B5044608467CB1D5
:100F8000084B5B6A984760602046FFF743FF40B11B
:100F90002046FFF769FF2046BDE81040FFF7B2BFCB
:100FA000012010BD241501082DE9F041EFF3108751
:100FB00072B61D4E1D4D73699847336904469847B4
:100FC0002B684BB94FF000082B688BB9286828BBF9
:100FD00087F31088BDE8F081011B241A1A688A4241
:100FE0008CBF121900221A605B69002BF6D1E9E769
:100FF0001C681CB1B36998478442E7D22C686369C6
:101000002B60A4F80880D4E9033098476389B3F5CE
:10101000807FD9D12046FFF775FFD5E7037A002BF3
:10102000D6D1FFF705FFD3E7241501088C24002053
:101030002DE9F04F97B000298046039140F30E81CF
:101040009A46044603991378A4EB0800013923B9A2
:101050000023237017B0BDE8F08F8842F8DA252B03
:1010600004D004F8013B1646721CEBE792F801C06D
:10107000ACF13003D3F1000E4EEB030EACF13003B4
:10108000092B02F1010629D8324600254FF00A0942
:10109000164612F8013BA3F13000092819D933781C
:1010A000692B00F09C801CD8632B28D0642B00F0A7
:1010B0009680582B5BD0252B19D13378002B00F06C
:1010C000928004F8013BA4EB08038B4280F28980F4
:1010D000CAE709FB0533A3F13005D9E74FF0FF3527
:1010E000DDE7752B7DD0782B43D0732B1ED02523C5
:1010F00004F8013BA4EB08038B4272DADDE7002D14
:1011000005F1FF39D8BF4FF000094A46204620219B
:1011100000F0BCF85346A144002D53F8042B89F885
:101120000020D8BF01252C449A469DE74C4B5AF825
:10113000047B002F08BF1F463846F0F741F9A5EBA6
:10114000000B8542B8BF4FF0000B5A468146202164
:10115000204600F09BF8A34400234B4502DB0BEB39
:10116000090481E7FA5C0BF803200133F5E74EF040
:10117000400E1020DFF8EC903B4F1EF0400F08BFF0
:101180004F465346BCF1300F0197A4EB08020CBF49
:10119000302720271EF0020FA1EB0202029753F81E
:1011A000041B22D0002920DA4942013D4FF02D0EC8
:1011B00005AF009700278946DDF804A0B1FBF0F1E8
:1011C00000FB119B48451AF80BB0DDF800A00AF8A7
:1011D00001BB07F10107CDF800A0ECD90EE04EF0FD
:1011E000020E0A20C6E7013E6DE711B14FF0000E76
:1011F000DEE730208DF814008E460127BCF1300F59
:10120000A5EB070504D02020002D05F1FF3509DCF2
:10121000BEF1000F04D02D21013A04F8011B83D048
:1012200025440AE0013A04F8010BEDD17CE702996C
:1012300004F8011B013A3FF477AF291B0029F6DCC3
:1012400005A9394422442744A7423FF46DAF11F861
:10125000010D04F8010B9442F6D165E70020F9E690
:1012600030260108372601085C26010810B501392F
:101270000244904201D1002005E0037811F8014FAB
:10128000A34201D0181B10BD0130F2E7024403460F
:10129000934200D1704703F8011BF9E770B50D4D7B
:1012A0000D4C641BA4100026A64209D10B4D0C4C1A
:1012B00000F0B2F8641BA4100026A64205D170BD50
:1012C00055F8043B98470136EEE755F8043B98473C
:1012D0000136F2E764270108642701086427010842
:1012E0006827010800F003B8002200F00EB80A4495
:1012F000914200F1FF3300D1704710B511F8014B56
:1013000003F8014F9142F9D110BD13460A46194620
:10131000FFF7BCBF00000000C1F30A522DE9F843FB
:10132000A2F2FF36132E0B4607460C46054632DC6A
:10133000002E14DA34A3D3E90023F0F74FF800228B
:101340000023F0F77FFA38B1002C56DA24F000447D
:10135000254355D02E4C002523462F4625E02D4A07
:1013600042FA06F801EA080202431ED026A3D3E996
:101370000023F0F733F800220023F0F763FA002887
:10138000EAD0002CBEBF4FF480133341E41824EAA6
:1013900008040025E0E7332E0BDDB6F5806F04D19D
:1013A0000246F0F71BF807460B4638461946BDE8DB
:1013B000F883A2F213424FF0FF3828FA02F810EA3D
:1013C000080FF2D010A3D3E90023F0F707F80022AA
:1013D0000023F0F737FA0028BED0002C0ADA142ECA
:1013E00001D1013406E0C6F134060123B3401D44A7
:1013F000AF42F6D825EA0805AEE700252C46ABE754
:101400004FF00044A8E700BF9C7500883CE4377E9D
:101410000000F0BFFFFF0F00F8B500BFF8BC08BC2C
:101420009E467047F8B500BFF8BC08BC9E467047A2
:1014300000000000010000000200000000000000A9
:101440008813000010270000204E000030750000B7
:10145000409C000050C3000060EA0000C0D40100BE
:1014600080A903000053070000EA063700000000CF
:101470005000000040F70937000000005000000055
:10148000C194C10000000000B2270000000000006D
:10149000000000000000000000000000000000004C
:1014A00000000000B5010008F1010008A4140108C3
:1014B000FC7F003F00350113C41200089F2700087D
:1014C0008127000865270008852700086127000894
:1014D000B12700080D0A484D4143205665726966E0
:1014E000792053756363657373203D202575200D46
:1014F0000A005975336E3148344F3152354E3953E5
:1015000032543653256473253033643A00000000AA
:10151000A12C0008412D0008B12C00084D2D000819
:10152000112D0008592D000800000000C12C0008F2
:10153000792C0008452C0008FD2B0008552C0008CC
:10154000692C0008092C00080D2C0008212C00082B
:101550000130000829300008AD2F0008992F00083D
:10156000496E697469616C20414320434F444520B2
:10157000626C616E6B2E2E2E200D0A005354535F49
:10158000534552564943455F4D41534B3A256420DC
:101590000D0A000D0A202D2D2D2D2D2D2D2D2D2D3B
:1015A0002D2D2D2D2D2D2D2D2D52464143205072A8
:1015B0006F636573730D0A0052464143000D0A20A4
:1015C0002D2D2D2D2D2D2D2D2D2D2D2D2D2D2D2D4B
:1015D0002D2D2D5665726966792052464143205360
:1015E000756363657373206F72204E6F740D0A000C
:1015F00020202B2B2B20204C6971756964204465B9
:101600007465637465640020202D2D2D20204E6F9D
:10161000204C6971756964000D0A205036205465AC
:101620007374696E672050726F636573730D0A007F
:101630000D0A20536F6170205374617465203D2042
:101640002573200D0A0053776974636820746F2036
:10165000436C61737320256320646F6E650D0A000F
:10166000414243000D0A205478506572696F6469E5
:1016700063697479206368616E67656420746F20A4
:10168000257520286D73656329200D0A002A2A2AF2
:101690002A2A2A2A2A2A2A2A2A2A2A2A2A2048655B
:1016A00061727442656174506572696F64696369DF
:1016B0007479204368616E67656420746F3A2025F1
:1016C0007520286D73290D0A00414250004F544186
:1016D00041000D0A232323232323203D204A4F4981
:1016E0004E4544203D2000414250203D3D3D3D3D82
:1016F0003D3D3D3D3D3D3D3D3D3D3D3D3D3D3D3D1A
:101700003D0D0A004F544141203D3D3D3D3D3D3D95
:101710003D3D3D3D3D3D3D3D3D3D3D3D3D3D0D0A5C
:10172000000D0A205354535F4C6F52615F57414E76
:101730005F4A6F696E6564203D202573200D0A00A5
:101740000D0A232323232323203D204A4F494E20E3
:101750004641494C45440D0A0023232323232320DB
:10176000552F4C204652414D453A4A4F494E207C18
:101770002044523A2564207C205057523A25640D6B
:101780000A004C6D48616E646C65722053746F7012
:10179000206F6E20676F696E67202E2E2E0D0A0057
:1017A0004C6D48616E646C65722053746F70706527
:1017B000640D0A004C6D48616E646C65722073772D
:1017C0006974636820746F20414250206D6F6465B6
:1017D0000D0A0053454E4420524551554553540D72
:1017E0000A004E65787420547820696E20203A20D3
:1017F0007E2564207365636F6E642873290D0A006B
:101800000D0A23232323232320424541434F4E2007
:101810004C4F53540D0A000D0A2323232323232066
:10182000424541434F4E2052454345495645442089
:101830007C2044523A2564207C20525353493A2557
:1018400064207C20534E523A2564207C2046513A35
:101850002564207C2054494D453A2564207C204451
:101860004553433A2564207C20494E464F3A303256
:1018700058253032582530325820253032582530FE
:101880003258253032580D0A000D0A232323232312
:101890002320424541434F4E204E4F542052454352
:1018A00045495645440D0A004E564D204441544189
:1018B0002053544F5245440D0A004E564D2044418A
:1018C000544120524553544F5245440D0A004E4155
:1018D000434B000D0A232323232323203D3D3D3D7D
:1018E0003D3D3D3D3D3D204D4350532D436F6E6684
:1018F00069726D203D3D3D3D3D3D3D3D3D3D3D3DA4
:101900003D0D0A0023232323232320552F4C20465B
:1019100052414D453A25303464207C20504F52547A
:101920003A2564207C2044523A2564207C2050577C
:10193000523A256400207C204D534720545950458D
:101940003A00434F4E4649524D4544205B25735D56
:101950000D0A00554E434F4E4649524D45440D0A1F
:10196000004E564D204441544120555020544F20A4
:10197000444154450D0A004E564D204441544120E7
:1019800053544F5245204641494C45440D0A0023CB
:101990002320425554544F4E2D3120444554454345
:1019A0005445443A2020253264200D0A00505658F0
:1019B0005858000D0A496E697469616C20426F6F56
:1019C00074207769746820456D70747920436F6E58
:1019D0006669672C20466C6173682077697468209B
:1019E00064656661756C7420636F6E6669672E2E20
:1019F0002E2E0D0A000D0A0A0A2323232323205921
:101A0000554E484F524E5F5354535F46573A2564E4
:101A1000205357562564204857563A2564204D5484
:101A20004D3A25642E256420523A25642E25642ED5
:101A3000256420232323230D0A0A0A004150504C19
:101A400049434154494F4E5F56455253494F4E3AD0
:101A5000205625582E25582E25580D0A004D575F23
:101A60004C4F524157414E5F56455253494F4E3AA3
:101A700020205625582E25582E25580D0A004D5742
:101A80005F524144494F5F56455253494F4E3A20A9
:101A90002020205625582E25582E25580D0A004C5A
:101AA000325F535045435F56455253494F4E3A209B
:101AB000202020205625582E25582E25580D0A0066
:101AC00052505F535045435F56455253494F4E3A2B
:101AD00020202020205625582D25582E25582E25EB
:101AE000580D0A002159756E486F726E2053545379
:101AF0002052657669766521000D0A2059756E6859
:101B00006F726E20535453204E6F64652052657679
:101B1000697665202E2E2E200D0A003E3E3E3E3E6A
:101B20003E3E3E3E3E3E3E3E3E3E3E3E3E3E3E3ED5
:101B3000204D61736B203D205B2025303278205D85
:101B4000200D0A002323232323232059554E484FD9
:101B5000524E20506572696F6469636974792043DD
:101B600068616E67656420746F205B202564205D6A
:101B7000205365636F6E64730D0A002323232323B0
:101B8000232059554E484F524E2053616D706C6959
:101B90006E67204F722048656172742D42656174D2
:101BA00020496E74657276616C204368616E67656A
:101BB0006420746F205B202564205D205365636F73
:101BC0006E64730D0A000D0A20746C765F62756690
:101BD000202564203D2025303278206366672D3E25
:101BE000705B25645D3D25303278200D0A0023238B
:101BF00023232323205253532053696D706C652097
